:020000040800F2
:1080000010E10020A1810008A98100083DAA000814
:10801000AD810008AF810008B181000800000000B8
:10802000000000000000000000000000B381000814
:10803000B581000800000000B7810008B981000880
:10804000BB810008BB810008BB810008BB81000820
:10805000BB810008BB810008BB810008BB81000810
:10806000BB810008BB810008BB810008BB81000800
:10807000BB810008BB810008379900083F990008C0
:10808000BB81000847990008BB810008BB8100083C
:10809000BB810008BB810008BB810008BB810008D0
:1080A000BB810008BB810008BB810008BB810008C0
:1080B00091F10208BB810008BB810008BB81000868
:1080C000BB810008BB810008BB810008BB810008A0
:1080D000BB810008770003087F00030887000308BE
:1080E0009D9D0008BB810008BB810008BB81000882
:1080F000BB810008BB810008BB8100084F990008C4
:10810000BB810008BB810008BB810008BB8100085F
:10811000670003086F000308BB810008BB810008EB
:10812000BB810008BB810008BB810008BB8100083F
:10813000BB810008BB810008BB810008BB8100082F
:10814000BB810008BB810008BB810008BB8100081F
:10815000BB810008579900085F9900088F00030849
:10816000BB810008BB810008BB810008BB810008FF
:10817000BB810008BB810008BB810008BB810008EF
:10818000BB810008BB810008DFF810D000F058FC6C
:1081900000480047751E0308AFF3008010E100207F
:1081A0000648804706480047FEE7FEE7FEE7FEE791
:1081B000FEE7FEE7FEE7FEE7FEE7FEE729F102083D
:1081C000898100082DE9F0410024061B254671F144
:1081D000000605DA01240027D0EB070067EB010158
:1081E000161E73F1000605DA0027D2EB07020125FF
:1081F00067EB030300F0C1FA86460E4617469C461D
:10820000AC4204D00025D0EB050E65EB010624B18D
:108210000020D2EB000760EB030C704631463A4673
:108220006346BDE8F081202A06DBCB17203A41FAED
:1082300002F043EAE07306E041FA02F3D040C2F1F3
:108240002002914008431946704740EA01039B070A
:1082500003D009E008C9121F08C0042AFAD203E0BB
:1082600011F8013B00F8013B521EF9D27047421E43
:1082700012F8013F002BFBD111F8013B02F8013B42
:10828000002BF9D17047421C10F8011B0029FBD1CB
:10829000801A704730B505460020034600E05B1C9D
:1082A000934205D2EC5CC85C201A01D1002CF6D1B7
:1082B00030BD2DE9FE4F804681EA0300C00F0C4619
:1082C000009021F0004123F00045B8EB0200A941E5
:1082D00005D24046214690461C460B46024623F0F6
:1082E0000040104347D0270DC7F30A00C3F30A51DB
:1082F0000290401A019040286BDAC3F3130040F457
:10830000801B0098924620B10023D2EB030A63EB56
:108310000B0B01985946C0F14002504600F05EFA3E
:1083200006460D4650465946019AFFF77CFF10EB72
:1083300008006141002487EA115284EAE7731A4376
:1083400040D0009A62B3019A012A4FEA075215DC25
:10835000001B61EB02014FF0004202EA0752CDE937
:108360000042001C41F5801132462B4600F0EAFA2B
:1083700003B0BDE8F08F40462146F9E7001B61EBF2
:108380000201001C41F5801300185B412018A2F582
:10839000001747EB030140EAD570B6196D4111E0B3
:1083A0006D084FEA360645EAC0754FEA0752001BD2
:1083B00061EB0201001C41F5801149084FEA3000D1
:1083C0000019514132462B4603B0BDE8F04F00F092
:1083D000AABA0098012240000023D0EB020263EB0E
:1083E000E073009821464FEAE074B8EB000061EBBF
:1083F0000401E9E783F000435BE781F0004158E7BF
:108400002DE9FE4F81EA030404F0004421F000410D
:1084100000944FF0000B23F0004350EA01045ED0BB
:1084200052EA03045BD0C3F30A54C1F30A552C4447
:10843000A4F2F3340194A0FB0254C1F3130141F4FC
:108440008011C3F3130343F4801301FB024400FBC8
:10845000034E840A970A44EA815447EA8357A4FBEF
:10846000076802958D0A05FB07854FEA932C04FBEC
:108470000C542705029D4FEA065847EA1637B5EB1C
:1084800008056EEB070C870E920E47EA811742EA49
:108490008312A7FB0201B6EB0B0164EB00042B0D6A
:1084A00043EA0C335E1844EB1C50DA465146E7FBB6
:1084B0000201C5F313044FEA0B3343EA14534FEAA6
:1084C0000432019C43EA0603A4F10C040294009CCC
:1084D000CDE900B400F036FA03B0BDE8F08F00201B
:1084E0000146F9E72DE9F04D81EA030404F0004B61
:1084F00021F0004514464FF0000A23F0004150EAF5
:10850000050220D054EA01021DD0C5F30A570246E5
:10851000C5F31303C1F31300C1F30A5640F48015E9
:1085200043F48013A7EB0608101BD64608F2FD386B
:1085300073EB050002D308F1010801E092185B41DA
:10854000B8F1000F03DA00200146BDE8F08D0020ED
:108550004FF48011064684460EE0171B73EB0507A7
:1085600005D3121B63EB050306434CEA010C4908D3
:108570004FEA300092185B4150EA0107EDD152EA10
:10858000030012D082EA040083EA0501084305D003
:10859000101BAB4106D20122002306E000224FF05F
:1085A000004302E06FF0010253101AEB06004CEB9F
:1085B000085110EB0A0041EB0B01BDE8F04D00F053
:1085C000B2B9F0B4CA17CB0F50405140C61841F1B0
:1085D00000054FEAC372314628004FF0960303D0DE
:1085E000B623F0BC00F071B930460021F9E70EB5B2
:1085F000C10F80EAE0700844CA07002140F233430B
:108600008DE80E000A460B4600F09CF903B000BD51
:108610000EB540F2334102910021CDE900110A4626
:108620000B4600F08FF903B000BD3EB5CA17CB0F63
:10863000002450405140C0186141DA0740F23343F2
:108640000094CDE901232246234600F07BF903B0D4
:1086500030BD10B500F0004420F00040C20DC0F362
:10866000160040F400007F2A02DA0020014610BD07
:108670000021962A03DCC2F19602D04002E0963A2D
:1086800000F0ACF8002CF2D00023D0EB030063EB39
:10869000010110BD70B5C1F30A5201F0004500247C
:1086A000C1F3130140F2FF3341F480119A4201DA21
:1086B000002070BD40F233439A42A2F2334203DC01
:1086C000524200F09AF800E090402C43F1D0404232
:1086D00070BD70B5C1F30A5201F000450024C1F32A
:1086E000130140F2FF3341F480119A4202DA002074
:1086F000014670BD40F233439A42A2F2334203DC9A
:10870000524200F07AF801E000F068F82C43F0D013
:108710000023D0EB030063EB010170BD00F00042C9
:1087200030F000400AD0C10D01F56071C0F31600B1
:1087300042EA0151C2084007114370470020014638
:10874000704701F0004330B421F0004150EA0102CB
:1087500006D00A0DA2F56072C1F31301002A02DCF3
:1087600030BC00207047440F44EAC104C100E01847
:1087700030BC00EBC25000F09FB82DE9F05F054619
:10878000002092469B4688460646814640241BE0D0
:10879000284641464746224600F02FF853465A469F
:1087A000C01A914110D311461846224600F016F81F
:1087B0002D1A67EB01084F4622460120002100F0E8
:1087C0000DF817EB00094E41201EA4F10104DFDC77
:1087D000484631462A464346BDE8F09F202A04DB3E
:1087E000203A00FA02F1002070479140C2F12003C4
:1087F00020FA03F3194390407047202A04DB203A03
:1088000021FA02F00021704721FA02F3D040C2F1B0
:108810002002914008431946704700000FB400231E
:1088200000B589B00CA900910B996FF00042CB60A4
:108830001E4B06931E4B07930423CDE901321D4ABC
:10884000089202466B46002000F0A6F909B05DF8D8
:1088500014FB70B586B006464FF0FF300091CDE9AD
:108860000101002015460C4604903246694604A8D2
:10887000FFF7D4FF02460498211825B108B1084635
:1088800000E020462860049800280DD0002A02DD70
:108890000098884208D0081B0094CDE901043246B4
:1088A000694604A8FFF7BAFF06B070BDD18D000875
:1088B000EF8D0008658A00080029A8BF7047401C9A
:1088C000490008BF20F00100704710B4B0FA80FCE6
:1088D00000FA0CF050EA010404BF10BC704749B123
:1088E000CCF1200421FA04F411FA0CF118BF012193
:1088F00021430843A3EB0C01CB1D4FEA00614FEA73
:10890000102042BF002010BC704700EBC350104441
:108910000029A4BF10BC7047401C490008BF20F0CC
:10892000010010BC704710B5141E73F1000408DA82
:10893000401C41F1000192185B411A4301D120F023
:10894000010010BD2DE9F04D92469B4611B1B1FAE0
:1089500081F202E0B0FA80F220329046FFF73EFF4B
:1089600004460F4640EA0A0041EA0B0153465A46C4
:10897000084313D0114653EA010019D0C8F1400250
:108980005046FFF73AFF05460E46504659464246C6
:10899000FFF724FF084305D0012004E020463946B4
:1089A000BDE8F08D0020054346EAE0762C433743CE
:1089B0000A986305E40AA0EB08000022FD0A44EAD5
:1089C00047540A3002D500200146E9E70105101995
:1089D0006941DDE9084500196941BDE8F04DA2E7AC
:1089E00070B521F0004303430CD0C1F30A550024B5
:1089F000D5EB040564EB0403D617AD1AB34102DBD3
:108A00000020014670BD201841EB025170BD0000EE
:108A100030B5041E71F1000404DB4FF00044404205
:108A200064EB0101141E73F1000405DB1C464FF0DA
:108A30000043524263EB0403994208BF904230BDA9
:108A4000064C074D06E0E06840F0010394E807009B
:108A500098471034AC42F6D3FFF79AFBB0A6030850
:108A6000D0A60308C0B24FF4F05100F03BBA0000AA
:108A70002DE9FF4F087883B09946FF2805D0491C9F
:108A80002D2804D00024002008E000200BE0012461
:108A9000F9E700EB800003EB4000491C0B78FF2B4B
:108AA000F7D104B1404200230293147819461D46C1
:108AB0002D2C01D02B2C04D1521C2D2C13D0002492
:108AC0000294AA461478FF2C0FD00A25A3FB057840
:108AD00001FB05814FF0000C03FB0C11521CE31944
:108AE0004AEB0101EEE70124EAE7814453EA010081
:108AF00002D019F5C87F06DA03980021C0E90011F9
:108B000007B0BDE8F08F0025AE4E2F46DFF8B882E3
:108B1000184600F0FBF9CDE90001B9F1000002DAD6
:108B2000C9F1000400E004460023A74A1AEB030B36
:108B300042EB045A12E0E00707D02A463346384693
:108B40004146FFF75DFC074688462A4633461046F5
:108B50001946FFF755FC05460E466410002CEAD175
:108B6000DDE90001B9F1000F5A46534606DAFFF776
:108B7000B9FC3A464346FFF7B5FC05E0FFF740FC79
:108B80003A464346FFF73CFC029A0AB181F00041A5
:108B9000039AC2E90001B3E72DE9FF4F1F468DB0EC
:108BA000D7E901464FF0FF382E2045464FF0000927
:108BB0000B90B9696D1C0E988847396A82468847C0
:108BC0000028F6D1BAF1FF3F0AD024F4D064002E79
:108BD00011DDBAF12B0F08D0BAF12D0F0BD102E045
:108BE000404611B08DE744F48064B9696D1C0E985D
:108BF00088478246761E6946600501D52D2000E033
:108C00002B208DF8000001F1010B0DF1200809E087
:108C1000B9696D1C0E98884782460F9844F4007419
:108C2000761E0560002E02DDBAF1300FF0D00B99F0
:108C30008A453ED144F0800406E00F99681CA9F1F2
:108C4000010944F400740860B9696D1C761E0E9821
:108C5000884782463028F0D02BE00B998A4505D111
:108C6000200603D444F08004761E18E0504628F015
:108C70004DFD08B30DF11301761E44F400748B45CD
:108C800008D2AAF130000BF8010B200607D5A9F194
:108C9000010003E0200602D409F101008146A0058D
:108CA00002D50F99681C0860B9696D1C0E98884739
:108CB0008246002ED1DC53E0002E51DDBAF1650F63
:108CC00002D0BAF1450F4BD1A00549D5B9696D1C49
:108CD00024F44074761E0E9888478246002E0CDDE0
:108CE0002B2804D0BAF12D0F07D144F48074B96950
:108CF0006D1C0E9888478246761EE00501D52D2111
:108D000000E02B2108F8011BCDF82C8021E00DF1AB
:108D10002901761E44F4007488450CD2AAF1300073
:108D200010F0FF0088F8000002D10B99884509D99E
:108D300008F1010806E0E00501D5244801E042F20F
:108D40000F708146B9696D1C0E98884782460F984E
:108D50000560002E04DD504628F0D8FC0028D6D14E
:108D6000F9690E988847FF208BF8000088F800000A
:108D70000020069007904B466A4608A906A8FFF710
:108D800077FEA00502D46FF001002AE714F0240F4B
:108D90000AD0E00714D1DDE906123868031D3B60F4
:108DA0000068C0E900120BE0DDE90601FFF7C9FC2D
:108DB0000146E00704D13868021D3A60006801608E
:108DC00028460EE7000014400000F03FF1D8FFFFF6
:108DD000426842B1016811F8013B23B1521EC0E95B
:108DE0000012184670470121C160881E7047426812
:108DF0005AB1C368016843B983688B4205D0491EE4
:108E0000521CC0E90012002070474FF0FF3070473D
:108E10002DE9F04D00231A461B1A8A4103DB00207E
:108E20000146BDE8F08DC1F30A52C1F3130141F4CC
:108E300080154FF0000BD10702D100186D41521E72
:108E40000027044640F2FF11384601EB620A3E4615
:108E50008046024600204FF48011FFF7CEFCC21975
:108E60007141BB1846EB0100B4EB030C75EB000C31
:108E700004D3E41A65EB000517460E46241908F1E1
:108E800001006D4180463428E3DDF91946EB060008
:108E9000091BA84103D24FF0FF32134601E0002224
:108EA00013461BEB070046EB0A51BDE8F04DFFF7F8
:108EB0003ABD000030B5041E71F1000404DB4FF030
:108EC0000044404264EB0101141E73F1000405DB11
:108ED0001C464FF00043524263EB04038B4208BF31
:108EE000824230BD7F2801D9002208E0064A02EB09
:108EF0005002C007127800D1120902F00F020120BF
:108F0000904008407047000070A603080EB540F27C
:108F1000334202920022CDE900221346FFF712FDF0
:108F200003B000BD70B58C1810F8015B15F0070395
:108F300001D110F8013B2A1106D110F8012B03E0F2
:108F400010F8016B01F8016B5B1EF9D12B0705D4FA
:108F50000023521E0DD401F8013BFAE710F8013B43
:108F6000CB1A921C03E013F8015B01F8015B521E5F
:108F7000F9D5A142D8D3002070BD10B502461078B3
:108F800003E012F8014B2318D8B20B1EA1F1010423
:108F9000A1B2F6D110BD000070B5ADF5287D044634
:108FA0000D460020A790A690002604EB44004549FA
:108FB00001EBC000408AA84203DC00200DF5287DAB
:108FC00070BD0020A69077E004EB44003D4B03EB1E
:108FD000C000028A04EB440003EBC00080892844EF
:108FE00081B2394800F010F90020A79011E004EB9D
:108FF0004400344901EBC0004068BDF89C12405C5D
:1090000001A9BDF89C228854BDF89C02401C80B286
:10901000A79004EB44002B4901EBC000008ABDF887
:109020009C128842E3DC04EB4400264A02EBC000B9
:10903000008A401E81B201A8FFF79FFF23490870F4
:1090400004EB44001F4901EBC000008A401E01A947
:10905000085C1E490978884226D10020A79016E0B6
:1090600004EB4400174901EBC0004068BDF89C12B6
:10907000405C04EB4401134A02EBC1018968BDF86E
:109080009C228854BDF89C02401C80B2A79004EB3F
:1090900044000C4901EBC000008A401EBDF89C1240
:1090A0008842DDDC012089E7642028F067FDBDF8F7
:1090B0009802401C80B2A690BDF89802062883DB77
:1090C00000207BE76C7C03087C9A0020310A00209A
:1090D0002DE9F043ADF5257D04460E460025002719
:1090E000A846A94604EB4400324901EBC000408A7F
:1090F000B04204DC00200DF5257DBDE8F08300259D
:1091000018E004EB44002B4901EBC0008068405D8F
:1091100004EB4401274A02EBC1014968485504EBBE
:109120004400114601EBC0004068405D0DF80500A9
:10913000681C85B204EB44001E4901EBC000008AA4
:10914000401EA842DDDC04EB44000A4602EBC000EE
:10915000008A401E81B26846FFF70FFF04EB44010E
:10916000144A02EBC101098A491E0DF801000027CB
:109170001BE004EB44000F4B03EBC000028A04EB3E
:10918000440003EBC0008089304481B2684600F09F
:109190004FF931462046FFF7FFFE012800D1AAE72C
:1091A000642028F0EBFC781C87B2062FE1DB00205E
:1091B000A1E700006C7C030808B50020009022F0B5
:1091C00073FF0F49087000F09BF80D4800782428C1
:1091D00004D0272807D028280FD109E0002109480A
:1091E00080F8151E09E00121064880F8151E04E0EC
:1091F0000221044880F8151E00BF00BF08BD000012
:109200002C0A0020BC2200202DE9F04106460D4624
:1092100017460024012028F070FA00202849088011
:109220000DE022F023FF00F0800000B10BE00120F0
:1092300028F0A4FC22480088401C214908802048CE
:109240000088C828EDDB00BF1D480088C82832DA36
:1092500010211C4801F0E6FB08211A4801F0E4FB4C
:10926000E82000F031F8C5F3871000F02DF8A906CA
:10927000080E00F029F8002000F026F8002404E091
:10928000002000F021F8601C84B2042CF8DB0024DC
:1092900005E0FF2000F018F83055601C84B2BC4295
:1092A000F7DB1021074801F0BFFB002028F025FA6A
:1092B0000120BDE8F081002028F01FFA0020F8E727
:1092C0002E0A00200000024010B5044600BF022113
:1092D0000A4822F0F9FF0028F9D02146074822F079
:1092E000FFFF00BF0121054822F0EEFF0028F9D062
:1092F000024822F0F2FFC0B210BD00000030014071
:1093000010B5012028F0F9F900201E4908800DE071
:1093100022F0ACFE00F0800000B10BE0012028F04C
:109320002DFC18480088401C164908801548008804
:10933000C828EDDB00BF13480088C8281CDA1021BC
:10934000114801F06FFB08210F4801F06DFB3D2033
:10935000FFF7BAFF2A20FFF7B7FF8020FFF7B4FF1F
:10936000A720FFF7B1FF1021074801F05DFB0020A7
:1093700028F0C3F9012010BD002028F0BEF900201C
:10938000F9E700002E0A00200000024070B50546F3
:109390000E460024012028F0B0F900202249088060
:1093A0000DE022F063FE00F0800000B10BE0012030
:1093B00028F0E4FB1C480088401C1B4908801A4820
:1093C0000088C828EDDB00BF17480088C82825DAC8
:1093D0001021164801F026FB0821144801F024FB57
:1093E0008420FFF771FF0020FFF76EFF0020FFF7DA
:1093F0006BFF0020FFF768FF002404E0285DFFF703
:1094000063FF601C84B2B442F8DB1021074801F00E
:109410000BFB002028F071F9012070BD002028F01E
:109420006CF90020F9E700002E0A0020000002403D
:1094300070B506460C461546012028F05EF929460F
:109440003046FFF7A3FF08B9002070BD00201F4978
:1094500008800DE022F00AFE00F0800000B10BE071
:10946000012028F08BFB19480088401C1749088010
:1094700016480088C828EDDB00BF14480088C828BB
:109480001EDA1021124801F0CDFA0821104801F02F
:10949000CBFA8320FFF718FFC4F38710FFF714FF00
:1094A000A106080EFFF710FF0020FFF70DFF1021A7
:1094B000074801F0B9FA002028F01FF90120C4E79D
:1094C000002028F01AF90020BFE700002E0A002033
:1094D0000000024030B502460020002304E012F8EC
:1094E000014B60405C1CE3B28B42F8DB30BD0000F6
:1094F00010B50446392028F059FDE0B228F076FD79
:10950000C4F3072028F072FDC4F3074028F06EFD75
:10951000200E28F06BFD4FF48051034801F084FACF
:1095200026F0F8FE10BD0000000402402DE9F041D5
:1095300007460E4614463A2028F038FDF0B228F0CF
:1095400055FD301228F052FD4FF480510F4801F0C4
:109550006BFA19E026F0DEFE05461D2D11D13846C6
:1095600000F0ACF805463B2028F020FD4FF4805178
:10957000064801F059FA2F4434B12088284420804D
:1095800002E02846BDE8F081E4E700000004024064
:109590002DE9F04107460E4614463C2028F006FD12
:1095A000F0B228F023FD301228F020FD4FF4805156
:1095B000104801F039FA0CB10020208019E026F0A3
:1095C000A9FE05461E2D11D1384600F02BF905469F
:1095D0003D2028F0EBFC4FF48051064801F024FABE
:1095E0002F4434B120882844208002E02846BDE87A
:1095F000F081E4E70004024010B522F02FFC08B12E
:1096000000F02EF8302000F0A9F810BD10B5044687
:109610002146362000F08EF810BD10B5044614B176
:10962000204600F0ABF8342000F098F810BD10B5DB
:109630000446204600F0A2F820785C2802D020786A
:109640002F2803D10021642000F008F9322000F017
:1096500085F810BD10B5682000F04CF810BD000072
:1096600010B5222028F0A2FC28F095FC04464FF407
:109670008051024801F0D8F9204610BD0004024094
:109680002DE9F04128F087FC044628F084FC0546CB
:1096900028F081FC064628F07EFC07464FF48051F6
:1096A000054801F0C1F944EA052040EA064040EAD5
:1096B0000760BDE8F08100000004024070B5044678
:1096C000272028F073FC28F066FC0646054646B1C4
:1096D00000BF28F060FC2070641C701EC0B2061E23
:1096E000F7D14FF48051024801F09EF9284670BD31
:1096F0000004024010B504460C2028F057FC204618
:1097000028F074FCFFF7BCFF10BD000070B50446E4
:109710000A2028F04BFC204628F068FC28F03BFC8F
:1097200005464FF48051024801F07EF9284670BD8D
:109730000004024070B505460C46284628F036FC69
:10974000204628F053FC4FF48051034801F06CF997
:1097500026F0E0FD70BD00000004024010B5044694
:10976000204628F023FC4FF48051034801F05CF9B7
:1097700026F0D0FD10BD0000000402402DE9F041AC
:109780000646012028F012FC28F005FC43282BDABD
:109790002B20FFF7BBFF102826DA2F2028F006FC2D
:1097A000002028F023FC3220FFF7D8FF0446142CB9
:1097B0001AD1CF20FFF7AAFF0446ACB14C20FFF727
:1097C00099FF00EB042739464C2000F047F8502061
:1097D000FFF790FF00EB04273946502000F03EF8D9
:1097E0000021702000F03AF82F2028F0DFFB3578B8
:1097F000284628F0FBFB09E0761C35785C2D01D06B
:109800002F2D00D10025284628F0F0FB002DF3D1A4
:109810004FF48051024801F007F9BDE8F0810000E3
:109820000004024070B504462D2028F0BFFB28F04C
:10983000B2FB0646054646B100BF207828F0D6FBAD
:10984000641C701EC0B2061EF7D14FF4805102484E
:1098500001F0EAF8284670BD0004024070B50546E4
:109860000C460D2028F0A2FB284628F0BFFBE0B2F2
:1098700028F0BCFBC4F3072028F0B8FBC4F3074072
:1098800028F0B4FB200E28F0B1FB4FF480510248C1
:1098900001F0CAF870BD00000004024070B5024635
:1098A0000C46FF25FF2309E012F8010B80EA0501B1
:1098B0000648405C80EA03050548435C201EA4F18D
:1098C0000106B4B2F0D145EA032070BDCF79030898
:1098D000CF7A03082DE9F04103460C4600200146EB
:1098E000024606E013F8010B411842F10002601E27
:1098F00084B2002CF6DC080C40EA024C100C8DB24D
:109900001CEB050140F10002080C40EA024041183E
:109910006FEA010080B2BDE8F08130B50246002058
:10992000002305E012F8015B2C18E0B25C1CE3B2E6
:109930008B42F7DB30BD10B515F022FF10BD10B51E
:1099400015F0BCFE10BD10B515F088FE10BD10B5A9
:1099500015F0E4FE10BD10B517F080FE10BD10B577
:1099600021F05EFE10BD00000246094B9A4201D272
:10997000084801E00648103801F000531BB1064BBF
:109980000B40C36002E0044B0B4083607047000053
:1099900010640240006002407D0F7D0F21B102681B
:1099A00042F00102026003E0026822F0010202605C
:1099B00070470000016821F0010101600021016091
:1099C00041608160C1600161212141614A49884251
:1099D00004D13D21484A103A91608CE04649183143
:1099E000884205D14FF47461434A103A916082E095
:1099F00041493031884205D14FF474113E4A103A42
:109A0000916078E03C494831884205D14FF074615B
:109A1000394A103A91606EE037496031884204D18A
:109A20003649354A103AD16065E033497831884289
:109A300004D13349304A103AD1605CE02E4990316C
:109A4000884204D12F492C4A103AD16053E02A4968
:109A5000A831884205D14FF03D51274A103AD160D4
:109A600049E02949884204D13D21274A083A11603A
:109A700041E025491831884205D14FF47461224AEA
:109A8000083A116037E020493031884205D14FF45F
:109A900074111D4A083A11602DE01B494831884273
:109AA00005D14FF07461184A083A116023E0164955
:109AB0006031884204D11149134A121F11601AE023
:109AC00011497831884204D10D490F4A121F1160A3
:109AD00011E00D499031884204D10A490A4A121F07
:109AE000116008E00849A831884204D14FF03D5187
:109AF000054A121F11607047106002403D000020AF
:109B0000400F002000003D201064024010B501F01D
:109B100080034BB122B1436943F08003436103E00A
:109B2000436923F08003436180290BD02AB1036885
:109B300001F01E042343036004E0036801F01E04E7
:109B4000A343036010BD000010B500220268134B50
:109B50001A40CC680B6823434C6923438C69234328
:109B6000CC6923430C6A23434C6A23438C6A234306
:109B70004C6B23438C6B23431A430260426922F0EF
:109B80000702D1E90B3423431A4342610B69436056
:109B90004B6883608B68C36010BD00003F801CF081
:109BA0001CB500240121202022F064F9302000900F
:109BB00001208DF8040000208DF8060003208DF8A8
:109BC000050000208DF807006946164800F0B6FE33
:109BD0003021144800F028FF0021134880F8541762
:109BE00000201249887001204870C8704FF4FA7044
:109BF000886000F01DF80C48007E802810D12420D9
:109C0000094918314871082008713020C8701420A3
:109C100088702020487000210348017600F04AF83F
:109C20001CBD000000140240BC320020103A00208D
:109C30001CB528F07FF8D02028F048F828F0AEF8BE
:109C4000002028F043F828F0A9F828F073F8D12074
:109C500028F03CF828F0A2F800240EE0062C05DAE3
:109C6000012028F003F80DF8040004E0002027F09C
:109C7000FDFF0DF80400601CC4B2072CEEDB28F0D9
:109C800073F89DF806000A4948719DF805000871AF
:109C90009DF80400C8709DF8020088709DF80100CE
:109CA00048709DF800100248183801761CBD00006D
:109CB000D43200201CB500241D48007E8DF8000021
:109CC0001B48183040788DF801001948183080780A
:109CD0008DF8020001208DF8030015481830C07877
:109CE0008DF804001248183000798DF805001048EE
:109CF000183040798DF8060028F01CF8D02027F0A5
:109D0000E5FF28F04BF8002027F0E0FF28F046F8A8
:109D100000BF07E01DF8040027F0D8FF28F03EF848
:109D2000601CC4B2072CF5DB28F01EF81CBD000037
:109D3000BC32002070B502460C460025002309E025
:109D400012F8010B80EA05010648405C80EA030531
:109D50000548435C201EA4F10106B4B2F0D145EAE7
:109D6000032070BDCF790308CF7A030810B50446ED
:109D70000B460021072A00DD072244EA04200146A1
:109D80002BB901FA02F081B20912084610BD012B6D
:109D900002D11141C8B2F9E700BFF7E7704710B52B
:109DA00004460B460021072A00DD072244EA04206E
:109DB000014613B91141C8B210BD012B05D101FAFA
:109DC00002F081B209120846F6E700BFF4E700008E
:109DD000F0B5ADF21C5D04460D460020CDF8180527
:109DE000CDF81405002604EB4400584901EBC000EF
:109DF000408AA84203DC00200DF21C5DF0BD00206B
:109E0000CDF814059AE051480122C168504800F08D
:109E1000B1FA4E48406800788DF800009DF80000C7
:109E200038287DD104EB4400484B03EBC000C068E8
:109E300004EB4403454F07EBC3031B8A03FB0501F7
:109E400004EB44003B4603EBC000028A404800F0AC
:109E500091FA0020CDF8180512E004EB44003B49CC
:109E600001EBC0004068BDF81815405CBDF818252E
:109E70000DF80200BDF81805401C80B2CDF8180599
:109E800004EB4400314901EBC000008ABDF818150D
:109E90008842E2DC04EB44002C4A02EBC000008A5A
:109EA000401E81B2684600F02BFB064604EB4400DE
:109EB000264901EBC000008A401E1DF80000B04298
:109EC00033D10020CDF8180520E004EB44001F49F1
:109ED00001EBC0004068BDF81815415C04EB44007C
:109EE0001A4A02EBC0008068BDF81825024404EB52
:109EF0004400164B03EBC000008A401E6843115417
:109F0000BDF81805401C80B2CDF8180504EB4400DC
:109F10000E4901EBC000008A401EBDF8181500E094
:109F200003E08842D1DC012066E7642027F026FEAA
:109F3000BDF81405401C80B2CDF81405BDF8140519
:109F40000628FFF660AF002056E70000C42A030889
:109F5000C06C00202DE9F041ADF5A36D04460E461E
:109F600000250027A8460020009004EB4400474944
:109F700001EBC000408AB04204DC00200DF5A36D67
:109F8000BDE8F08100210846FFF722FF01287AD1C1
:109F9000002520E004EB44003C4901EBC000806850
:109FA000411904EB4400394A02EBC000008A401E0C
:109FB0007043085C04EB440102EBC1014968485559
:109FC00004EB4400114601EBC0004068405D01A96C
:109FD0004855681C85B204EB44002C4901EBC000D5
:109FE000008AA842D6DC00274BE004EB4400274B54
:109FF00003EBC000C06804EB4403DFF890C00CEB37
:10A00000C3031B8A03FB060104EB4400634603EB16
:10A01000C000008A401E82B21D4800F02DFA04EBF9
:10A0200044001A4A02EBC000008A401E81B201A817
:10A0300000F066FA009004EB4400144A02EBC00002
:10A04000C06804EB4402114B03EBC202128A1044B5
:10A0500004EB440203EBC202128A02FB0600411E1B
:10A060000122684600F008FA31462046FFF7B0FEAC
:10A07000012801D182E706E0642027F07FFD781CEB
:10A0800087B2062FB1DB002078E70000C42A03085E
:10A09000C06C002070B5ADF5A36D00250024002034
:10A0A00000905249088080E000256FE0002414E011
:10A0B0004E48008800EB40004D4951F83000005DEB
:10A0C0004A49098801EB4101494A02EBC10149684B
:10A0D000085501A90855601C84B24448008800EB6B
:10A0E0004000434901EBC000008A401EA042DFDC73
:10A0F0003E48008800EB40000A4602EBC000008AA0
:10A10000401E81B201A800F0FBF90090374800889A
:10A1100000EB4000364B03EBC000C068334B1B889C
:10A1200003EB4303324E06EBC3031B8A03FB05011B
:10A130002E48008800EB4000334603EBC000008A45
:10A14000401E82B22B4800F097F92848008800EBA7
:10A150004000324602EBC000C068244A128802EB7D
:10A160004202334603EBC202128A10441F4A12888D
:10A1700002EB420203EBC202128A02FB0500411EFF
:10A180000122684600F078F9681C85B217480088FB
:10A1900000EB4000164901EBC000408AA84285DC74
:10A1A00012480088401C11490880104800880D287A
:10A1B000FFF67AAF104890F8080E20F001010E4823
:10A1C00080F8081E90F8080E20F00600801D0A494D
:10A1D00081F8080E002001F6086148800021012066
:10A1E000FFF7B8FE0DF5A36D70BD00001000002054
:10A1F000C42A0308C06C0020BC2200201CB5012129
:10A20000084621F037FE01208DF8040002208DF869
:10A21000050000208DF8060001208DF807001820A9
:10A2200000906946144800F089FB05221146124847
:10A2300000F0CCFB052206210F4800F0C7FB0522E9
:10A2400007210D4800F0C2FBA020009002208DF8ED
:10A25000040003208DF8050000208DF806008DF81D
:10A2600007006946044800F069FB402000906946F9
:10A27000014800F063FB1CBD000002402DE9F843DB
:10A2800000240027A046002000900025FFF7B6FF1D
:10A2900000F0C2F800BF00E06D1C30488542FBD3DF
:10A2A0006E4608212E4800F0BDFB10212C4800F01E
:10A2B000BBFB062000F094F80821294800F0B4FB0D
:10A2C0000821274800F0AEFB1021254800F0ACFB28
:10A2D000012000F085F8002000F082F808212048D5
:10A2E00000F0A2FB1F48D0F82C11B0F83021B0F8D4
:10A2F000320102FB0010B0F5003F02D900BE00BFE2
:10A30000FEE71948006808B9FFF7C4FE00201749A6
:10A31000088017E0002406E0144908782146FFF77A
:10A3200057FD601C84B21148008800EB40000D49C5
:10A3300001EBC000408AA042EEDC0C480088401CC3
:10A340000A490880094800880D28E3DB0848D0F84E
:10A35000140207490871BDE8F8830000FFFF0F00F1
:10A3600000000240C42A03081C02434210000020DF
:10A37000BC1200202DE9F04105460C461646002788
:10A38000012027F0B7F90821144800F04BFB1021F9
:10A39000124800F049FB032000F022F8C4F3074004
:10A3A00000F01EF8C4F3072000F01AF8E0B200F045
:10A3B00017F800BF06E0002000F012F828706D1CAE
:10A3C000781C87B2B742F6DB0821044800F02CFB6A
:10A3D000002027F08FF9BDE8F08100000000024066
:10A3E00010B5044600BF02210A4821F06DFF002885
:10A3F000F9D02146074821F073FF00BF012105482D
:10A4000021F062FF0028F9D0024821F066FFC0B2B7
:10A4100010BD00000030014000B585B001210803E7
:10A4200021F078FD134821F023FF0020ADF8000053
:10A43000ADF80400ADF80600ADF808004FF4007068
:10A44000ADF80A003820ADF80C000020ADF80E0081
:10A450000720ADF810004FF48270ADF80200694695
:10A46000044821F03FFF0121024821F0F5FE05B02C
:10A4700000BD0000003001402DE9F04105460C46CA
:10A4800016460027012027F035F908211B4800F067
:10A49000C9FA1021194800F0C7FA0620FFF7A0FFFB
:10A4A0000821164800F0C0FA0821144800F0BAFA52
:10A4B0001021124800F0B8FA0220FFF791FFC4F310
:10A4C0000740FFF78DFFC4F30720FFF789FFE0B2D5
:10A4D000FFF786FF00BF05E02878FFF781FF6D1CBE
:10A4E000781C87B2B742F7DB0821044800F09CFAD9
:10A4F000002027F0FFF8BDE8F081000000000240D6
:10A5000010B50246107803E012F8014B2318D8B2B8
:10A510000B1EA1F10104A1B2F6D110BD2C48807C24
:10A52000012854D100212A4881742A480078C0B9F2
:10A5300001202849087028480068C0002749D1F840
:10A54000301240EA81002549D1F82C1240EA41003E
:10A550002249D1F8281208430F2181432048017075
:10A5600017E000201B4908701B480068C0001B4909
:10A57000D1F8301240EA81001849D1F82C1240EA93
:10A5800041001649D1F8281208430F21814315488C
:10A5900001701348007813490978884217D1104890
:10A5A00000781149087008460078104909788842F7
:10A5B0000DD00D480078064988730B4800780B4988
:10A5C00008700948007810B10120014948737047AC
:10A5D000BC120020DE0A0020340242420000424247
:10A5E000DF0A0020E00A0020E10A0020DD0A002046
:10A5F00010B5ADF57C7D00247CA00068FB900020A8
:10A600000090FEF7F9FF14287CD17948FFF70FF886
:10A610007849087008460078142874D1FFF71AF8B2
:10A620000021754A03C2BDF80000FEF761FF6A46CB
:10A630004FF4FA7101A8FEF779FF70A101A827F085
:10A6400051FC704908800846008810B300BF04E040
:10A6500000216D480155601C84B2282CF8DB01A94B
:10A66000684A1288881869A127F03CFC684908806C
:10A67000002409E063480088C01C204401A9095C4B
:10A6800061480155601C84B261480088001FA042E7
:10A69000F0DC60A101A827F025FC5A490880084693
:10A6A000008820B3002405E00021574828300155D8
:10A6B000601C84B2282CF7DB01A9524A1288881842
:10A6C00052A127F00FFC5249088000240AE04D48AF
:10A6D00000880830204401A9095C4B482830015506
:10A6E000601C84B24A4800880938A042EFDC4CA1C3
:10A6F00001A827F0F7FB434908800846008830B3DB
:10A70000002407E06BE05BE000213F48503001553A
:10A71000601C84B2142CF7DB01A93A4A128888180D
:10A720003AA127F0DFFB3A49088000240AE03548C7
:10A7300000880C30204401A9095C33485030015591
:10A74000601C84B2324800880D38A042EFDC38A18A
:10A7500001A827F0C7FB2B4908800846008820B3D2
:10A76000002405E00020284946390855601C84B2C1
:10A77000322CF7DB01A9234A1288881823A127F07D
:10A78000B1FB2349088000240AE01E480088801D90
:10A79000204401A9085C1C4946390855601C84B254
:10A7A0001B480088C01FA042EFDC00210320FFF7F8
:10A7B000D1FB0120FEF72AFF01200DF57C7D10BDA5
:10A7C0000C480078422803D10948FEF726FF0BE029
:10A7D0000120FEF71BFF00200649087004E000215D
:10A7E0001548C17527F010FB00BFE6E70D0A000011
:10A7F000480A0020380A0020400A002041504E3DFF
:10A80000000000005E0A0020E03A00203B0000004B
:10A810005C0A0020574946494E414D453D00000025
:10A820005749464950415353574F52443D00000049
:10A830005345525645523D00BC32002010B50446E7
:10A840003548844208D10121084621F023FB00212C
:10A85000012021F01FFB5EE03048844208D1012135
:10A86000022021F017FB0021022021F013FB52E00F
:10A870002B48844208D10121042021F00BFB002148
:10A88000042021F007FB46E02648844208D101213C
:10A89000082021F0FFFA0021082021F0FBFA3AE01D
:10A8A0002148844208D10121102021F0F3FA00212F
:10A8B000102021F0EFFA2EE01C48844208D101213B
:10A8C000202021F0E7FA0021202021F0E3FA22E005
:10A8D0001748844208D10121402021F0DBFA0021F1
:10A8E000402021F0D7FA16E01248844208D1012115
:10A8F000802021F0CFFA0021802021F0CBFA0AE05D
:10A900000D48844207D10121801521F0C3FA0021AE
:10A91000A01521F0BFFA10BD000002400004024063
:10A9200000080240000C02400010024000140240E7
:10A9300000180240001C024000200240F0B50A4608
:10A9400000210023002400BF3DE0012505FA01F3AA
:10A95000156805EA03049C4234D105684F000326BC
:10A96000BE40B543056015794E00B54006683543D5
:10A9700005601579012D02D01579022D16D1856853
:10A980004F000326BE40B543856055794E00B54063
:10A99000866835438560456801268E40B54345602D
:10A9A000456896798E40B6B235434560C5684F001C
:10A9B0000326BE40B543C560D5794E00B540C66894
:10A9C0003543C560491C1029BFD3F0BDF0B5002345
:10A9D00000244D07ED0E02FA05F3CE1000F120051C
:10A9E00055F826504E07F70E0F26BE40B543CF1040
:10A9F00000F1200646F82750CE1000F1200555F84A
:10AA0000265045EA0304CE1000F1200545F8264003
:10AA1000F0BD0246002013690B400BB1012000E09D
:10AA20000020704741837047018370470249887B4B
:10AA30000021014A91737047BC120020034800684E
:10AA400000F0010000B100BE00BFFEE7F0ED00E045
:10AA50004AF6AA2001490860704700000030004013
:10AA600030B502460024002305E012F8015B2819E6
:10AA7000C4B2581CC3B28B42F7DB6042C0B230BDD7
:10AA800010B5002427F0C0F9642027F077F810BD36
:10AA90002DE9F043ADF2DC7D80460E461446994622
:10AAA0000025002783A00068CDF8D807002001907A
:10AAB000042C7CDC80480079302101EB101004EB81
:10AAC000C40101EB04117D4A114408717A480079F0
:10AAD00000F00F00303004EBC40101EB041111440D
:10AAE00048717548C078302101EB101004EBC401A7
:10AAF00001EB0411114488716F48C07800F00F0019
:10AB0000303004EBC40101EB04111144C871FEF7AD
:10AB100073FD14287ED16A480078142809D004EB0C
:10AB2000C40101EB0411654A8818FEF780FD6449F1
:10AB300008706348007814286DD1B6F57A7F01DD7E
:10AB40004FF47A76FEF786FD00215E4A03C25D4827
:10AB50000068FEF7CDFC5848C078302101EB10109A
:10AB60008DF808005448C07800F00F0030308DF8A0
:10AB700009005148807801EB10108DF80A004E480A
:10AB8000807800F00F0030308DF80B004A48407894
:10AB900001EB10108DF80C004748407800F00F00D2
:10ABA00030308DF80D0044481838007E00E07CE01D
:10ABB00001EB10108DF80E003F481838007E00F0B1
:10ABC0000F0030308DF80F00B9F1000F03D1542081
:10ABD0008DF8100005E0B9F1010F02D152208DF877
:10ABE00010003A208DF8110000252CE0284605EBD6
:10ABF000D071491018F801100F110A2097FBF0F0DE
:10AC0000C0EBC00107F130000844C1B202AA05F14F
:10AC10000A0001E043E02EE01154284605EBD07114
:10AC2000491018F8011001F00F070A2097FBF0F007
:10AC3000C0EBC00107F130000844C1B205F10B00C0
:10AC40001154A81C85B2B5EB460FCFDB0A2000EBF0
:10AC5000460081B201AA02A8FEF79AFC01AA0221CD
:10AC60000DF5FB60FEF794FC0120FEF7CFFC002001
:10AC70001349087019E012480078422808D104EB03
:10AC8000C40101EB04110D4A8818FEF7C6FC0CE064
:10AC90000120FEF7BBFC00200949087005E00021F7
:10ACA00005481838C17527F0AFF80DF2DC7DBDE816
:10ACB000F08300000D0A0000D4320020600A00205A
:10ACC000380A0020400A002070B5BAB0002139913E
:10ACD00038913791369135913491339132910022E8
:10ACE000309231922E922F922D912C912B912A916C
:10ACF00029912891279126912491169115911491CB
:10AD000013911291119110919FEDFE0A8DED0F0A92
:10AD1000FDA006C8CDE90D12FDA006C8CDE90B12B5
:10AD2000BAE0FD48807858B30020FB498870FB48A2
:10AD3000B0F8B009FA490968C1F57A7188421FD1A3
:10AD4000F7480068C0F57A7081B2F448A0F8A819F5
:10AD50000021F348001FFEF721FEF249F048001FD2
:10AD6000FEF702FE0120F04908704FF47A70EC49BA
:10AD70008C39C1F88C000121E948001FFEF70EFE56
:10AD8000E548807B50B30021E3488173E748408861
:10AD9000E3498C39496CC1F57A7188421ED1E0488B
:10ADA0008C38406CC0F57A70E04908394880002141
:10ADB000DB484C38FEF7F2FDDD49D9484C38FEF748
:10ADC000D3FD0120DB4908704FF47A70D4498C39E7
:10ADD00048640121D2484C38FEF7E0FDCE48807E21
:10ADE00050B30021CC488176D0488088CC498C393A
:10ADF0004969C1F57A7188421ED1C9488C384069C9
:10AE0000C0F57A70C949083988800021C4487C3867
:10AE1000FEF7C4FDC849C2487C38FEF7A5FD0120F5
:10AE2000C64908704FF47A70BD498C3948610121D8
:10AE3000BB487C38FEF7B2FDB74890F8260058B3FF
:10AE40000021B54880F82610B848C088B4498C392C
:10AE5000C96AC1F57A7188421ED1B1488C38C06A7E
:10AE6000C0F57A70B1490839C8800021AC4864380F
:10AE7000FEF794FDB249AA486438FEF775FD01203B
:10AE8000B04908704FF47A70A5498C39C862012125
:10AE9000A3486438FEF782FD9F488178807B014497
:10AEA0009D48807E01449C4890F826000844002874
:10AEB0007FF437AF0DF045B99B48007820B10020F2
:10AEC000994908702D9019E09A48007828B100201F
:10AED0009849087001212D9110E09848007828B118
:10AEE00000209649087002212D9107E095480078CE
:10AEF00020B100209349087003212D919DF8B410D2
:10AF000001EB4100C0EBC1108F4911F83000C1289E
:10AF100036D19DF8B41001EB4100C0EBC1108A4955
:10AF200001EBC000807808282AD101217B4880F8F5
:10AF3000001A9DF8B40030B101280AD002280ED0C2
:10AF4000032818D111E04FF480418048FFF76AFDD3
:10AF500011E04FF400517D48FFF764FD0BE04FF422
:10AF600080517A48FFF75EFD05E04FF400617748B5
:10AF7000FFF758FD00BF00BF00207549086099E742
:10AF800065480C389DF8B41010F811000121B1EBA0
:10AF9000D01F4CF031879DF8B40000EB400101EB6D
:10AFA00000106C4901EB0010407B022841F06B84DB
:10AFB00001F05FBC9DF8B40000EB4001C1EBC01094
:10AFC000614901EBC000007C01069DF8B40000EB74
:10AFD0004002C2EBC0105C4A02EBC000407C41EA78
:10AFE00000419DF8B40000EB4002C2EBC010564A8D
:10AFF00002EBC000807C41EA00219DF8B40000EB28
:10B000004002C2EBC010504A02EBC000C07C0843B3
:10B01000139051489DF8B41050F8212013988242A3
:10B0200001F090834C4A9DF8B400139942F8201027
:10B030009DF8B40000EB4001C1EBC010424901EBA8
:10B04000C000C17B9DF8B40000EB4002C2EBC01011
:10B050003D4A02EBC000807B41EA0021299133493F
:10B0600008399DF8B40031F81010BDF8A4000A307A
:10B07000814211DB2D4908399DF8B40031F81010D8
:10B08000BDF8A4000A30081A82B2284908399DF890
:10B09000B40021F8102008E00020244908399DF868
:10B0A000B42021F8120001F0ECBB9DF8B40000EBD5
:10B0B0004001C1EBC010244901EBC000C01D0A9043
:10B0C000BDF8A410FEF7EAFB12909DF8B41001EB56
:10B0D0004100C0EBC1101C4901EBC002BDF8A40047
:10B0E0000830125C9DF8B40000EB4001C1EBC010C9
:10B0F000154901EBC003BDF8A400C01D185C42EA6D
:10B1000000222BE0000000000169323031303000B5
:10B110000169323045303000E83E0020BC6200203A
:10B120008C60024000880020120000206C6C00201F
:10B130000080201013000020208000101400002048
:10B140000088001015000020D87A00200018024066
:10B150008802424214410020C08A00201298824294
:10B1600041F0CF829DF8B40000EB4001C1EBC0106C
:10B17000F74901EBC000407C00F00F0101EBD170FA
:10B180000A9141100A98A0EB4100C1B215919DF8B7
:10B19000B40000EB4001C1EBC010ED4901EBC00071
:10B1A000C07C00F00F0101EBD17040100A911490A7
:10B1B0000020399025E09DF8B40000EB4001C1EB80
:10B1C000C010E34901EBC001BDF8E4001430095C94
:10B1D0000A91DDE914210A98FEF7C8FD01469DF8A1
:10B1E000B40000EB4002C2EBC010D94A02EBC0022F
:10B1F000BDF8E40014301154BDF8E400401C81B2E5
:10B200003991BDF8A400C01FBDF8E4108842D2DC1B
:10B21000D048C07DA8B1BDF8A400801C81B20A91BD
:10B220009DF8B40000EB4001C1EBC010C84901EB30
:10B23000C000C01D012309909DF8B4200A99FFF7B2
:10B2400027FC9DF8B41001EB4100C0EBC110C049D0
:10B2500001EBC00090F8321026919DF8B41001EB7C
:10B260004100C0EBC110BA4901EBC00090F83310A7
:10B270009DF8B40040F2692210FB02F0B64A02EBDE
:10B28000800080F8A01034211191BDF89800152895
:10B2900001F0108210DCA0F10B000A2881F00B8273
:10B2A000DFE810F0DE04EA048F05EB04090A090A5E
:10B2B00020062106090A070AA1287DD007DC5028AC
:10B2C0007BD0512808D0522841F0F581FDE3A22817
:10B2D00074D0A428F8D1F9E3BDF8A410BDF8440057
:10B2E000081AC1B22491FBE39DF8B41001EB4100B0
:10B2F000C0EBC110964901EBC001BDF84400095CE8
:10B300002B91BDF84400401C81B211919DF8B410FE
:10B3100001EB4100C0EBC1108D4901EBC001BDF84C
:10B320004400095C2C919DF8B00001287DD1BDF846
:10B330004400401C81B211919DF8B41001EB410012
:10B34000C0EBC111824800EBC101BDF84400095CAB
:10B350003591BDF84400401C81B211919DF8B400B4
:10B3600000EB4001C1EBC010794901EBC001BDF811
:10B370004400095C3291BDF84400401C81B2119137
:10B380009DF8B41001EB4100C0EBC110704901EB16
:10B39000C001BDF84400095C3391BDF84400401C75
:10B3A00081B211919DF8B41001EB4100C0EBC110C6
:10B3B000674901EBC00102E0F3E3F3E3F3E3BDF817
:10B3C0004400095C3491BDF84400401C81B21191E5
:10B3D000BDF844103791002128912EE2BDF84400B9
:10B3E000401C81B211919DF8B41001EB4100C0EBFB
:10B3F000C110574901EBC001BDF84400095C25911B
:10B40000BDF84400401C81B211919DF89400C0F336
:10B41000801000287ED00021504A9DF8AC0002EB3D
:10B4200000129DF8A000115400E00CE29DF8942059
:10B430009DF8AC0000EB400101EB0010484901EB26
:10B44000001130319DF8A00001EB001082709DF8D2
:10B45000AC0000EB400101EB0010414901EB001092
:10B4600030309DF8A01000EB01108078C0F3800010
:10B4700020BB9DF8AC0000EB400101EB0010384907
:10B4800001EB001030309DF8A01000EB0110807827
:10B49000C0F3C00090B99DF8AC1001EB410000EB87
:10B4A00001102F4901EB001030309DF8A01000EB87
:10B4B00001108078C0F340000028ABD0002030900D
:10B4C00031900021399122E09DF8B41001EB410048
:10B4D000C0EBC1101E4901EBC001BDF84420BDF80E
:10B4E000E4001044095CBDF8E400C0F10300C000B2
:10B4F00001FA00F0C117DDE93034184341EA0402D3
:10B50000CDE93002BDF8E400401C80B23990BDF8AE
:10B51000E40000E081E10428D6DB9DF8AC0030991E
:10B5200000EB400202EB00100D4A02EB0012303239
:10B530009DF8A00002EB00104160BDF84400001D22
:10B5400081B21191002230923192002139912CE088
:10B55000D87A0020BC320020D4450020483F00208B
:10B56000144100209DF8B40000EB4001C1EBC01075
:10B57000FE4901EBC001BDF84420BDF8E4001044D1
:10B58000095CBDF8E400C0F10300C00001FA00F05E
:10B59000C117DDE93024104341EA0402CDE930024D
:10B5A000BDF8E400401C80B23990BDF8E4000428E6
:10B5B000D8DB9DF8AC00309940F2692210FB02F014
:10B5C000EB4A02EB8002A4329DF8A00000EBC00021
:10B5D00002EB0010C0F81A10BDF84400001D81B243
:10B5E00011910022309231920021399122E09DF890
:10B5F000B41001EB4100C0EBC110DC4901EBC0010C
:10B60000BDF84420BDF8E4001044095CBDF8E40036
:10B61000C0F10300C00001FA00F0C117DDE93034C9
:10B62000184341EA0402CDE93002BDF8E400401CB1
:10B6300080B23990BDF8E4000428D8DB9DF8AC0056
:10B64000309940F2692210FB02F0C94A02EB8002F5
:10B65000A4329DF8A00000EBC00002EB0010C0F87F
:10B660001E10BDF84400001D81B2119100223092DD
:10B6700031920021399122E09DF8B40000EB4001A5
:10B68000C1EBC010B94901EBC001BDF84420BDF8C1
:10B69000E4001044095CBDF8E400C0F10200C00001
:10B6A00001FA00F0C117DDE93024104341EA040239
:10B6B000CDE93002BDF8E400401C80B23990BDF8FD
:10B6C000E4000328D8DB9DF8AC0040F2692110FBB0
:10B6D00001F0A74901EB8000A4309DF8A01001EB18
:10B6E000C10100EB011034300A9000683099084322
:10B6F0000A990860BDF84400C01C80B21190002275
:10B70000309231920020399022E09DF8B40000EB95
:10B710004001C1EBC010954901EBC001BDF84420C8
:10B72000BDF8E4001044095CBDF8E400C0F1050078
:10B73000C00001FA00F0C117DDE93034184341EAD6
:10B740000402CDE93002BDF8E400401C80B239901B
:10B75000BDF8E4000628D8DB9DF8AC00DDE9301226
:10B7600040F2692310FB03F0814B03EB8003A43309
:10B770009DF8A00000EBC00003EB001040F8221F72
:10B780004260BDF84400801D81B2119100223092C8
:10B7900031920021399122E09DF8B40000EB400184
:10B7A000C1EBC010714901EBC001BDF84420BDF8E8
:10B7B000E4001044095CBDF8E400C0F10500C000DD
:10B7C00001FA00F0C117DDE93024104341EA040218
:10B7D000CDE93002BDF8E400401C80B23990BDF8DC
:10B7E000E4000628D8DB9DF8AC00DDE9302140F20A
:10B7F000692310FB03F05E4B03EB8003A4339DF839
:10B80000A00000EBC00003EB001022308260C1609A
:10B81000BDF84400801D81B21191BDF84410BDF8FF
:10B82000DC00091ABDF8C800801E814200DB09E077
:10B830009DF8A000401CC1B22891BDF8DC00002892
:10B840007FF4CCAD36E19DF8B40000EB4001C1EBD4
:10B85000C010464901EBC001BDF84400085C032854
:10B86000F0D1BDF84400401C81B211919DF8B400A4
:10B8700000EB4001C1EBC0103C4901EBC001BDF839
:10B880004400095C3591BDF84400401C81B211911F
:10B890009DF8B41001EB4100C0EBC110334901EB3E
:10B8A000C001BDF84400095C3291BDF84400401C61
:10B8B00081B211919DF8B41001EB4100C0EBC110B1
:10B8C0002A4901EBC001BDF84400095C3391BDF881
:10B8D0004400401C81B211919DF8B41001EB41006D
:10B8E000C0EBC110214901EBC001BDF84400095C67
:10B8F0003491BDF84400401C81B21191BDF8441050
:10B90000379100212891CFE0BDF84400401C81B25E
:10B9100011919DF8B41001EB4100C0EBC110134927
:10B9200001EBC001BDF84400095C2591BDF844005D
:10B93000401C81B211919DF89400C0F38010D0B3E7
:10B9400000210C4A9DF8AC0002EB00129DF8A0000B
:10B9500011549DF894209DF8AC0000EB400101EBE0
:10B960000010054901EB0011303107E0D87A0020C2
:10B97000D4450020483F0020144100209DF8A0003D
:10B9800001EB001082709DF8AC1001EB410000EB60
:10B990000110FE4901EB001030309DF8A01000EBC3
:10B9A00001108078C0F3800028B1002030903190E1
:10B9B0000021399128E067E09DF8B41001EB4100C7
:10B9C000C0EBC110F24901EBC001BDF84420BDF845
:10B9D000E40010440A5C9DF8AC0040F2692110FBC1
:10B9E00001F0EC4901EB8001A4319DF8A00000EBCF
:10B9F000C00001EB00113F31BDF8E4000A54BDF86E
:10BA0000E400401C81B23991BDF8E4000A28D3DB80
:10BA1000BDF844000A3081B2119100223092319277
:10BA20000021399127E09DF8B40000EB4001C1EB03
:10BA3000C010D74901EBC001BDF84420BDF8E400B7
:10BA400010440A5C9DF8AC0040F2692110FB01F043
:10BA5000D04901EB8001A4319DF8A00000EBC000AB
:10BA600001EB00115831BDF8E4000A54BDF8E400C0
:10BA7000401C81B23991BDF8E4000228D3DBBDF847
:10BA80004400801C81B21191BDF84410BDF8DC0067
:10BA9000091ABDF8C800801E814200DB09E09DF84C
:10BAA000A000401CC1B22891BDF8DC0000287FF442
:10BAB0002BAF00BFBDF84410BDF8A400801D81422B
:10BAC0000CDCBDF8A410891D02E00DE2A4E007E043
:10BAD000BDF84400081AC1B2249101E0002124916C
:10BAE000249800287FF400AC9DF8B41040F269203F
:10BAF00011FB00F0A74901EB800008309DF8B4105D
:10BB000040F2692211FB02F1A24A02EB810191F895
:10BB1000A01001EB410202EB011100EB410090F893
:10BB2000240000F00100D8B30021399141E0002148
:10BB3000369117E0BDF8E41001EB410000EB011075
:10BB4000924901EB00103030BDF8D81000EB011025
:10BB5000807800F0010000B112E0BDF8D800401C70
:10BB600081B23691BDF8E41001EB410000EB011009
:10BB7000864901EB0010C179BDF8D8008142D9DCBB
:10BB800000BFBDF8E41001EB410000EB01107F495C
:10BB900001EB0010C179BDF8D800814204DD0CE052
:10BBA00038E038E03AE038E0BDF8E400401C81B20B
:10BBB0003991BDF8E4000228B9DB00BFBDF8E4000C
:10BBC000022827DB0D219DF8B40040F2692210FB0A
:10BBD00002F0704A02EB8000417101229DF8B4002E
:10BBE00040F2692110FB01F06A4901EB8000083046
:10BBF0009DF8B41040F2692311FB03F1654B03EB90
:10BC0000810191F8A01001EB410303EB011100EB5E
:10BC100041004284FDE3FDE7FCE7FBE79DF8B4004B
:10BC200000EB4001C1EBC010594901EBC001BDF868
:10BC30004400095C9DF8B40040F2692210FB02F058
:10BC4000544A02EB8000817150219DF8B40040F20B
:10BC5000692210FB02F04F4A02EB80004171D8E3E9
:10BC60000B209DF8B41040F2692211FB02F1494A01
:10BC700002EB81014871CCE3CBE30021399132E042
:10BC80009DF8B40000EB4001C1EBC010404901EB4E
:10BC9000C001BDF84420BDF8E40010440A5C9DF8E2
:10BCA000B40040F2692110FB01F03A4901EB800138
:10BCB00008319DF8B40040F2692310FB03F0354BC6
:10BCC00003EB800090F8A00000EB400303EB0010B2
:10BCD00001EB40011631BDF8E4000A54BDF8E40060
:10BCE000401C81B23991BDF8E4000A28C8DB00216C
:10BCF00039912AE09DF8B40040F2692110FB01F06F
:10BD0000244901EB800108319DF8B40040F269221A
:10BD100010FB02F01F4A02EB800090F8A00000EB3D
:10BD2000400202EB001001EB40011631BDF8E400C7
:10BD30000A5C1949BDF8E400085C824200D008E0C2
:10BD4000BDF8E400401C81B23991BDF8E4000A2836
:10BD5000D0DB00BFBDF8E4000A2831D00F4840888E
:10BD600000282DDD9DF8B40040F2692110FB01F0A0
:10BD7000084901EB800008309DF8B41040F26922B8
:10BD800011FB02F1034A02EB810109E0144100209A
:10BD9000D87A0020D4450020FE1F0308C4300020BC
:10BDA00091F8A01001EB410202EB011100EB410000
:10BDB00024300A90007820F00100401C0A99087095
:10BDC00027E39DF8B40000EB4001C1EBC010FE4931
:10BDD00001EBC001BDF84400401C095C9DF8B400B3
:10BDE00000EB4002C2EBC010F74A02EBC002BDF804
:10BDF0004400105C41EA00229DF8B40040F2692141
:10BE000010FB01F0F14901EB800108319DF8B4000D
:10BE100040F2692310FB03F0EC4B03EB800090F839
:10BE2000A00000EB400303EB001001EB4000428454
:10BE30009DF8B40040F2692110FB01F0E34901EBE9
:10BE4000800008309DF8B41040F2692211FB02F125
:10BE5000DE4A02EB810191F8A01001EB410202EBF6
:10BE6000011100EB4100408CD949498888422DDD01
:10BE70009DF8B40040F2692110FB01F0D34901EBB9
:10BE8000800008309DF8B41040F2692211FB02F1E5
:10BE9000CE4A02EB810191F8A01001EB410202EBC6
:10BEA000011100EB410024300A90007820F00102DB
:10BEB0000A9802700D209DF8B41040F2692211FB1F
:10BEC00002F1C24A02EB810148710AE051209DF85B
:10BED000B41040F2692211FB02F1BC4A02EB81016D
:10BEE000487196E295E294E252219DF8B40040F246
:10BEF000692210FB02F0B54A02EB80004171BDF8E7
:10BF0000A410BDF84400814207DDBDF8A410BDF8BF
:10BF10004400081AC1B2249101E0002124919DF847
:10BF2000B41001EB4100C0EBC110A74901EBC00107
:10BF3000BDF84400401C095C9DF8B40000EB4002D1
:10BF4000C2EBC010A04A02EBC002BDF84400105C76
:10BF500041EA20229DF8B40040F2692110FB01F073
:10BF60009A4901EB800108319DF8B40040F2692341
:10BF700010FB03F0954B03EB800090F8A00000EB62
:10BF8000400303EB001001EB40004270BDF8440099
:10BF9000801C81B211919DF8B40000EB4001C1EB0F
:10BFA000C010894901EBC001BDF84400095C36911D
:10BFB000BDF84400401C81B211919DF8B40000EB23
:10BFC0004001C1EBC010804901EBC001BDF8440045
:10BFD000095C3491BDF84400401C81B211910021EC
:10BFE000379119E37B48D0F81412BDF8DC000844FF
:10BFF0000521B0FBF1F201FB120000EBC00101EBE7
:10C000000012744920319DF8B40000EB4003C3EBEB
:10C01000C0106D4B03EBC003BDF84400185C01F881
:10C020002200BDF84400401C81B2119100223092E0
:10C0300031920021399122E09DF8B40000EB4001DB
:10C04000C1EBC010604901EBC001BDF84420BDF850
:10C05000E4001044095CBDF8E400C0F10300C00036
:10C0600001FA00F0C117DDE93034184341EA040257
:10C07000CDE93002BDF8E400401C80B23990BDF833
:10C08000E4000428D8DB5348D0F81412BDF8DC00D3
:10C0900008440521B0FBF1F201FB120000EBC001E6
:10C0A00001EB00114B48203000EB81013098C1F8C2
:10C0B0000100BDF84400001D81B2119100223092B0
:10C0C00031920021399122E09DF8B40000EB40014B
:10C0D000C1EBC0103C4901EBC001BDF84420BDF8E4
:10C0E000E4001044095CBDF8E400C0F10300C000A6
:10C0F00001FA00F0C117DDE93024104341EA0402DF
:10C10000CDE93002BDF8E400401C80B23990BDF8A2
:10C11000E4000428D8DB2F48D0F81412BDF8DC0066
:10C1200008440521B0FBF1F201FB120000EBC00155
:10C1300001EB00112748203000EB81013098C1F855
:10C140000500BDF84400001D81B21191002230921B
:10C1500031920021399122E09DF8B40000EB4001BA
:10C16000C1EBC010184901EBC001BDF84420BDF877
:10C17000E4001044095CBDF8E400C0F10200C00016
:10C1800001FA00F0C117DDE93034184341EA040236
:10C19000CDE93002BDF8E400401C80B23990BDF812
:10C1A000E4000328D8DB0B48D0F81412BDF8DC00FB
:10C1B00008440521B0FBF1F201FB120000EBC001C5
:10C1C00001EB0011034807E0D87A0020D445002095
:10C1D000C4300020BC120020203000EB81013098D8
:10C1E000C1F80900BDF84400C01C81B211910022C1
:10C1F000309231920021399122E09DF8B40000EB99
:10C200004001C1EBC010FE4901EBC001BDF8442064
:10C21000BDF8E4001044095CBDF8E400C0F105007D
:10C22000C00001FA00F0C117DDE93034184341EADB
:10C230000402CDE93002BDF8E400401C80B2399020
:10C24000BDF8E4000628D8DBEE48D0F81412BDF89B
:10C25000DC0008440521B0FBF1F201FB120000EB09
:10C26000C00101EB0011E748203000EB8102DDE95D
:10C27000301042F80D1F5060BDF84400801D81B29F
:10C2800011910022309231920021399122E09DF8E3
:10C29000B40000EB4001C1EBC010D94901EBC00173
:10C2A000BDF84420BDF8E4001044095CBDF8E4008A
:10C2B000C0F10500C00001FA00F0C117DDE930242B
:10C2C000104341EA0402CDE93002BDF8E400401C0D
:10C2D00080B23990BDF8E4000628D8DBC948D0F810
:10C2E0001412BDF8DC0008440521B0FBF1F201FB9B
:10C2F000120000EBC00101EB0011C248203000EB3E
:10C3000081010D31DDE930208A60C860BDF844004C
:10C31000801D81B21191BB48D0F81412BDF8DC0029
:10C3200008440521B0FBF1F201FB120000EBC00153
:10C3300001EB0011B348203000EB81019DF8B400FF
:10C3400000EB4002C2EBC010AD4A02EBC002BDF8E8
:10C350004400105C81F82600BDF84400401C81B206
:10C360001191A848D0F81412BDF8DC00084405214A
:10C37000B0FBF1F201FB120000EBC00101EB001178
:10C38000A048203000EB81019DF8B40000EB400292
:10C39000C2EBC0109A4A02EBC002BDF84400105C28
:10C3A00081F82500BDF84400401C81B211919548E8
:10C3B000D0F81412BDF8DC0008440521B0FBF1F2FE
:10C3C00001FB120000EBC00101EB00118D48203091
:10C3D00000EB81019DF8B40000EB4002C2EBC010FD
:10C3E000874A02EBC002BDF84400105C81F82400CB
:10C3F000BDF84400401C81B211918248D0F814125B
:10C40000BDF8DC0008440521B0FBF1F201FB12008D
:10C4100000E075E100EBC00101EB0011794820302C
:10C4200000EB81019DF8B40000EB4002C2EBC010AC
:10C43000734A02EBC002BDF84400105C81F823008F
:10C44000BDF84400401C81B211916E48D0F814121E
:10C45000BDF8DC0008440521B0FBF1F201FB12003D
:10C4600000EBC00101EB00116648203000EB8101B8
:10C470009DF8B40000EB4002C2EBC010604A02EB32
:10C48000C002BDF84400105C81F82200BDF84400F1
:10C49000401C81B211915B48D0F81412BDF8DC0049
:10C4A00008440521B0FBF1F201FB120000EBC001D2
:10C4B00001EB00115348203000EB81019DF8B400DE
:10C4C00000EB4002C2EBC0104D4A02EBC002BDF8C7
:10C4D0004400105C81F82100BDF84400401C81B28A
:10C4E00011910022309231920021399122E09DF881
:10C4F000B40000EB4001C1EBC010414901EBC001A9
:10C50000BDF84420BDF8E4001044095CBDF8E40027
:10C51000C0F10300C00001FA00F0C117DDE93024CA
:10C52000104341EA0402CDE93002BDF8E400401CAA
:10C5300080B23990BDF8E4000428D8DB3148D0F847
:10C540001412BDF8DC0008440521B0FBF1F201FB38
:10C55000120000EBC00101EB00112A48203000EB73
:10C5600081013098C1F82700BDF84400001D81B258
:10C570001191002139912AE02248D0F81412BDF817
:10C58000DC0008440521B0FBF1F201FB120000EBD6
:10C59000C00101EB00111B48203000EB81012B3161
:10C5A000BDF8E4209DF8B40000EB4003C3EBC010DD
:10C5B000134B03EBC003BDF84440BDF8E400204436
:10C5C000185C8854BDF8E400401C81B23991BDF874
:10C5D000E4000628D0DBBDF84400801D81B2119133
:10C5E0000848D0F81412BDF8DC0008440521B0FB5F
:10C5F000F1F081B202200A91FCF76AFD002103E00C
:10C60000D87A0020BC1200200620FDF7A3FCBDF85C
:10C61000DC00401C81B23791BDF8DC10BDF8D800B9
:10C620008142FFF6DFACFE48D0F81402FC49C98B0A
:10C63000884208D2FA48D0F81402BDF8D81008444D
:10C64000F749C1F8140200210520FDF783FC0122FF
:10C650009DF8B40040F2692110FB01F0F14901EBB3
:10C66000800108319DF8B40040F2692310FB03F00B
:10C67000EC4B03EB800090F8A00000EB400303EBD1
:10C68000001001F810201F20E7490871BDF8441080
:10C69000BDF8A400801D814208DCBDF8A410891DEE
:10C6A000BDF84400081AC1B2249101E00021249190
:10C6B00026E025E024E000219DF8B40040F2692244
:10C6C00010FB02F0D74A02EB80004171399112E071
:10C6D00000219DF8B40000EB4002C2EBC010D34A29
:10C6E00002EBC002BDF8E4000D301154BDF8E400C7
:10C6F000401C81B23991BDF8E4000528E8DB00BF99
:10C7000027E00021399112E000219DF8B40000EBF0
:10C710004002C2EBC010C54A02EBC002BDF8E40003
:10C720000D301154BDF8E400401C81B23991BDF8C0
:10C73000E4000528E8DB0020BD499DF8B42021F87D
:10C7400012009EE00020BA499DF8B42021F81200A2
:10C7500097E0B7489DF8B41030F81100F0B39DF899
:10C76000B40000EB4001C1EBC010B04901EBC001C7
:10C77000BDF8A4001130085CFA2802D111213791CC
:10C7800013E09DF8B40000EB4001C1EBC010A749D5
:10C7900001EBC001BDF8A4000A30085CFA2802D100
:10C7A0000A21379101E000213791BDF8DC00002813
:10C7B00057DD0021399125E09DF8B40000EB4001E0
:10C7C000C1EBC010994901EBC001BDF8A420BDF830
:10C7D000DC000244BDF8E400104400E049E0095CDC
:10C7E0009DF8B40000EB4002C2EBC0108F4A02EB90
:10C7F000C002BDF8E400C01D1154BDF8E400401CA7
:10C8000081B239918A499DF8B40031F81010BDF811
:10C81000E4008142D0DC002139911DE00021BDF807
:10C82000A420BDF8DC000244814B9DF8B40033F82D
:10C8300010000244BDF8E40002449DF8B40000EB8F
:10C840004003C3EBC010794B03EBC0008154BDF82B
:10C85000E400401C81B23991BDF8E4002828DDDBFA
:10C8600005E0002072499DF8B42021F81200002153
:10C8700029916F489DF8B41030F8110000287EF41B
:10C8800099AB0BF05EBC6B48C07DB0B168499DF8B8
:10C89000B40031F810100A919DF8B40000EB40018B
:10C8A000C1EBC010614901EBC001012309919DF862
:10C8B000B420DDE90901FEF7EBF89DF8B40000EBC8
:10C8C000400101EB00105C4901EB001081792C91D3
:10C8D0009DF8B00009288BF05A82DFE810F0735100
:10C8E00009007F14C5239030D132DF365042744D99
:10C8F0009DF8B40000EB4001C1EBC0104B4901EBC7
:10C90000C000417808460A91002112F0C5FDC1B26D
:10C910002891002136911CE09DF8B40000EB400105
:10C9200001EB0010444901EB00113031BDF8D80093
:10C9300001EB001041789DF8A000814204D1BDF8C0
:10C94000D800C1B2289112E0BDF8D800401C81B2D5
:10C9500036919DF8B40000EB400101EB0010364920
:10C9600001EB0010C179BDF8D8008142D4DC00BFD2
:10C970009DF8B40000EB4001C1EBC0102B4901EB66
:10C98000C000807800F0F000A0280DD19DF8B40020
:10C9900000EB4001C1EBC010244901EBC0008078DE
:10C9A00000F00F0129910AE09DF8B40000EB40016E
:10C9B000C1EBC0101D4901EBC00081782991BDF881
:10C9C000A40008B9102129919DF8B40000EB4001A2
:10C9D000C1EBC010154901EBC001BDF8A400401C1B
:10C9E000095C2691BDF8A400401C81B20A919DF813
:10C9F000B40000EB4001C1EBC0100C4901EBC001D9
:10CA00000991DDE9090113F0E3F937909DF8B400CD
:10CA100000EB4001C1EBC010044901EBC0010DE087
:10CA2000BC120020D44500205C3B0020D87A0020B6
:10CA3000646C0020BC32002014410020BDF8A4002A
:10CA4000801C095CBDF8DC00814242F0C5839DF882
:10CA5000B40000EB4001C1EBC010FE4901EBC00087
:10CA60004078002842F3B8839DF8B40000EB400101
:10CA7000C1EBC010F74901EBC001BDF8A400C01C18
:10CA80000A5C9DF8B40040F2692110FB01F0F24904
:10CA900001EB8001A4319DF8A00000EBC00001EB88
:10CAA000001080F83C200021EC4A9DF8B40002EB15
:10CAB00000129DF8A0001154E948007F012840D1E0
:10CAC0009DF8B40000EB400101EB0010E54901EBDB
:10CAD000001030309DF8A01000EB0110801C0A906F
:10CAE000007820F0800080300A990870BDF8980026
:10CAF000B62814D0C52819D0D52802D0D9281CD1E1
:10CB000006E0BDF8A400032801DA0021269117E011
:10CB1000BDF8A400032801DA0021269110E0BDF839
:10CB2000A400032801DA0021269109E0BDF8A40041
:10CB3000032801DA0021269102E00021269100BF9E
:10CB400000BF9DF8B40000EB400101EB0010C549A7
:10CB500001EB001030309DF8A01000EB0110801C9C
:10CB60000A90007820F0400040300A990870BDF823
:10CB70009800C52801F03D8417DCB5287ED00DDC77
:10CB8000112802F0BB81122802F00282132802F061
:10CB90008B82B22842F01F8301F0F7BBB6286ED01B
:10CBA000B9286DD0C328F5D1FDE3D92869D007DCB9
:10CBB000CA2867D0CE2802F0D080D528EAD109E073
:10CBC000E12802F0DD80E52802F0ED80E728E1D1E0
:10CBD00002F07DB99DF8B40000EB4001C1EBC0103C
:10CBE0009C4901EBC000C1789F4880F80E1E9DF85B
:10CBF000B40040F2692110FB01F0974901EB80017C
:10CC0000A4319DF8A00000EBC00001EB00100178FA
:10CC10009DF8B40040F2692210FB02F08E4A02EB4C
:10CC20008000007981427DDA9DF8B40000EB40017C
:10CC300001EB00108B4901EB001030309DF8A01083
:10CC400000EB0110801C0A90874890F80E0E01211D
:10CC5000A1EBD0100A99097860F300010A980170DD
:10CC6000814890F80E0EC0F34010E0BB9DF8B40070
:10CC700000EB400101EB00107A4904E0FEE3FEE323
:10CC8000FEE3FEE3FEE301EB001030309DF8A01060
:10CC900000EB01108078C0F3401020B39DF8B40081
:10CCA00000EB400101EB00106E4901EB0010303049
:10CCB0009DF8A01000EB0110801C0A90007820F075
:10CCC0000200801C0A9908709DF8B40040F26921A6
:10CCD00010FB01F0114601EB8000A4309DF8A0107C
:10CCE00001EBC10100E00EE000EB011018300A90EA
:10CCF000007820F00200801C0A9908709DF8B4109A
:10CD00000220FDF727F900219DF8B40040F26922C6
:10CD100010FB02F0504A02EB8000C17002229DF825
:10CD2000B40000E021E040F2692110FB01F04A4923
:10CD300001EB8001A4319DF8A00000EBC00001EBE5
:10CD400000100270B6229DF8B40040F2692110FB79
:10CD500001F0414901EB8000A4309DF8A01001EBE7
:10CD6000C10100EB01104271FDE39DF8B40000EB3E
:10CD7000400101EB00103B4901EB001030309DF801
:10CD8000A01000EB0110801C0A90374890F80E0E9E
:10CD90000121A1EBD0100A990A7860F300020A7011
:10CDA0009DF8B40000EB400101EB00102D4901EBB0
:10CDB000001030309DF8A01000EB0110801C0A908C
:10CDC000294890F80E0E42090A98007862F3410053
:10CDD0000A9908709DF8B40000EB400101EB0010C7
:10CDE000204901EB001030309DF8A01000EB01103D
:10CDF0008078C0F340029DF8B40040F2692110FB36
:10CE000001F0154901EB8000A4309DF8A01001EB62
:10CE1000C10100EB0110007EC0F3400082427DD0D2
:10CE20009DF8B40040F2692110FB01F00A4901EBC2
:10CE30008000A4309DF8A01001EBC10100EB0110AF
:10CE400018300A909DF8B40000EB400101EB00108F
:10CE500004490BE0D87A0020D4450020483F002048
:10CE6000BC12002014410020BC22002001EB001065
:10CE700030309DF8A01000EB0110807842080A982D
:10CE8000007862F341000A9908709DF8B40000EB45
:10CE9000400101EB0010FE4901EB001030309DF81D
:10CEA000A01000EB01108078C0F34000B8B3D92285
:10CEB0009DF8B40040F2692110FB01F0F54901EB47
:10CEC0008000A4309DF8A01001EBC10100EB01101F
:10CED0004271F14890F8A008E8BB9DF8B40040F218
:10CEE000692110FB01F0EB4901EB8000A4309DF8B3
:10CEF000A01001EBC10100EB011090F87D0050B3D0
:10CF000011239DF8B40040F2692110FB01F0E149C2
:10CF100001EB8001A4319DF8A00001E04AE15AE054
:10CF200000EBC00001EB001090F87E0040F2692198
:10CF300010FB01F0D74901EB8001A4319DF8B4004A
:10CF400040F2692210FB02F0D24A02EB8002A432C6
:10CF50009DF8A00000E0B7E000EBC00002EB00107D
:10CF600090F87F0000EBC00001EB001080F87630F5
:10CF7000F3239DF8B40040F2692110FB01F0C5498C
:10CF800001EB8001A4319DF8A00000EBC00001EB93
:10CF9000001090F87E0040F2692110FB01F0BD49BD
:10CFA00001EB8001A4319DF8B40040F2692210FB2E
:10CFB00002F0B84A02EB8000A4309DF8A02002EBFA
:10CFC000C20200EB021090F87F0000EBC00001EB02
:10CFD00000104371E9E001229DF8B40040F269219C
:10CFE00010FB01F0AB4901EB8001A4319DF8A000DA
:10CFF00000EBC00001EB00104273D9229DF8B40091
:10D0000040F2692110FB01F0A24901EB8001A4313B
:10D010009DF8A00000EBC00001EB0010427101225E
:10D020009DF8B40040F2692110FB01F0994901EB31
:10D030008000A4309DF8A01001EBC10100EB0110AD
:10D0400080F83E20944890F8A008E8BB9DF8B40012
:10D0500040F2692110FB01F08E4901EB8000A43001
:10D060009DF8A01001EBC10100EB011090F87D00CC
:10D0700050B39DF8B40040F2692110FB01F08549DE
:10D0800001EB8001A4319DF8A00000EBC00001EB92
:10D09000001090F87E0000EB400101EB00107C498D
:10D0A00001EB001130319DF8B40040F2692210FB11
:10D0B00002F0784A02EB8002A4329DF8A00000EB57
:10D0C000C00002EB001000E06FE090F87F0001EB81
:10D0D0000010801C0A90007820F004020A98027068
:10D0E00000239DF8B40040F2692110FB01F069496A
:10D0F00001EB8000A4309DF8A01001EBC10100EB12
:10D10000011090F87E0040F2692110FB01F06149A6
:10D1100001EB8000A4309DF8B41040F2692211FBAD
:10D1200002F15C4A02EB8102A4329DF8A01001EBEF
:10D13000C10102EB011191F87F1001EBC10100EB7D
:10D14000011080F87630F3239DF8B40040F2692195
:10D1500010FB01F04F4901EB8000A4309DF8A010B6
:10D1600001EBC10100EB011090F87E0040F2692153
:10D1700010FB01F0474901EB8000A4309DF8B4108A
:10D1800040F2692211FB02F1424A02EB8101A43113
:10D190009DF8A02002EBC20201EB021191F87F1072
:10D1A00001EBC10100EB011043719DF8B4100220A6
:10D1B000FCF7D0FE9DF8B40000EB400101EB00103D
:10D1C000334901EB001130319DF8A00001EB001054
:10D1D000807800F001029DF8B40040F2692110FB54
:10D1E00001F02C4901EB8000A4309DF8A01001EB68
:10D1F000C10100EB0110007E00F00100824276D0F8
:10D200009DF8B40040F2692110FB01F0214901EBC7
:10D210008000A4309DF8A01001EBC10100EB0110CB
:10D2200018300A909DF8B40000EB400101EB0011AA
:10D23000174800EB011030309DF8A01000EB0110F2
:10D2400080780A990A7860F300020A709DF8B400A9
:10D2500000EB400101EB00100D4901EB00103030F4
:10D260009DF8A01000EB0110807800F00100E8BBF1
:10D270009DF8B40000EB400101EB0010044901EB04
:10D28000001030309DF8A01000EB0110807805E010
:10D2900014410020D4450020BC320020C0F34010CF
:10D2A00030B39DF8B40040F2692110FB01F0FE4953
:10D2B00001EB8000A4309DF8A01001EBC10100EB50
:10D2C000011090F83E0098B99DF8B40040F2692131
:10D2D00010FB01F0F44901EB8000A4309DF8A01090
:10D2E00001EBC10100EB0110407B02E063E03BE297
:10D2F0003EE0E8BB9DF8B40000EB400101EB0010FC
:10D30000EA4901EB001030309DF8A01000EB01104D
:10D310008078C0F3400058BB01229DF8B40040F271
:10D32000692110FB01F0E04901EB8001A4319DF877
:10D33000A00000EBC00001EB00104273D9229DF861
:10D34000B40040F2692110FB01F0D74901EB8001E4
:10D35000A4319DF8A00000EBC00001EB0010427169
:10D3600001229DF8B40040F2692110FB01F000E0B9
:10D370000BE0CD4901EB8000A4309DF8A01001EB3B
:10D38000C10100EB011080F83E2000229DF8B4009E
:10D3900040F2692110FB01F0C34901EB8000A43089
:10D3A0009DF8A01000E0FDE301EBC10100EB0110CE
:10D3B00080F83D20D3E19DF8B40040F2692110FBD4
:10D3C00001F0B94901EB8000A4309DF8A01001EBF9
:10D3D000C10100EB011090F83E0098B901229DF8C0
:10D3E000B40040F2692110FB01F0AF4901EB80006D
:10D3F000A4309DF8A01001EBC10100EB011080F8F2
:10D400003D2027E000229DF8B40040F2692110FB86
:10D4100001F0A54901EB8001A4319DF8A00000EBCB
:10D42000C00001EB001080F83D209DF8B40000EB37
:10D43000400101EB00109D4901EB001130319DF8D6
:10D44000A00001EB0010801C0A90007820F001027F
:10D450000A980270964890F8A008B0B19DF8B40000
:10D4600000EB400101EB0010904901EB001030305F
:10D470009DF8A01000EB0110807A04E0F4E3F4E3DF
:10D48000F4E3FDE2F3E302286FD18A48407F0128EC
:10D490006BD18848D0F814028649C98B884264D27F
:10D4A0009DF8B40040F2692110FB01F07E4901EBC8
:10D4B0008000A4309DF8A01001EBC10100EB011029
:10D4C00090F83D0001284FD19DF8B40040F2692149
:10D4D00010FB01F0744901EB8000A4309DF8A0100E
:10D4E00001EBC10100EB011090F87D00E0BB9DF85D
:10D4F000B40000EB400101EB00106C4901EB00119E
:10D5000030319DF8A00001EB001001789DF8B400C7
:10D5100040F2692210FB02F0634A02EB8000417086
:10D52000C3229DF8B40040F2692110FB01F05E496E
:10D5300001EB8001A4319DF8A00000EBC00001EBDD
:10D540000010427100229DF8B40000EB400101EB95
:10D550000010564901EB001130319DF8A00001EB9D
:10D560000010426002E06CE148E0D8E09DF8B410A1
:10D570000220FCF7EFFC0021399119E000229DF810
:10D58000B40040F2692110FB01F0474901EB800132
:10D59000A4319DF8A00000EBC00001EB00113F3169
:10D5A000BDF8E4000A54BDF8E400401C81B2399192
:10D5B000BDF8E4000A28E1DB0021399119E00022DE
:10D5C0009DF8B40040F2692110FB01F0364901EBEF
:10D5D0008001A4319DF8A00000EBC00001EB001118
:10D5E0005B31BDF8E4000A54BDF8E400401C81B290
:10D5F0003991BDF8E4000F28E1DBB0E09DF8B400FC
:10D6000040F2692110FB01F0274901EB8000A430B2
:10D610009DF8A01001EBC10100EB011090F83D0056
:10D6200001287CD19DF8B40040F2692110FB01F083
:10D630001D4901EB8001A4319DF8A00000EBC00062
:10D6400001EB001090F87E0040F2692110FB01F020
:10D65000154901EB8001A4319DF8B40040F2692224
:10D6600010FB02F0104A02EB8000A4309DF8A020CD
:10D6700002EBC20200EB021090F87F0000EBC0004A
:10D6800001EB001090F87600032868D100239DF884
:10D69000B40040F2692110FB01F0034901EB800165
:10D6A000A4319DF8A00007E0D445002014410020DB
:10D6B000BC320020BC12002000EBC00001EB0010C7
:10D6C00090F87E0040F2692110FB01F0FE4901EB69
:10D6D0008001A4319DF8B40040F2692210FB02F0F1
:10D6E000F94A02EB8002A4329DF8A00000EBC000D2
:10D6F00002EB001090F87F0000EBC00001EB00107F
:10D7000080F876309DF8B40000EB400101EB00108A
:10D71000EE4901EB001130319DF8A00000E01EE061
:10D7200001EB001001789DF8B40040F2692210FB73
:10D7300002F0E54A02EB80004170C3229DF8B4007C
:10D7400040F2692110FB01F0DF4901EB8000A430B9
:10D750009DF8A01001EBC10100EB011042719DF892
:10D76000B4100220FCF7F6FB9DF8B40000EB40017A
:10D7700001EB0010D54901EB001030309DF8A010EE
:10D7800000EB01108078C0F3400088B1D9229DF8E9
:10D79000B40040F2692110FB01F0CB4901EB80009D
:10D7A000A4309DF8A01001EBC10100EB0110427103
:10D7B0009DF8B40040F2692110FB01F0C24901EB71
:10D7C0008000A4309DF8A01001EBC10100EB011016
:10D7D0008078B22835D19DF8B40000EB400101EB10
:10D7E0000010BA4901EB001030309DF8A01000EB9A
:10D7F00001108078C0F3400018BB9DF8B40000EB26
:10D80000400101EB0010B14901EB001030309DF8F0
:10D81000A01000EB01108078C0F3401088B9E52219
:10D820009DF8B40040F2692110FB01F0A64901EB1C
:10D830008000A4309DF8A01001EBC10100EB0110A5
:10D8400042719DF8B40000EB400101EB00109F49CC
:10D8500001EB001030309DF8A01000EB0110807833
:10D860000121B1EBD01F4FD19DF8B40000EB400176
:10D8700001EB0010954901EB001030309DF8A0102D
:10D8800000EB0110807800F00100E8BB9DF8B400C7
:10D8900040F2692110FB01F08B4901EB8000A430BC
:10D8A0009DF8A01001EBC10100EB011090F83E00C3
:10D8B00050BB9DF8B40000EB400101EB0010834920
:10D8C00001EB001030309DF8A01000EB01108078C3
:10D8D000C0F3C000C0B99DF8B40000EB400101EBFB
:10D8E00000107A4901EB001030309DF8A01000EBD9
:10D8F0000110407A00F0010030B19DF8B40040F210
:10D90000692110FB01F000E049E06F4901EB800064
:10D91000A4309DF8A01001EBC10100EB011090F8BC
:10D920008E0000F00100D0BB9DF8B40040F26921E8
:10D9300010FB01F0644901EB8000A4309DF8A010B9
:10D9400001EBC10100EB011090F8800038B3002119
:10D9500039912AE09DF8B40040F2692110FB01F0F2
:10D96000594901EB8001A4319DF8A00000EBC000F3
:10D9700001EB001000F18101BDF8E4000A5C9DF8A4
:10D98000B40000EB400101EB0010504901EB001125
:10D990000E31BDF8E400085C824201D009E06DE080
:10D9A000BDF8E400401C81B23991BDF8E4000628BE
:10D9B000D0DB00BFBDF8E40006285FD10621399115
:10D9C00029E09DF8B40040F2692110FB01F03E49C6
:10D9D00001EB8001A4319DF8A00000EBC00001EB39
:10D9E000001000F18101BDF8E4000A5C9DF8B4006C
:10D9F00000EB400101EB0010344901EB00100E3048
:10DA0000BDF8E410405C824200D008E0BDF8E400BC
:10DA1000401C81B23991BDF8E4000A28D1DB00BF77
:10DA2000BDF8E4000A2829D09DF8B40040F269212D
:10DA300010FB01F0244901EB8000A4309DF8A010F8
:10DA400001EBC10100EB01108E300A90007820F04C
:10DA50000100401C0A99087012229DF8B40040F29F
:10DA6000692110FB01F0184901EB8000A4309DF8FA
:10DA7000A01001EBC10100EB0110427101F0ABBB42
:10DA80009DF8B40000EB400101EB00100F4901EBE1
:10DA90000010007B90BBBDF8A400082800D0EDE783
:10DAA0000021399130E09DF8B40000EB4001C1EB5A
:10DAB000C010074901EBC001BDF8E400C01C085CC0
:10DAC00000F00F00092805E0D44500201441002093
:10DAD000D87A002000DD1BE09DF8B40000EB400187
:10DAE000C1EBC010FD4901EBC001BDF8E400C01C52
:10DAF000085C00F0F000902801DD09E079E0BDF855
:10DB0000E400401C81B23991BDF8E4000628CADB6C
:10DB100000BFBDF8E400062800DAAFE79DF8B400C6
:10DB200000EB4001C1EBC010EC4901EBC000C07834
:10DB300001049DF8B40000EB4002C2EBC010E74ABC
:10DB400002EBC000007941EA00219DF8B40000EB2F
:10DB50004002C2EBC010E14A02EBC0004079014331
:10DB60009DF8B40040F2692210FB02F0DC4A02EB9F
:10DB70008002A4329DF8A00000EBC00002EB001070
:10DB8000C0F81A109DF8B40000EB4001C1EBC010C2
:10DB9000D24901EBC000807901049DF8B40000EB8C
:10DBA000400200E0A0E1C2EBC010CC4A02EBC00092
:10DBB000C07941EA00219DF8B40000EB4002C2EBBD
:10DBC000C010C64A02EBC000007A01439DF8B400C1
:10DBD00040F2692210FB02F0C14A02EB8000A4303F
:10DBE0009DF8A02002EBC20200EB0210C0F81E104C
:10DBF000BEE0BDF8A4000A2800D03FE7002139911B
:10DC000028E09DF8B40000EB4001C1EBC010B3491F
:10DC100001EBC001BDF8E400C01C085C00F00F007F
:10DC2000092800DD1AE09DF8B40000EB4001C1EBCB
:10DC3000C010AA4901EBC001BDF8E400C01C085C9B
:10DC400000F0F000902800DD08E0BDF8E400401C82
:10DC500081B23991BDF8E4000828D2DB00BFBDF8DD
:10DC6000E400082804DA09E786E15DE2F0E170E10A
:10DC70009DF8B40000EB4001C1EBC010974901EBE7
:10DC8000C000C07801069DF8B40000EB4002C2EB72
:10DC9000C010924A02EBC000007941EA00419DF8B1
:10DCA000B40000EB4002C2EBC0108C4A02EBC00093
:10DCB000407941EA00219DF8B40000EB4002C2EB3C
:10DCC000C010864A02EBC000807901439DF8B40081
:10DCD00040F2692210FB02F0814A02EB8002A4327A
:10DCE0009DF8A00000EBC00002EB0010C0F81A1075
:10DCF0009DF8B40000EB4001C1EBC010774901EB87
:10DD0000C000C07901069DF8B40000EB4002C2EBF0
:10DD1000C010724A02EBC000007A41EA00419DF84F
:10DD2000B40000EB4002C2EBC0106C4A02EBC00032
:10DD3000407A41EA00219DF8B40000EB4002C2EBBA
:10DD4000C010664A02EBC000807A01439DF8B4001F
:10DD500040F2692210FB02F0614A02EB8000A4301D
:10DD60009DF8A02002EBC20200EB0210C0F81E10CA
:10DD70009DF8B40040F2692110FB01F0584901EB15
:10DD80008001A4319DF8A00000EBC00001EB001061
:10DD900001789DF8B40040F2692210FB02F0504A6D
:10DDA00002EB8000007981422FDA00219DF8B40057
:10DDB00040F2692210FB02F0494A02EB8000C17078
:10DDC00004229DF8B40040F2692110FB01F044499F
:10DDD00001EB8001A4319DF8A00000EBC00001EB35
:10DDE00000100270C5229DF8B40040F2692110FBBA
:10DDF00001F03B4901EB8000A4309DF8A01001EB3D
:10DE0000C10100EB0110427166E09DF8B40000EB27
:10DE1000400101EB0010334901EB001030309DF858
:10DE2000A01000EB01108078C0F3400090B1D52223
:10DE30009DF8B40040F2692110FB01F0284901EB84
:10DE40008000A4309DF8A01001EBC10100EB01108F
:10DE5000427141E09DF8B40040F2692110FB01F0ED
:10DE60001F4901EB8000A4309DF8A01001EBC10117
:10DE700000EB0110807B01282ED100229DF8B40018
:10DE800040F2692110FB01F0154901EB8001A4313A
:10DE90009DF8A00000EBC00001EB00108273B622D9
:10DEA0009DF8B40040F2692110FB01F00C4901EB30
:10DEB0008001A4319DF8A00000EBC00001EB001030
:10DEC000427100219DF8B40040F2692210FB02F07B
:10DED000034A02EB8000C170D0E50000D87A002030
:10DEE000D445002014410020D5229DF8B40040F212
:10DEF000692110FB01F0FE4901EB8001A4319DF87E
:10DF0000A00000EBC00001EB0010427101219DF860
:10DF1000B40040F2692210FB02F0F54A02EB8000E7
:10DF2000C1709DF8B40000EB400101EB0010A2F5B8
:10DF3000986101EB001130319DF8A00001EB001059
:10DF4000801C0A90007820F0200020300A99087088
:10DF500094E5D5229DF8B40040F2692110FB01F050
:10DF6000E34901EB8000A4309DF8A01001EBC10152
:10DF700000EB0110427181E59DF8B40040F2692187
:10DF800010FB01F0DA4901EB8000A430BDF8D81095
:10DF900001EBC10100EB0110807901283AD1002288
:10DFA0009DF8B40040F2692110FB01F0D04901EB6B
:10DFB0008001A431BDF8D80000EBC00001EB0010D7
:10DFC0008271D9229DF8B40040F2692110FB01F062
:10DFD000C74901EB8001A4319DF8A00000EBC0000F
:10DFE00001EB001042719DF8B40000EB400101EB21
:10DFF0000010C04901EB001130319DF8A00001EB89
:10E000000010801C0A90007820F00400001D0A997E
:10E0100008701CE0C3229DF8B40040F2692110FB97
:10E0200001F0B34901EB8001A4319DF8A00000EBA1
:10E03000C00001EB0010427100219DF8B40040F2D5
:10E04000692210FB02F0AA4A02EB8000C17015E5BC
:10E050009DF8B40040F2692110FB01F0A44901EBE6
:10E060008000A430BDF8D81001EBC10100EB011015
:10E07000807901283AD100229DF8B40040F269214C
:10E0800010FB01F09A4901EB8001A431BDF8D800E2
:10E0900000EBC00001EB00108271D9229DF8B400A2
:10E0A00040F2692110FB01F0914901EB8001A4319C
:10E0B0009DF8A00000EBC00001EB001042719DF83C
:10E0C000B40000EB400101EB00108A4901EB0011A4
:10E0D00030319DF8A00001EB0010801C0A90007800
:10E0E00020F00400001D0A9908701CE0C3229DF86E
:10E0F000B40040F2692110FB01F07D4901EB800181
:10E10000A4319DF8A00000EBC00001EB00104271AB
:10E1100000219DF8B40040F2692210FB02F0744A1D
:10E1200002EB8000C170A9E49DF8B40000EB40014F
:10E1300001EB00106F4901EB0010007B38BB9DF82C
:10E14000B40000EB4001C1EBC0106B4901EBC00013
:10E1500001799DF8B40000EB4002C2EBC010664AA2
:10E1600002EBC000C07841EA00229DF8B40040F202
:10E17000692110FB01F05E4901EB8000A4309DF89D
:10E18000A01001EBC10100EB0110426332E09DF8E9
:10E19000B40000EB4001C1EBC010574901EBC000D7
:10E1A000C07801049DF8B40000EB4002C2EBC0103F
:10E1B000514A02EBC000007941EA00219DF8B40009
:10E1C00000EB4002C2EBC0104B4A02EBC0004079AA
:10E1D00001439DF8B40040F2692210FB02F0444A6A
:10E1E00002EB8000A4309DF8A02002EBC20200EBFD
:10E1F000021041639DF8B40040F2692110FB01F068
:10E200003B4901EB8001A4319DF8A00000EBC00068
:10E2100001EB001001789DF8B40040F2692210FB78
:10E2200002F0334A02EB8000007981422FDA0021AC
:10E230009DF8B40040F2692210FB02F02C4A02EB78
:10E240008000C17003229DF8B40040F2692110FBE8
:10E2500001F0274901EB8001A4319DF8A00000EBFB
:10E26000C00001EB00100270D9229DF8B40040F20A
:10E27000692110FB01F01E4901EB8000A4309DF8DC
:10E28000A01001EBC10100EB011042717CE09DF890
:10E29000B40040F2692110FB01F0154901EB800048
:10E2A000A430BDF8D81001EBC10100EB011080795A
:10E2B00001284CD100229DF8B40040F2692110FBE6
:10E2C00001F00B4901EB8001A431BDF8D80000EB4F
:10E2D000C00001EB00108271D9229DF8B40040F219
:10E2E000692110FB01F0024901EB8001A43105E036
:10E2F000D445002014410020D87A00209DF8A000C9
:10E3000000EBC00001EB001042719DF8B40000EB7F
:10E31000400101EB0010FE4901EB001130319DF886
:10E32000A00001EB0010801C0A90007820F004008F
:10E33000001D0A99087001209DF8B41040F269226E
:10E3400011FB02F1F34A02EB8101C8701CE0C52207
:10E350009DF8B40040F2692110FB01F0ED4901EB9A
:10E360008001A4319DF8A00000EBC00001EB00107B
:10E37000427100219DF8B40040F2692210FB02F0C6
:10E38000E44A02EB8000C17037E400219DF8B4003C
:10E3900040F2692210FB02F0DE4A02EB8000C170FD
:10E3A0009DF8B40000EB400101EB0010D84901EBEF
:10E3B000001130319DF8A00001EB0010801C0A9084
:10E3C000007820F00400001D0A990870D5229DF8FD
:10E3D000B40040F2692110FB01F0CE4901EB80004E
:10E3E000A4309DF8A01001EBC10100EB01104271B7
:10E3F00039E49DF8B40000EB400101EB0010C44982
:10E4000001EB0010007BD0BBBDF8A4000C2800D0AD
:10E4100029E40021399128E09DF8B40000EB400187
:10E42000C1EBC010BC4901EBC001BDF8E400C01C49
:10E43000085C00F00F00092800DD1AE09DF8B40028
:10E4400000EB4001C1EBC010B34901EBC001BDF8C6
:10E45000E400C01C085C00F0F000902800DD08E03B
:10E46000BDF8E400401C81B23991BDF8E4000A28EF
:10E47000D2DB00BFBDF8E4000A2801DA2CE57DE01C
:10E4800000202E902F90002139911EE0DDE92E1002
:10E49000000240EA11620902CDE92E129DF8B40093
:10E4A00000EB4001C1EBC0109B4901EBC001BDF87E
:10E4B000E400C01C085CDDE92E341843CDE92E04CD
:10E4C000BDF8E400401C80B23990BDF8E400052896
:10E4D000DCDB9DF8B400DDE92E1240F2692310FB6D
:10E4E00003F08C4B03EB8003A4339DF8A00000EBFA
:10E4F000C00003EB001040F8221F426000222E9261
:10E500002F92002139911FE0DDE92E10000240EA30
:10E5100011620902CDE92E129DF8B40000EB400112
:10E52000C1EBC0107C4901EBC001BDF8E40008302C
:10E53000085CDDE92E3440EA0302CDE92E24BDF863
:10E54000E400401C81B23991BDF8E4000528DBDB12
:10E550009DF8B400DDE92E2140F2692310FB03F0A1
:10E560006C4B03EB8000A4309DF8A03003EBC30399
:10E5700000EB031022308260C160B8E0BDF8A40057
:10E580000E2800D0E8E30021399128E09DF8B4007E
:10E5900000EB4001C1EBC0105F4901EBC001BDF8C9
:10E5A000E400C01C085C00F00F00092800DD1AE040
:10E5B0009DF8B40000EB4001C1EBC010564901EBDF
:10E5C000C001BDF8E400C01C085C00F0F000902819
:10E5D00000DD08E0BDF8E400401C81B23991BDF8CF
:10E5E000E4000C28D2DB00BFBDF8E4000C2800DA00
:10E5F000B2E300202E902F90002139911FE0DDE939
:10E600002E10000240EA11620902CDE92E129DF897
:10E61000B40000EB4001C1EBC0103F4901EBC00169
:10E62000BDF8E400C01C085CDDE92E3440EA0302BA
:10E63000CDE92E24BDF8E400401C81B23991BDF82B
:10E64000E4000628DBDB9DF8B400DDE92E2140F272
:10E65000692310FB03F02F4B03EB8003A4339DF8D9
:10E66000A00000EBC00003EB001040F8222F416037
:10E6700000222E922F92002139911FE0DDE92E1009
:10E68000000240EA11620902CDE92E129DF8B400A1
:10E6900000EB4001C1EBC0101F4901EBC001BDF808
:10E6A000E4000930085CDDE92E3440EA0302CDE9DC
:10E6B0002E24BDF8E400401C81B23991BDF8E4007D
:10E6C0000628DBDB9DF8B400DDE92E1240F2692359
:10E6D00010FB03F00F4B03EB8000A4309DF8A0303B
:10E6E00003EBC30300EB031022308160C2609DF88E
:10E6F000B40040F2692110FB01F0064901EB8001F2
:10E70000A4319DF8A00000EBC00001EB001005E073
:10E7100014410020D4450020D87A002001789DF8CB
:10E72000B40040F2692210FB02F0FE4A02EB8000C6
:10E73000007981427ED1FC4890F8A00888B19DF80C
:10E74000B40000EB400101EB0010A2F5986101EB71
:10E75000001030309DF8A01000EB0110807A0228E4
:10E7600069D1F248D0F814020521B0FBF1F201FBA7
:10E77000120000EBC00101EB0011EC48203000EB6F
:10E7800081000021C0F81D10E848D0F814020521CE
:10E79000B0FBF1F201FB120000EBC00101EB001134
:10E7A000E248203000EB81000D300A909DF8B40063
:10E7B00040F2692110FB01F0DA4901EB8001A4313C
:10E7C0009DF8A00000EBC00001EB001022301022E9
:10E7D000014609900A98F9F738FDD448D0F8140298
:10E7E0000521B0FBF1F201FB120000EBC00101EBCF
:10E7F0000011CE48203000EB81029DF8B40040F2B9
:10E80000692110FB01F0C74901EB8001A4319DF89B
:10E81000A00000EBC00001EB001050F81A1F42F8F6
:10E82000011F40685060C148D0F814020521B0FBB8
:10E83000F1F201E02CE2FEE001FB120000EBC0016E
:10E8400001EB0013B94920319DF8B40000EB400200
:10E8500002EB0010B64A02EB001230329DF8A00025
:10E8600002EB0010007801F82300B048D0F8140241
:10E870000521B0FBF1F201FB120000EBC00101EB3E
:10E880000011AA48203000EB8101A748826941F8B5
:10E89000212F808B8880A548D0F814020521B0FB79
:10E8A000F1F201FB120000EBC00101EB00119F48E7
:10E8B000203000EB81029DF8B40040F2692110FB8A
:10E8C00001F0984901EB8001A4319DF8A00000EB14
:10E8D000C00001EB0010406BC2F809009348D0F86B
:10E8E00014020521B0FBF1F201FB120000EBC001A4
:10E8F00001EB00118D48203000EB81029DF8B4003F
:10E9000000EB400101EB0010894901EB00113031AF
:10E910009DF8A00001EB00104068C2F8270000211C
:10E9200039914CE08148D0F814020521B0FBF1F296
:10E9300001FB120000EBC00101EB00117B4820300D
:10E9400000EB81012B31BDF8E4409DF8B40040F2AA
:10E95000692210FB02F0734A02EB8002A4329DF898
:10E96000A00000EBC00002EB001090F87E0040F227
:10E97000692210FB02F06B4A02EB8002A4329DF880
:10E98000B40040F2692310FB03F0664B03EB8003F5
:10E99000A4339DF8A00000EBC00003EB001090F83A
:10E9A0007F0000EBC00002EB00123F32BDF8E40034
:10E9B000105C0855BDF8E400401C81B23991BDF8E7
:10E9C000E4000A28AEDB5948D0F814020521B0FB58
:10E9D000F1F080B201460A900220FAF779FB00219B
:10E9E0000620FBF7B7FA5148D0F814024F49C98BFB
:10E9F000884206D24D48D0F81402401C4B49C1F859
:10EA0000140200210520FBF7A5FA9DF8B40000EBE5
:10EA1000400101EB0010464901EB001030309DF839
:10EA2000A01000EB0110801C0A90007820F0080272
:10EA30000A98027015E09DF8B40000EB400101EB6C
:10EA400000103B4901EB001030309DF8A01000EBA6
:10EA50000110801C0A90007820F0080008300A9904
:10EA600008709DF8B40000EB400101EB0010304944
:10EA700001EB001030309DF8A01000EB0110801C5D
:10EA80000A90007820F020020A9802709DF8B410D5
:10EA90000220FBF75FFA9DF8B4009DF8A01001EB8F
:10EAA0000010C217CDE92E0200222E9800EBC00103
:10EAB00001EB00111F4800EB8100C0F81D209DF8FC
:10EAC000B41040F2692011FB00F0164901EB800000
:10EAD000A4309DF8A01001EBC10100EB0110223021
:10EAE0000A902E9800EBC00101EB0011114800EBD9
:10EAF00081010D3110220991DDE90901F9F7A5FB2A
:10EB00009DF8B40040F2692110FB01F0054901EBCA
:10EB10008001A4319DF8A00000EBC00001EB0011C2
:10EB20002E9809E0D4450020BC320020BC12002001
:10EB300014410020E014002000EBC00202EB0012A0
:10EB4000F94800EB820051F81A2F40F8012F49686C
:10EB500041609DF8B40000EB400101EB0010F34967
:10EB600001EB001130319DF8A00001EB001001789D
:10EB70002E9800EBC00202EB0012EB4800F82210C6
:10EB80002E9800EBC00101EB0011E74800EB81017A
:10EB9000E748826941F8212F808B88809DF8B40076
:10EBA00040F2692110FB01F0E24901EB8001A43140
:10EBB0009DF8A00000EBC00001EB0010416B2E9807
:10EBC00000EBC00202EB0012D74800EB8200C0F855
:10EBD00009109DF8B40000EB400101EB0010D3498F
:10EBE00001EB001130319DF8A00001EB00104168ED
:10EBF0002E9800EBC00202EB0012CB4800EB820023
:10EC0000C0F827100021399124E09DF8B40040F2AB
:10EC1000692110FB01F0C74901EB8001A4319DF887
:10EC2000A00000EBC00001EB00113F31BDF8E40093
:10EC30000A5C2E9800EBC00101EB0011BA4800EB12
:10EC400081012B31BDF8E4000A54BDF8E400401CFA
:10EC500081B23991BDF8E4000A28D6DB2E9881B242
:10EC600008200A91FBF776F900229DF8B40040F2E3
:10EC7000692110FB01F0AF4901EB8000A4309DF841
:10EC8000A01001EBC10100EB011080F83E2051E023
:10EC90009DF8B40000EB400101EB0010A34901EB2B
:10ECA000001030309DF8A01000EB0110801C0A907D
:10ECB000007820F00400001D0A9908709DF8B40047
:10ECC00000EB400101EB0010984901EB00103030DF
:10ECD0009DF8A01000EB0110801C0A90007820F035
:10ECE000800080300A99087001209DF8B41040F22D
:10ECF000692211FB02F18F4A02EB8101C8709DF875
:10ED0000B40040F2692110FB01F0114601EB8000D4
:10ED100002799DF8B40040F2692110FB01F08549A9
:10ED200001EB8000A4309DF8A01001EBC10100EBC5
:10ED300001100270D5229DF8B40040F2692110FB49
:10ED400001F07C4901EB8000A4309DF8A01001EB9C
:10ED5000C10100EB011042713DE2D5229DF8B400E3
:10ED600040F2692110FB01F0724901EB8000A430F0
:10ED70009DF8A01001EBC10100EB011042712AE2E5
:10ED8000D5229DF8B40040F2692110FB01F06949D9
:10ED900001EB8000A4309DF8A01001EBC10100EB55
:10EDA0000110427117E20121614880F8C4179DF8F3
:10EDB000B40040F2692110FB01F05E4901EB8001D3
:10EDC000A4319DF8A00000EBC00001EB0010017819
:10EDD0009DF8B40040F2692210FB02F0554A02EBA4
:10EDE0008000007981422FDA00219DF8B40040F2C2
:10EDF000692210FB02F04F4A02EB8000C170012231
:10EE00009DF8B40040F2692110FB01F0494901EB83
:10EE10008001A4319DF8A00000EBC00001EB0010C0
:10EE2000027011229DF8B40040F2692110FB01F03C
:10EE3000404901EB8000A4309DF8A01001EBC10116
:10EE400000EB0110427141E09DF8B40040F26921ED
:10EE500010FB01F0374901EB8000A4309DF8A010B1
:10EE600001EBC10100EB01108078B2282ED1002106
:10EE70009DF8B40040F2692210FB02F02D4A02EB2B
:10EE80008000C170B2229DF8B40040F2692110FBED
:10EE900001F0284901EB8001A4319DF8A00000EBAE
:10EEA000C00001EB0010427100229DF8B40040F256
:10EEB000692110FB01F01F4901EB8000A4309DF88F
:10EEC000A01001EBC10100EB0110827083E1002171
:10EED000174880F8C417D5229DF8B40040F2692184
:10EEE00010FB01F0134901EB8000A4309DF8A01045
:10EEF00001EBC10100EB011042716CE101229DF8B0
:10EF0000B40040F2692110FB01F00A4901EB8001D5
:10EF1000A4319DF8A00000EBC00001EB001080F8C8
:10EF20008020002139912EE0E014002014410020BF
:10EF3000BC320020D44500209DF8B40000EB400115
:10EF4000C1EBC010FE4901EBC001BDF8E400C01CDC
:10EF50000A5C9DF8B40040F2692110FB01F0F94908
:10EF600001EB8001A4319DF8A00000EBC00001EB93
:10EF7000001000F18101BDF8E4000A54BDF8E4007E
:10EF8000401C81B23991BDF8E4000A28D4DB22E1AB
:10EF90009DF8B40000EB4001C1EBC010E84901EB63
:10EFA000C000C07801049DF8B40000EB4002C2EB41
:10EFB000C010E34A02EBC000007941EA00209DF84E
:10EFC000B41001EB4102C2EBC111DD4A02EBC101F9
:10EFD00049790843B0F5E13F65D19DF8B40000EBF5
:10EFE000400101EB0010D84901EB001030309DF8D2
:10EFF000A01000EB0110801C0A90007820F00402A1
:10F000000A98027000229DF8B40040F2692110FBBA
:10F0100001F0CC4901EB8000A4309DF8A01001EB79
:10F02000C10100EB0110A0F88C2013229DF8B40060
:10F0300040F2692110FB01F0C24901EB8000A430CD
:10F040009DF8A01001EBC10100EB011042719DF889
:10F05000B40000EB400101EB0010BB4901EB0010D4
:10F06000407903464FF480524FF4E1310A909DF805
:10F07000B40010F0BFFE9DF8B40040F2692110FB0F
:10F0800001F0B04901EB8001A4319DF8A00000EB34
:10F09000C00001EB00108E300A90007820F00800CC
:10F0A00008300A99087096E09DF8B40000EB400122
:10F0B000C1EBC010A24901EBC00001799DF8B4007A
:10F0C00000EB4002C2EBC0109D4A02EBC000C078CA
:10F0D00041EA00229DF8B40040F2692110FB01F0E2
:10F0E000984901EB8001A4319DF8A00000EBC0001D
:10F0F00001EB0010A0F88C209DF8B40040F26921CB
:10F1000010FB01F08F4901EB8001A4319DF8A000B4
:10F1100000EBC00001EB0010B0F88C109DF8B400BB
:10F1200000EB400202EB0010874A02EB0010408B1C
:10F1300081424FDBE5229DF8B40040F2692110FBCB
:10F1400001F0804901EB8001A4319DF8A00000EBA3
:10F15000C00001EB0010427100229DF8B40040F2A3
:10F16000692110FB01F0774901EB8001A4319DF882
:10F17000A00000EBC00001EB001002709DF8B4008D
:10F1800000EB400101EB00106F4901EB0011303141
:10F190009DF8A00001EB0010801C0A90007820F080
:10F1A00080020A9802709DF8B40040F2692110FBB9
:10F1B00001F0644901EB8000A4309DF8A01001EB40
:10F1C000C10100EB01108E300A90007820F001029E
:10F1D0000A98027000BF00BF08F0D9BD9DF8B400C6
:10F1E00000EB4001C1EBC010554911F83000042874
:10F1F00002D1042126910BE09DF8B41001EB4100EF
:10F20000C0EBC1104E4911F83000152800D12690EE
:10F210009DF8B41001EB4100C0EBC111484800EB70
:10F22000C10041789DF8B40000EB4002C2EBC01071
:10F23000434A12F8300041EA002041F2300188428E
:10F2400002D1A62026903DE09DF8B41001EB4100CC
:10F25000C0EBC1103A4901EBC00041789DF8B40001
:10F2600000EB4002C2EBC010354A12F8300041EA10
:10F27000002041F23101884202D1A720269021E0EE
:10F280009DF8B41001EB4100C0EBC1102C4911F8FE
:10F290003000022816D19DF8B41001EB4100C0EBFC
:10F2A000C110274901EBC00001799DF8B40000EBC3
:10F2B0004002C2EBC010224A02EBC000C07841EA13
:10F2C000002126919DF8B41040F2692011FB00F056
:10F2D0001C4901EB80008178289100211B4A9DF890
:10F2E000B40002EB00129DF8A00011541848007FF2
:10F2F000012815D19DF8B41001EB410000EB01107D
:10F30000114901EB001030309DF8A01000EB011006
:10F31000801C0A90007820F0800080300A990870E4
:10F320009DF8B41001EB410000EB0110064901EB20
:10F33000001030309DF8A01000EB0110801C09E097
:10F34000D87A0020D445002014410020483F0020F6
:10F35000BC1200200A90007820F0400040300A994A
:10F360000870BDF8981043F23002881A91427DD09F
:10F3700009DC04297BD015297AD0A6290DD0A7292C
:10F3800041F0628634E1B0F5C06F72D0A0F2016046
:10F3900000286FD00428F3D1FEE300219DF8B400CB
:10F3A00040F2692210FB02F0FE4A02EB8000C170BD
:10F3B0009DF8B41040F2692011FB00F0114601EBFA
:10F3C0008000A4309DF8A01001EBC10100EB0110FA
:10F3D0000078032824DC04229DF8B40040F269215F
:10F3E00010FB01F0EF4901EB8001A4319DF8A00072
:10F3F00000EBC00001EB00100270A8229DF8B400E1
:10F4000040F2692110FB01F0E64901EB8000A430D5
:10F410009DF8A01001EBC10100EB01104271E5E085
:10F420009DF8B40040F2692110FB01F0DD4901EBC9
:10F430008000A4309DF8A01001EBC10100EB011089
:10F44000007808282ADC09229DF8B40040F26921DE
:10F4500010FB01F0D34901EB8001A4319DF8A0001D
:10F4600000EBC00001EB0010027004E075E1F0E178
:10F47000FEE3FEE3FEE3A9229DF8B40040F2692119
:10F4800010FB01F0C74901EB8000A4309DF8A010EB
:10F4900001EBC10100EB01104271A7E09DF8B4003F
:10F4A00040F2692110FB01F0BE4901EB8000A4305D
:10F4B0009DF8A01001EBC10100EB011000780D28B0
:10F4C00024DC0E229DF8B40040F2692110FB01F00B
:10F4D000B44901EB8001A4319DF8A00000EBC0000D
:10F4E00001EB00100270A2229DF8B40040F26921E5
:10F4F00010FB01F0AB4901EB8000A4309DF8A01097
:10F5000001EBC10100EB011042716FE09DF8B40006
:10F5100040F2692110FB01F0A24901EB8000A43008
:10F520009DF8A01001EBC10100EB01104079A52866
:10F5300015D19DF8B40000EB400101EB00109A4991
:10F5400001EB001030309DF8A01000EB0110801C82
:10F550000A90007820F00400001D0A9908709DF8B8
:10F56000B40040F2692110FB01F08E4901EB8000EC
:10F57000A4309DF8A01001EBC10100EB01108078D0
:10F58000A12833D09DF8B40040F2692110FB01F0AE
:10F59000844901EB8001A4319DF8A00000EBC0007C
:10F5A00001EB001082789DF8B40040F2692110FB55
:10F5B00001F07C4901EB8001A4319DF8A00000EB33
:10F5C000C00001EB00104271A1229DF8B40040F28E
:10F5D000692110FB01F0734901EB8000A4309DF814
:10F5E000A01001EBC10100EB0110827001F02CBDF5
:10F5F00000219DF8B40040F2692210FB02F0694A34
:10F6000002EB8000C1709DF8B40040F2692110FB4C
:10F6100001F0114601EB8000A4309DF8A01001EB31
:10F62000C10100EB0110007805281DDC00219DF8C8
:10F63000B40040F2692210FB02F05A4A02EB80004B
:10F64000C17006229DF8B40040F2692110FB01F060
:10F65000544901EB8000A4309DF8A01001EBC101DA
:10F6600000EB0110027024E09DF8B40040F2692123
:10F6700010FB01F04B4901EB8000A4309DF8A01075
:10F6800001EBC10100EB01100078092811DC0A220E
:10F690009DF8B40040F2692110FB01F0414901EBF3
:10F6A0008000A4309DF8A01001EBC10100EB011017
:10F6B00002709DF8B40040F2692110FB01F0394955
:10F6C00001EB8000A4309DF8A01001EBC10100EB1C
:10F6D00001104079A4282DD19DF8B40000EB400121
:10F6E00001EB0010304901EB001030309DF8A01004
:10F6F00000EB0110801C0A90007820F020002030E0
:10F700000A99087000229DF8B40040F2692110FBAC
:10F7100001F0244901EB8000A4309DF8A01001EB1A
:10F72000C10100EB011080F83D209DF8B4100220CB
:10F73000FAF710FCA1229DF8B40040F2692110FBF9
:10F7400001F0184901EB8000A4309DF8A01001EBF6
:10F75000C10100EB0110427148E70020399015E02B
:10F760009DF8B40000EB4001C1EBC0100F4901EB64
:10F77000C001BDF8E400C01C0A5C17A9BDF8E40094
:10F780000A54BDF8E400401C81B23991BDF8E40090
:10F790000628E5DB062117A822F008FA0021CDE9AA
:10F7A000300105E0D445002014410020D87A002023
:10F7B000DDE93021100A40EA0160801841EB212187
:10F7C0004FF480724FF00003CDE90801F8F7FAFC1E
:10F7D0009DF8B40040F2692110FB01F0FE4901EBF5
:10F7E0008000A4309DF8A01001EBC10100EB0110D6
:10F7F000027100209DF8B41040F2692211FB02F161
:10F80000F54A02EB8101C87001229DF8B40040F274
:10F81000692110FB01F0F04901EB8000A4309DF854
:10F82000A01001EBC10100EB01100270A7229DF8AE
:10F83000B40040F2692110FB01F0E74901EB8000C0
:10F84000A4309DF8A01001EBC10100EB0110427142
:10F85000CCE69DF8B40040F2692110FB01F0DE49CE
:10F8600001EB8000A4309DF8A01001EBC10100EB7A
:10F870000110007806282EDC00219DF8B40040F22B
:10F88000692210FB02F0D44A02EB8000C17007220B
:10F890009DF8B40040F2692110FB01F0CE4901EB64
:10F8A0008001A4319DF8A00000EBC00001EB001026
:10F8B0000270A7229DF8B40040F2692110FB01F00C
:10F8C000C54901EB8000A4309DF8A01001EBC101F7
:10F8D00000EB011042719DF8B40040F2692110FB69
:10F8E00001F0BD4901EB8000A4309DF8A01001EBB0
:10F8F000C10100EB0110007801282FDC00219DF8E8
:10F90000B40040F2692210FB02F0B34A02EB80001F
:10F91000C17002229DF8B40040F2692110FB01F091
:10F92000AD4901EB8001A4319DF8A00000EBC000BF
:10F9300001EB00100270A3229DF8B40040F269218F
:10F9400010FB01F0A44901EB8000A4309DF8A01049
:10F9500001EBC10100EB011042711DE29DF8B40002
:10F9600040F2692110FB01F09B4901EB8000A430BB
:10F970009DF8A01001EBC10100EB011000780728F1
:10F980002FDC00219DF8B40040F2692210FB02F048
:10F99000914A02EB8000C17008229DF8B40040F249
:10F9A000692110FB01F08C4901EB8001A4319DF825
:10F9B000A00000EBC00001EB00100270A3229DF834
:10F9C000B40040F2692110FB01F0834901EB800093
:10F9D000A4309DF8A01001EBC10100EB01104271B1
:10F9E000DAE19DF8B40040F2692110FB01F07A4998
:10F9F00001EB8000A4309DF8A01001EBC10100EBE9
:10FA0000011000780B282FDC00219DF8B40040F293
:10FA1000692210FB02F0704A02EB8000C1700C22D8
:10FA20009DF8B40040F2692110FB01F06A4901EB36
:10FA30008001A4319DF8A00000EBC00001EB001094
:10FA40000270A1229DF8B40040F2692110FB01F080
:10FA5000614901EB8000A4309DF8A01001EBC101C9
:10FA600000EB0110427197E19DF8B40040F269216A
:10FA700010FB01F0584901EB8000A4309DF8A01064
:10FA800001EBC10100EB011000780C282FDC0021F4
:10FA90009DF8B40040F2692210FB02F04E4A02EBDE
:10FAA0008000C1700D229DF8B40040F2692110FB66
:10FAB00001F0494901EB8001A4319DF8A00000EB61
:10FAC000C00001EB00100270A3229DF8B40040F2C8
:10FAD000692110FB01F0404901EB8000A4309DF842
:10FAE000A01001EBC10100EB0110427154E19DF83F
:10FAF000B40040F2692110FB01F0374901EB8000AE
:10FB0000A4309DF8A01001EBC10100EB01100078BA
:10FB10000E287CDC0F229DF8B40040F2692110FB16
:10FB200001F02D4901EB8001A4319DF8A00000EB0C
:10FB3000C00001EB00100270A1229DF8B40040F259
:10FB4000692110FB01F0244901EB8001A4319DF8EB
:10FB5000A00000EBC00001EB001042719DF8B40062
:10FB600040F2692110FB01F01B4901EB8001A43137
:10FB70009DF8A00000EBC00001EB001082709DF822
:10FB8000B40000EB400101EB0010144901EB00113F
:10FB900030319DF8A00000E0FEE301EB0010801C76
:10FBA0000A90007820F0800080300A9908709DF853
:10FBB000B40000EB400101EB0010084901EB00101C
:10FBC00030309DF8A01000EB0110801C0A900078E6
:10FBD00020F00400001D03E0D44500201441002063
:10FBE0000A9908709DF8B40000EB400101EB001089
:10FBF000FE4901EB001030309DF8A01000EB011021
:10FC00008078C0F34010B0B39DF8B40000E045E048
:10FC100000EB400101EB0010F44901EB0010303023
:10FC20009DF8A01000EB0110801C0A90007820F0D5
:10FC300020020A9802709DF8B40000EB400101EB2D
:10FC40000010EA4901EB001030309DF8A01000EBE5
:10FC500001108078C0F34000D0B99DF8B40000EBEB
:10FC6000400101EB0010E14901EB0010303003E0EE
:10FC700093E0C1E003E171E09DF8A01000EB0110FA
:10FC8000801C0A90007820F0080008300A9908705B
:10FC90009DF8B4100220FAF75DF97DE09DF8B400FC
:10FCA00040F2692110FB01F0D14901EB8001A43140
:10FCB0009DF8A00000EBC00001EB001001789DF85A
:10FCC000B40040F2692210FB02F0C94A02EB800046
:10FCD0000079814260D19DF8B40040F2692110FBA7
:10FCE00001F0114601EB8000A4309DF8A01001EB5B
:10FCF000C10100EB01108078A12830D0A3229DF82B
:10FD0000B40040F2692110FB01F0B94901EB800118
:10FD1000A4319DF8A00000EBC00001EB001042717F
:10FD20009DF8B40040F2692110FB01F0B04901EBED
:10FD30008000A4309DF8A01001EBC10100EB011080
:10FD40008078A22828D000209DF8B41040F26922C3
:10FD500011FB02F1A64A02EB8101C8701CE0A1224E
:10FD60009DF8B40040F2692110FB01F0A04901EBBD
:10FD70008001A4319DF8A00000EBC00001EB001051
:10FD8000427101219DF8B40040F2692210FB02F09B
:10FD9000974A02EB8000C17028E4A1229DF8B400CC
:10FDA00040F2692110FB01F0914901EB8001A4317F
:10FDB0009DF8A00000EBC00001EB001082709DF8E0
:10FDC000B40040F2692110FB01F0894901EB800188
:10FDD000A4319DF8A00000EBC00001EB00104271BF
:10FDE00000219DF8B40040F2692210FB02F0804A25
:10FDF00002EB8000C170AFE49DF8B40040F26921CD
:10FE000010FB01F07A4901EB8000A4309DF8A010AE
:10FE100001EBC10100EB0110007806282EDC002167
:10FE20009DF8B40040F2692210FB02F0704A02EB28
:10FE30008000C17007229DF8B40040F2692110FBD8
:10FE400001F06B4901EB8001A4319DF8A00000EBAB
:10FE5000C00001EB00100270A7229DF8B40040F230
:10FE6000692110FB01F0624901EB8001A4319DF88A
:10FE7000A00000EBC00001EB001042716CE4002117
:10FE80009DF8B40040F2692210FB02F0584A02EBE0
:10FE90008000C170A7229DF8B40040F2692110FBD8
:10FEA00001F0534901EB8001A4319DF8A00000EB63
:10FEB000C00001EB001042719DF8B40000EB40015E
:10FEC000C1EBC0104B4901EBC000407930287CD118
:10FED0009DF8B40040F2692110FB01F0444901EBA8
:10FEE0008001A4319DF8A00000EBC00001EB0010E0
:10FEF00001789DF8B40040F2692210FB02F03C4A00
:10FF000002EB8000007981425FD19DF8B40000EBE4
:10FF1000400101EB0010354901EB001030309DF835
:10FF2000A01000EB0110801C0A90007820F0010264
:10FF30000A9802709DF8B40000EB400101EB00103C
:10FF40002A4901EB001030309DF8A01000EB0110A1
:10FF5000801C0A90007820F002020A9802709DF836
:10FF6000B40040F2692110FB01F0214901EB80004F
:10FF7000A4309DF8A01001EBC10100EB0110C07886
:10FF800031282ED19DF8B40000EB400101EB0010A8
:10FF9000164901EB001030309DF8A01000EB011065
:10FFA000801C0A90007820F020020A98027000223B
:10FFB0009DF8B40040F2692110FB01F00C4901EBFF
:10FFC0008000A4309DF8A01000E038E001EBC101F2
:10FFD00000EB011080F83D209DF8B4100220F9F7E5
:10FFE000B9FF9DF8B40040F2692105E014410020FA
:10FFF000D4450020D87A002010FB01F0FE4901EB27
:020000040801F1
:100000008000A4309DF8A01001EBC10100EB0110AD
:1000100090F83E00012811D1A9229DF8B40040F2C9
:10002000692110FB01F0F44901EB8000A4309DF838
:10003000A01001EBC10100EB0110827078E29DF885
:10004000B40000EB4001C1EBC010EC4901EBC00073
:10005000407931287DD19DF8B40040F2692110FB30
:1000600001F0E54901EB8001A4319DF8A00000EB0F
:10007000C00001EB001001789DF8B40040F2692245
:1000800010FB02F0DC4A02EB80000079814260D173
:100090009DF8B40040F2692110FB01F0114601EB1C
:1000A0008000A4309DF8A01001EBC10100EB01100D
:1000B00090F83E0040BB01229DF8B40040F2692157
:1000C00010FB01F0CC4901EB8001A4319DF8A000A8
:1000D00000EBC00001EB001080F83D209DF8B4005B
:1000E00000EB400101EB0010C54901EB001130317C
:1000F0009DF8A00001EB0010801C0A90007820F011
:100100000100401C0A9908709DF8B40000EB400102
:1001100001EB0010BA4901EB001030309DF8A0103F
:1001200000EB0110801C0A90007820F002020A986F
:100130000270B44890F8A008E8BBB348407F01289B
:1001400039D1B148D0F81402AF49C98B884232D2B4
:1001500000E0A8E09DF8B40040F2692110FB01F036
:10016000A54901EB8000A4309DF8A01001EBC1016E
:1001700000EB011090F83D0001281CD19DF8B4005F
:1001800040F2692110FB01F09B4901EB8000A43093
:100190009DF8A01001EBC10100EB011090F87D006B
:1001A00048B94FF010429DF8B40040F2692110FBAD
:1001B00001F0914900E075E001EB8001A4319DF868
:1001C000A00000EBC00001EB001082609DF8B400BD
:1001D00000EB400101EB0010894901EB00113031C7
:1001E0009DF8A00001EB001001789DF8B40040F2EA
:1001F000692210FB02F0804A02EB800041709DF8FA
:10020000B40040F2692110FB01F0114601EB8001BE
:10021000A4319DF8A00000EBC00001EB00100178B4
:100220009DF8B40040F2692210FB02F0724A02EB22
:1002300080000079814235D100229DF8B40040F25F
:10024000692110FB01F06C4901EB8001A4319DF89C
:10025000A00000EBC00001EB0010C271A4229DF8C9
:10026000B40040F2692110FB01F0634901EB800109
:10027000A4319DF8A00000EBC00001EB00108270DB
:10028000A3229DF8B40040F2692110FB01F05A4905
:1002900001EB8000A4309DF8A01001EBC10100EB40
:1002A0000110427144E19DF8B40000EB4001C1EB44
:1002B000C010524901EBC000407933286DD19DF840
:1002C000B40000EB400101EB00104D4901EB0010C0
:1002D00030309DF8A01000EB0110801C0A900078CF
:1002E00020F00100401C0A9908709DF8B40000EB52
:1002F000400101EB0010424901EB001030309DF845
:10030000A01000EB0110801C0A90007820F0200261
:100310000A9802709DF8B40000EB400101EB001058
:10032000374901EB001030309DF8A01000EB0110B0
:10033000801C0A90007820F00200801C0A99087046
:100340009DF8B40040F2692110FB01F02A4901EB4D
:10035000800002799DF8B40040F2692110FB01F0A1
:10036000254901EB8000A4309DF8A01001EBC101EC
:1003700000EB011002709DF8B40000EB400101EBAE
:1003800000101F4901EB001030309DF8A01000EB69
:100390000110801C0A9001E076E33BE0007820F039
:1003A000800180310A9801709DF8B40000EB400193
:1003B00001EB0010124901EB001030309DF8A01045
:1003C00000EB01108078C0F3400020B99DF8B41014
:1003D0000220F9F7BFFDA2229DF8B40040F2692186
:1003E00010FB01F0044901EB8000A4309DF8A0103F
:1003F00001EBC1010AE00000D4450020D87A0020BA
:1004000014410020BC320020BC12002000EB01107F
:1004100082708DE09DF8B40000EB4001C1EBC0108C
:10042000FE4901EBC000407934287DD19DF8B4002D
:1004300000EB400101EB0010F94901EB00103030F6
:100440009DF8A01000EB0110801C0A90007820F0AD
:1004500020020A9802709DF8B40000EB400101EB05
:100460000010EF4901EB001030309DF8A01000EBB8
:100470000110801C0A90007820F002020A98027095
:1004800001229DF8B40040F2692110FB01F0E5491A
:1004900001EB8000A4309DF8A01001EBC10100EB3E
:1004A000011080F83E20A9229DF8B40040F2692195
:1004B00010FB01F0DB4901EB8000A4309DF8A01097
:1004C00001EBC10100EB011082709DF8B40040F215
:1004D000692110FB01F0D34901EB800002799DF8FE
:1004E000B40040F2692110FB01F0CE4901EB80011C
:1004F000A4319DF8A00000EBC00001EB00100270D9
:100500009DF8B40000EB400101EB0010C44901EB81
:10051000001130319DF8A00001EB0010801C0A9002
:10052000007820F0800000E002E080300A99087036
:1005300000202E902F900021399122E0DDE92E102D
:10054000000140EA11720901CDE92E129DF8B400B4
:1005500000EB4001C1EBC010B04901EBC001BDF898
:10056000E400801D085C3038C117DDE92E3440EA14
:1005700003022143CDE92E21BDF8E400401C81B2E5
:100580003991BDF8E4000628D8DB9DF8B4002E9917
:1005900040F2692210FB02F0A24A02EB8002A43270
:1005A0009DF8A00000EBC00002EB0010C0F81A108C
:1005B00000222E922F920021399122E0DDE92E10A7
:1005C000000140EA11720901CDE92E129DF8B40034
:1005D00000EB4001C1EBC010904901EBC001BDF838
:1005E000E4000D30085C3038C117DDE92E3440EAF4
:1005F00003022143CDE92E21BDF8E400401C81B265
:100600003991BDF8E4000428D8DB9DF8B4002E9998
:1006100040F2692210FB02F0824A02EB8002A4320F
:100620009DF8A00000EBC00002EB00104163002227
:100630002E922F920021399122E0DDE92E10000147
:1006400040EA11720901CDE92E129DF8B40000EBC9
:100650004001C1EBC010714901EBC001BDF8E400DD
:100660001130085C3038C117DDE92E34184341EAF7
:100670000402CDE92E02BDF8E400401C80B239909E
:10068000BDF8E4000628D8DB9DF8B4002E9940F2AE
:10069000692210FB02F0634A02EB8002A4329DF84B
:1006A000A00000EBC00002EB0010C0F81E109DF887
:1006B000B40000EB4001C1EBC010584901EBC00091
:1006C00042799DF8B40040F2692110FB01F05549D0
:1006D00001EB8001A4319DF8A00000EBC00001EB0C
:1006E0000010C2709DF8B40000EB400101EB001057
:1006F0004B4901EB001130319DF8A00001EB0010D7
:1007000082789DF8B40040F2692110FB01F0454960
:1007100001EB8001A4319DF8A00000EBC00001EBCB
:10072000001002769DF8B40040F2692110FB01F040
:100730003C4901EB8001A4319DF8A00000EBC00012
:1007400001EB001001789DF8B40040F2692210FB23
:1007500002F0344A02EB8000007981427EDA002107
:100760009DF8B40040F2692210FB02F02D4A02EB22
:100770008000C170A7229DF8B40040F2692110FBEF
:1007800001F0284901EB8001A4319DF8A00000EBA5
:10079000C00001EB0010427101219DF8B40040F24D
:1007A000692210FB02F01F4A02EB8000C1709DF825
:1007B000B40040F2692110FB01F0114601EB80000A
:1007C00002799DF8B40040F2692110FB01F015494F
:1007D00001EB8001A4319DF8A00000EBC00001EB0B
:1007E00000100270A1229DF8B40040F2692110FBB4
:1007F00001F00C4901EB8001A4319DF8A00000EB51
:10080000C00001EB001042719DF8B40000EB400104
:1008100001EB0010024901EB001105E0D87A00203D
:1008200014410020D445002030319DF8A00001EB98
:100830000010801C0A90007820F0800080300A9917
:1008400008709DF8B40000EB400101EB0010FE4978
:1008500001EB001030309DF8A01000E059E000EBF3
:100860000110801C0A90007820F00401091D0A98EC
:1008700001709DF8B40000EB400101EB0010F2495B
:1008800001EB001030309DF8A01000EB01108078D3
:10089000C0F34010E8B39DF8B40000EB400101EB59
:1008A0000010E94901EB001030309DF8A01000EB7A
:1008B0000110801C0A90007820F020020A98027033
:1008C0009DF8B40000EB400101EB0010DE4901EBA4
:1008D000001030309DF8A01000EB01108078C0F3BC
:1008E0004000E8BB9DF8B40000EB400101EB0010B4
:1008F000D54901EB001030309DF8A01000EB01103D
:10090000801C0A90007820F0080008300A990870CE
:1009100000E0B8E09DF8B4009DF8A01001EB0010D5
:10092000C217CDE92E0200222E9800EBC00101EB88
:100930000011C64800EB8100C0F81D209DF8B400EE
:1009400040F2692110FB01F0C14901EB8000A430A5
:100950009DF8A01001EBC10100EB0110223000E076
:100960008CE00A902E9800EBC00101EB0011B74813
:1009700000EB81010D3110220991DDE90901F7F742
:1009800064FC9DF8B40040F2692110FB01F0B0490D
:1009900001EB8001A4319DF8A00000EBC00001EB49
:1009A00000112E9800EBC00202EB0012A74800EBEA
:1009B000820051F81A2F40F8012F496841609DF8D4
:1009C000B40000EB400101EB00109F4901EB001166
:1009D00030319DF8A00001EB001001782E9800EB5B
:1009E000C00202EB0012994800F822102E9800EB8A
:1009F000C00101EB0011954800EB81019548826927
:100A000041F8212F808B88809DF8B40040F2692145
:100A100010FB01F08E4901EB8001A4319DF8A0008C
:100A200000EBC00001EB0010416B2E9800EBC00200
:100A300002EB0012854800EB8200C0F809109DF817
:100A4000B40000EB400101EB00107F4901EB001105
:100A500030319DF8A00001EB001041682E9800EBAA
:100A6000C00202EB0012794800EB8200C0F82710A8
:100A70002E9881B208200A91F9F76CFA9DF8B4100B
:100A80000220F9F767FADFE200219DF8B40040F296
:100A9000692210FB02F06E4A02EB8000C1709DF8E3
:100AA000B40040F2692110FB01F0114601EB800017
:100AB000A4309DF8A01001EBC10100EB01100078FB
:100AC0000A2812DC0B229DF8B40040F2692110FBC9
:100AD00001F05F4901EB8000A4309DF8A01001EB0C
:100AE000C10100EB0110027005E29DF8B40040F274
:100AF000692110FB01F0564901EB8001A4319DF8FA
:100B0000A00000EBC00001EB001001789DF8B400DC
:100B100040F2692210FB02F04D4A02EB800000799E
:100B200081427DD14B4890F8A008E8BB4A48D0F8F4
:100B300014020521B0FBF1F201FB120000EBC00131
:100B400001EB00114448203000EB81000021C0F887
:100B50001D104148D0F814020521B0FBF1F201FB51
:100B6000120000EBC00101EB00113B48203000EB0C
:100B700081000D300A909DF8B40040F2692110FB0D
:100B800001F0334901EB8001A4319DF8A00000EB96
:100B9000C00001EB001022301022014609900A9893
:100BA000F7F753FB2C4800E0C5E0D0F8140205210C
:100BB000B0FBF1F201FB120000EBC00101EB0011F0
:100BC0002548203000EB81029DF8B40040F26921F5
:100BD00010FB01F01E4901EB8001A4319DF8A0003B
:100BE00000EBC00001EB001050F81A1F42F8011F83
:100BF000406850601848D0F814020521B0FBF1F2AB
:100C000001FB120000EBC00101EB0013124920317F
:100C10009DF8B40000EB400202EB00100A4A00E02D
:100C200069E102EB001230329DF8A00002EB0010E7
:100C3000007801F823000848D0F814020521B0FB21
:100C4000F1F201FB120009E014410020E014002041
:100C5000D4450020BC320020BC12002000EBC001B3
:100C600001EB0011FA4800EB81029DF8B40040F25C
:100C7000692110FB01F0F74901EB8001A4319DF8D7
:100C8000A00000EBC00001EB0010406BC2F80900AF
:100C9000EF482038D0F814020521B0FBF1F201FB37
:100CA000120000EBC00101EB0011E94800EB8101EB
:100CB00000F5FF50826941F8212F808B8880E4483D
:100CC0002038D0F814020521B0FBF1F081B20220E7
:100CD0000A91F8F7FDF900210620F9F73BF9DC4805
:100CE0002038D0F81402DA492039C98B884208D25A
:100CF000D7482038D0F81402401CD5492039C1F813
:100D0000140200210520F9F725F99DF8B40000EB45
:100D1000400101EB0010D04901EB001030309DF88C
:100D2000A01000EB0110801C0A90007820F008024F
:100D30000A98027015E09DF8B40000EB400101EB49
:100D40000010C54901EB001030309DF8A01000EBF9
:100D50000110801C0A90007820F0080008300A99E1
:100D6000087000229DF8B40040F2692110FB01F0E8
:100D7000B84901EB8001A4319DF8A00000EBC00050
:100D800001EB001080F83E209DF8B4100220F9F726
:100D9000E1F89DF8B4109DF8A00000EB0110C21717
:100DA000CDE92E0200222E9800EBC00101EB0011CC
:100DB000AA4800EB8100C0F81D209DF8B40040F265
:100DC000692110FB01F0A34901EB8000A4309DF8DC
:100DD000A01001EBC10100EB011022300A902E9807
:100DE00000EBC00101EB00119C4800EB81010D31CB
:100DF00010220991DDE90901F7F727FA9DF8B400FF
:100E000040F2692110FB01F0924901EB8001A4310D
:100E10009DF8A00000EBC00001EB00112E9800EB44
:100E2000C00202EB00128D4800EB820051F81A2F2D
:100E300040F8012F496841609DF8B40000EB400183
:100E400001EB0010844901EB001130319DF8A00046
:100E500001EB001001782E9800EBC00202EB0012AB
:100E60007E4800F822102E9800EBC00101EB001123
:100E70007A4800EB81017A48826941F8212F808B02
:100E800088809DF8B40040F2692110FB01F071499F
:100E900001EB8001A4319DF8A00000EBC00001EB44
:100EA0000010416B2E9800EBC00202EB00126B4861
:100EB00000EB8200C0F809109DF8B40000EB40017F
:100EC00001EB0010644901EB001130319DF8A000E6
:100ED00001EB001041682E9800EBC00202EB0012FB
:100EE0005E4800EB8200C0F827102E9881B20820DF
:100EF0000A91F9F72FF8A7229DF8B40040F2692172
:100F000010FB01F0534901EB8001A4319DF8A000D2
:100F100000EBC00001EB00104271A2229DF8B4006A
:100F200040F2692110FB01F04A4901EB8001A43134
:100F30009DF8A00000EBC00001EB001082700022C1
:100F40002E922F920021399122E0DDE92E1000012E
:100F500040EA11720901CDE92E129DF8B40000EBB0
:100F60004001C1EBC0103F4901EBC001BDF8E400F6
:100F70000B30085C3038C117DDE92E34184341EAE4
:100F80000402CDE92E02BDF8E400401C80B2399085
:100F9000BDF8E4000A28D8DB9DF8B400DDE92E1284
:100FA00040F2692310FB03F02A4B03EB8003A433C8
:100FB0009DF8A00000EBC00003EB001040F8221FDA
:100FC000426000222E922F920021399122E0DDE929
:100FD0002E10000140EA11720901CDE92E129DF890
:100FE000B40000EB4001C1EBC0101E4901EBC00191
:100FF000BDF8E4001530085C3038C117DDE92E2457
:10100000104341EA0402CDE92E02BDF8E400401C81
:1010100080B23990BDF8E4000A28D8DB9DF8B4000E
:10102000DDE92E1240F2692310FB03F0094B03EBBC
:101030008000A4309DF8A03003EBC30300EB031045
:1010400022308160C26000BF00BF06F0A0BE000079
:10105000DC120020D445002014410020E0140020C0
:10106000BC320020D87A00209DF8B40000EB40018B
:10107000C1EBC010FC4911F83000042801D12690C2
:101080000BE09DF8B40000EB4001C1EBC010F64945
:1010900011F83000152800D126909DF8B40000EB1F
:1010A0004001C1EBC010F04901EBC00041789DF850
:1010B000B40000EB4002C2EBC010EB4A12F8300063
:1010C00041EA002041F23001884202D1A620269058
:1010D0003DE09DF8B40000EB4001C1EBC010E249D7
:1010E00001EBC00041789DF8B40000EB4002C2EB78
:1010F000C010DD4A12F8300041EA002041F231010F
:10110000884202D1A720269021E09DF8B40000EB90
:101110004001C1EBC010D44911F83000022816D1AB
:101120009DF8B40000EB4001C1EBC010CE4901EBCB
:10113000C00001799DF8B40000EB4002C2EBC01082
:10114000C94A02EBC000C07841EA002126919DF80F
:10115000B40040F2692110FB01F0C44901EB8000AA
:10116000817828910021C24A9DF8B40002EB001258
:101170009DF8A0001154BF48007F012815D19DF8AB
:10118000B40000EB400101EB0010BB4901EB001083
:1011900030309DF8A01000EB0110801C0A90007800
:1011A00020F0800080300A9908709DF8B40000EBB0
:1011B000400101EB0010B04901EB001030309DF808
:1011C000A01000EB0110801C0A90007820F0400075
:1011D00040300A990870BDF89800A7287ED006DC38
:1011E00004287CD015287BD0A6284AD14AE0A0F557
:1011F0005850303820B1112873D01228F5D1FCE3B3
:101200009DF8B40040F2692110FB01F0974901EB11
:101210008000A4309DF8A01001EBC10100EB01108B
:10122000007870BB00219DF8B40040F2692210FBE9
:1012300002F08E4A02EB8000C17001229DF8B400DA
:1012400040F2692110FB01F0884901EB8001A431D3
:101250009DF8A00000EBC00001EB00100270A72277
:101260009DF8B40040F2692110FB01F07F4901EBC9
:101270008000A4309DF8A01001EBC10100EB01102B
:101280004271FDE300219DF8B40040F2692210FB99
:1012900002F0764A02EB8000C1709DF8B40040F283
:1012A000692110FB01F0114601EB8000A4309DF88C
:1012B000A01001EBC10100EB01100078022829DC2D
:1012C00003229DF8B40040F2692110FB01F0674948
:1012D00001EB8001A4319DF8A00003E0CEE02CE1F9
:1012E00056E284E200EBC00001EB00100270A9227C
:1012F0009DF8B40040F2692110FB01F05B4901EB5D
:101300008000A4309DF8A01001EBC10100EB01109A
:101310004271A7E09DF8B40040F2692110FB01F092
:10132000524901EB8000A4309DF8A01001EBC101EF
:1013300000EB01100078052824DC06229DF8B4009B
:1013400040F2692110FB01F0484901EB8001A43112
:101350009DF8A00000EBC00001EB00100270A2227B
:101360009DF8B40040F2692110FB01F03F4901EB08
:101370008000A4309DF8A01001EBC10100EB01102A
:1013800042716FE09DF8B40040F2692110FB01F05A
:10139000364901EB8000A4309DF8A01001EBC1019B
:1013A00000EB01104079A52815D19DF8B40000EBA1
:1013B000400101EB0010304901EB001030309DF886
:1013C000A01000EB0110801C0A90007820F00400AF
:1013D000001D0A9908709DF8B40040F2692110FBC5
:1013E00001F0224901EB8000A4309DF8A01001EB30
:1013F000C10100EB01108078A12833D09DF8B40022
:1014000040F2692110FB01F0184901EB8001A43181
:101410009DF8A00000EBC00001EB001082789DF861
:10142000B40040F2692110FB01F0104901EB80018A
:10143000A4319DF8A00000EBC00001EB0010427148
:10144000A1229DF8B40040F2692110FB01F0074988
:1014500001EB8000A4309DF8A01001EBC10100EB6E
:10146000011082700DE70000D87A0020D4450020DA
:10147000483F0020BC120020144100209DF8B40019
:1014800040F2692110FB01F0FE4901EB8000A4301D
:101490009DF8A01001EBC10100EB01104079A428D8
:1014A0002DD19DF8B40000EB400101EB0010F6498E
:1014B00001EB001030309DF8A01000EB0110801CF3
:1014C0000A90007820F0200120310A980170002253
:1014D0009DF8B40040F2692110FB01F0E94901EBED
:1014E0008001A4319DF8A00000EBC00001EB0010CA
:1014F00080F83D209DF8B4100220F8F72BFD002164
:101500009DF8B40040F2692210FB02F0DD4A02EBC4
:101510008000C170A1229DF8B40040F2692110FB47
:1015200001F0D84901EB8000A4309DF8A01001EB38
:10153000C10100EB01104271A3E69DF8B40040F236
:10154000692110FB01F0CF4901EB8000A4309DF828
:10155000A01001EBC10100EB0110007801282FDC85
:1015600000219DF8B40040F2692210FB02F0C54A48
:1015700002EB8000C17002229DF8B40040F26921A4
:1015800010FB01F0BF4901EB8001A4319DF8A000E0
:1015900000EBC00001EB00100270A3229DF8B40024
:1015A00040F2692110FB01F0B64901EB8001A43142
:1015B0009DF8A00000EBC00001EB00104271E6E0D6
:1015C0009DF8B40040F2692110FB01F0AD4901EB38
:1015D0008000A4309DF8A01001EBC10100EB0110C8
:1015E000007804282FDC00219DF8B40040F2692225
:1015F00010FB02F0A34A02EB8000C17005229DF8A7
:10160000B40040F2692110FB01F09E4901EB80011A
:10161000A4319DF8A00000EBC00001EB00100270A7
:10162000A3229DF8B40040F2692110FB01F0954916
:1016300001EB8000A4309DF8A01001EBC10100EB8C
:1016400001104271A3E09DF8B40040F2692110FB43
:1016500001F08C4901EB8000A4309DF8A01001EB53
:10166000C10100EB01100078062812DCA1229DF8D0
:10167000B40040F2692110FB01F0824901EB8000C7
:10168000A4309DF8A01001EBC10100EB01104271E4
:101690007DE09DF8B40040F2692110FB01F079492A
:1016A00001EB8001A4319DF8A00000EBC00001EB2C
:1016B000001001789DF8B40040F2692210FB02F09E
:1016C000704A02EB80000079814260D19DF8B4003D
:1016D00040F2692110FB01F0114601EB8000A430BB
:1016E0009DF8A01001EBC10100EB01108078A1284A
:1016F00030D0A3229DF8B40040F2692110FB01F024
:10170000604901EB8001A4319DF8A00000EBC0000E
:1017100001EB001042719DF8B40040F2692110FB0A
:1017200001F0584901EB8000A4309DF8A01001EBB6
:10173000C10100EB01108078A22828D000209DF87C
:10174000B41040F2692211FB02F14E4A02EB810112
:10175000C8701CE0A1229DF8B40040F2692110FB82
:1017600001F0484901EB8001A4319DF8A00000EB95
:10177000C00001EB0010427101219DF8B40040F25D
:10178000692210FB02F03F4A02EB8000C17078E54D
:10179000A1229DF8B40040F2692110FB01F0394903
:1017A00001EB8001A4319DF8A00000EBC00001EB2B
:1017B000001042719DF8B40040F2692110FB01F065
:1017C000304901EB8001A4319DF8A00000EBC0007E
:1017D00001EB0010827000219DF8B40040F26922F4
:1017E00010FB02F0274A02EB8000C17049E500219E
:1017F0009DF8B40040F2692210FB02F0214A02EB8E
:101800008000C170A7229DF8B40040F2692110FB4E
:1018100001F01C4901EB8001A4319DF8A00000EB10
:10182000C00001EB001042719DF8B40000EB4001D4
:10183000C1EBC010154901EBC000407930287CD1C4
:101840009DF8B40040F2692110FB01F00D4901EB55
:101850008001A4319DF8A00000EBC00001EB001056
:1018600001789DF8B40040F2692210FB02F0054AAD
:1018700002EB8000007981425FD19DF8B40000EB5B
:10188000400105E0D445002014410020D87A002012
:1018900001EB0010A2F5986101EB001030309DF8CB
:1018A000A01000EB0110801C0A90007820F00102CB
:1018B0000A9802709DF8B40000EB400101EB0010A3
:1018C000FE4901EB001030309DF8A01000EB011034
:1018D000801C0A90007820F002020A9802709DF89D
:1018E000B40040F2692110FB01F0F54901EB8000E2
:1018F000A4309DF8A01001EBC10100EB0110C078ED
:1019000031282ED19DF8B40000EB400101EB00100E
:10191000EA4901EB001030309DF8A01000EB0110F7
:10192000801C0A90007820F020020A9802700022A1
:101930009DF8B40040F2692100E039E010FB01F0AD
:10194000DF4901EB8000A4309DF8A01001EBC1013C
:1019500000EB011080F83D209DF8B4100220F8F74C
:10196000F9FA9DF8B40040F2692110FB01F0D44966
:1019700001EB8000A4309DF8A01001EBC10100EB49
:10198000011090F83E00012811D1A9229DF8B40061
:1019900040F2692110FB01F0C94901EB8001A4313B
:1019A0009DF8A00000EBC00001EB001082707AE20D
:1019B0009DF8B40000EB4001C1EBC010C14901EB40
:1019C000C000407931287DD19DF8B40040F26921F2
:1019D00010FB01F0BA4901EB8001A4319DF8A00091
:1019E00000EBC00001EB001001789DF8B40040F25C
:1019F000692210FB02F0B24A00E0E9E302EB80004A
:101A0000007981425ED19DF8B40040F2692110FB5B
:101A100001F0114601EB8000A4309DF8A01001EB0D
:101A2000C10100EB011090F83E0040BB01229DF87F
:101A3000B40040F2692110FB01F0A14901EB8001E3
:101A4000A4319DF8A00000EBC00001EB001080F86D
:101A50003D209DF8B40000EB400101EB00119748D8
:101A600000EB011130319DF8A00001EB0010801C4B
:101A70000A90007820F00100401C0A99087000E0EC
:101A8000FEE39DF8B40000EB400101EB00108B4930
:101A900001EB001030309DF8A01000EB0110801C0D
:101AA0000A90007820F002020A980270864890F8A6
:101AB000A008E8BB8548407F012839D18348D0F889
:101AC000140200E0ACE08149C98B884230D29DF815
:101AD000B40040F2692110FB01F0794901EB80006C
:101AE000A4309DF8A01001EBC10100EB011090F8AB
:101AF0003D0001281CD19DF8B40040F2692110FB83
:101B000001F06F4901EB8000A4309DF8A01001EBBB
:101B1000C10100EB011090F87D0048B94FF0104270
:101B20009DF8B40040F2692110FB01F0644900E027
:101B300075E001EB8001A4319DF8A00000EBC0002E
:101B400001EB001082609DF8B40000EB400101EB56
:101B500000105A4901EB001130319DF8A00001EB53
:101B6000001001789DF8B40040F2692210FB02F0E9
:101B7000534A02EB800041709DF8B40040F26921A5
:101B800010FB01F0114601EB8001A4319DF8A0008B
:101B900000EBC00001EB001001789DF8B40040F2AA
:101BA000692210FB02F0464A02EB80000079814274
:101BB00035D100229DF8B40040F2692110FB01F0FC
:101BC0003F4901EB8001A4319DF8A00000EBC0006B
:101BD00001EB0010C271A4229DF8B40040F269210B
:101BE00010FB01F0364901EB8001A4319DF8A00003
:101BF00000EBC00001EB00108270A3229DF8B4003E
:101C000040F2692110FB01F02D4901EB8001A43164
:101C10009DF8A00000EBC00001EB0010427142E112
:101C20009DF8B40000EB4001C1EBC010254901EB69
:101C3000C000407933287DD19DF8B40000EB40010D
:101C400001EB00101D4901EB001030309DF8A01091
:101C500000EB0110801C0A90007820F00100401C6D
:101C60000A9908709DF8B40000EB400101EB0010E8
:101C7000124901EB001030309DF8A01000EB01106C
:101C8000801C0A90007820F020020A9802709DF8CB
:101C9000B40000EB400101EB0010084901EB00101B
:101CA00030309DF8A01000EB0110801C0A900078E5
:101CB00020F00200801C0A99087009E014410020FD
:101CC000D4450020D87A0020BC320020BC1200206D
:101CD0009DF8B40040F2692110FB01F0FE4901EBD0
:101CE000800002799DF8B40040F2692110FB01F0F8
:101CF000F94901EB8000A4309DF8A01001EBC1016F
:101D000000EB011002709DF8B40000EB400101EB04
:101D10000010F24901EB001030309DF8A01000EBEC
:101D20000110801C0A90007820F0800180310A9810
:101D3000017000E029E09DF8B40000EB400101EBE8
:101D40000010E64901EB001030309DF8A01000EBC8
:101D500001108078C0F3400020B99DF8B410022033
:101D6000F8F7F8F8A2229DF8B40040F2692110FBC0
:101D700001F0D94901EB8000A4309DF8A01001EBDF
:101D8000C10100EB011082708DE09DF8B40000EB02
:101D90004001C1EBC010D24901EBC00040793428AA
:101DA0007ED19DF8B40000EB400101EB0010CB495F
:101DB00001EB001030309DF8A01000EB0110801CEA
:101DC0000A90007820F020020A9802709DF8B40072
:101DD00000EB400101EB0010C04901EB0010303076
:101DE0009DF8A01000EB0110801C0A90007820F0F4
:101DF00002020A98027001229DF8B40040F26921A3
:101E000010FB01F0B44901EB8000A4309DF8A01054
:101E100001EBC10100EB011080F83E20A9229DF8E2
:101E2000B40040F2692110FB01F0AB4901EB8000E6
:101E3000A4309DF8A01001EBC10100EB01108270ED
:101E40009DF8B40040F2692110FB01F0A24901EBBA
:101E5000800002799DF8B40040F2692110FB01F086
:101E60009D4901EB8000A4309DF8A01001EBC10159
:101E700000EB011002709DF8B40000EB400101EB93
:101E80000010964901EB001030309DF8A01000EBD7
:101E90000110801C0A90007820F08000803000E063
:101EA00001E00A99087000202E902F9000213991AE
:101EB00022E0DDE92E10000140EA11720901CDE9AE
:101EC0002E129DF8B40000EB4001C1EBC010844914
:101ED00001EBC001BDF8E400801D085C3038C1177B
:101EE000DDE92E34184341EA0402CDE92E02BDF8A3
:101EF000E400401C80B23990BDF8E4000828D8DB2B
:101F00009DF8B4002E9940F2692210FB02F0724A4B
:101F100002EB8002A4329DF8A00000EBC00002EBAF
:101F20000010C0F81A1000222E922F920021399131
:101F300022E0DDE92E10000140EA11720901CDE92D
:101F40002E129DF8B40000EB4001C1EBC0106449B3
:101F500001EBC001BDF8E4000F30085C3038C11758
:101F6000DDE92E3440EA03022143CDE92E21BDF8FC
:101F7000E400401C81B23991BDF8E4000628D8DBAA
:101F80009DF8B4002E9940F2692210FB02F0524AEB
:101F900002EB8002A4329DF8A00000EBC00002EB2F
:101FA0000010416300222E922F920021399122E0ED
:101FB000DDE92E10000140EA11720901CDE92E126F
:101FC0009DF8B40000EB4001C1EBC010444901EBA7
:101FD000C001BDF8E4001530085C3038C117DDE9F8
:101FE0002E3440EA03022143CDE92E21BDF8E4005E
:101FF000401C81B23991BDF8E4000828D8DB9DF877
:10200000B4002E9940F2692210FB02F0324A02EB32
:102010008002A4329DF8A00000EBC00002EB00108B
:10202000C0F81E109DF8B40000EB4001C1EBC010D9
:102030002B4901EBC00042799DF8B40040F26921C0
:1020400010FB01F0244901EB8001A4319DF8A000B0
:1020500000EBC00001EB0010C2709DF8B40000EB73
:10206000400101EB00101D4901EB001130319DF8DA
:10207000A00001EB001082789DF8B40040F26921C5
:1020800010FB01F0144901EB8001A4319DF8A00080
:1020900000EBC00001EB001002769DF8B40040F2A6
:1020A000692110FB01F00C4901EB8001A4319DF87E
:1020B000A00000EBC00001EB001001789DF8B40017
:1020C00040F2692210FB02F0034A02EB8000007923
:1020D00081427CDA002105E0D44500201441002033
:1020E000D87A00209DF8B40040F2692210FB02F07B
:1020F000FE4A02EB8000C170A7229DF8B40040F2B6
:10210000692110FB01F0F94901EB8001A4319DF830
:10211000A00000EBC00001EB0010427101219DF80E
:10212000B40040F2692210FB02F0F04A02EB80009A
:10213000C1709DF8B40040F2692110FB01F0114616
:1021400001EB800002799DF8B40040F2692110FB98
:1021500001F0E64901EB8001A4319DF8A00000EBFD
:10216000C00001EB00100270A1229DF8B40040F203
:10217000692110FB01F0DD4901EB8001A4319DF8DC
:10218000A00000EBC00001EB001042719DF8B4000C
:1021900000EB400101EB0010D54901EB001130319B
:1021A0009DF8A00001EB0010801C0A90007820F040
:1021B000800080300A9908709DF8B40000EB40015F
:1021C00001EB0010CA4901EB0010303001E058E08B
:1021D00017E19DF8A01000EB0110801C0A90007818
:1021E00020F00400001D0A9908709DF8B40000EB6F
:1021F000400101EB0010BE4901EB001030309DF8AA
:10220000A01000EB01108078C0F34010C8B39DF817
:10221000B40000EB400101EB0010B54901EB0010E8
:1022200030309DF8A01000EB0110801C0A9000785F
:1022300020F020020A9802709DF8B40000EB4001E3
:1022400001EB0010AA4901EB001030309DF8A010FE
:1022500000EB01108078C0F34000E8BB9DF8B400AB
:1022600000EB400101EB0010A14901EB0010303000
:102270009DF8A01000EB0110801C0A90007801E08E
:10228000BAE3BDE020F0080108310A9801709DF81A
:10229000B4109DF8A00000EB0110C217CDE92E028A
:1022A00000222E9800EBC00101EB0011914800EBD9
:1022B0008100C0F81D209DF8B41040F2692011FB88
:1022C00000F08A4901EB8000A4309DF8A01001EBDA
:1022D000C10100EB011000E08DE022300A902E9841
:1022E00000EBC00101EB0011824800EB81010D31D0
:1022F00010220991DDE90901F5F7A7FF9DF8B40067
:1023000040F2692110FB01F0784901EB8001A43112
:102310009DF8A00000EBC00001EB00112E9800EB2F
:10232000C00202EB0012734800EB820051F81A2F32
:1023300040F8012F496841609DF8B40000EB40016E
:1023400001EB00106A4901EB001130319DF8A0004B
:1023500001EB001001782E9800EBC00202EB001296
:10236000644800F822102E9800EBC00101EB001128
:10237000604800EB81016048826941F8212F808B21
:1023800088809DF8B40040F2692110FB01F05749A4
:1023900001EB8001A4319DF8A00000EBC00001EB2F
:1023A0000010416B2E9800EBC00202EB0012514866
:1023B00000EB8200C0F809109DF8B40000EB40016A
:1023C00001EB00104A4901EB001130319DF8A000EB
:1023D00001EB001041682E9800EBC00202EB0012E6
:1023E000444800EB8200C0F827102E9881B20820E4
:1023F0000A91F7F7AFFD9DF8B4100220F7F7AAFD98
:10240000FAE200219DF8B40040F2692210FB02F0CC
:10241000364A02EB8000C1709DF8B40040F2692199
:1024200010FB01F0114601EB8000A4309DF8A010D4
:1024300001EBC10100EB01100078032812DC04223B
:102440009DF8B40040F2692110FB01F0274901EB2F
:102450008000A4309DF8A01001EBC10100EB011039
:10246000027000E29DF8B40040F2692110FB01F017
:102470001E4901EB8001A4319DF8A00000EBC000D3
:1024800001EB001001789DF8B40040F2692210FBC6
:1024900002F0164A02EB8000007981427ED1164894
:1024A00090F8A00808BB1548D0F814020521B0FB2D
:1024B000F1F201FB120000EBC00101EB00110F482B
:1024C000203000EB81000021C0F81D100B48D0F82F
:1024D00014020521B0FBF1F201FB120000EBC00178
:1024E00001EB0011054820300AE0DCE0D445002073
:1024F00014410020E0140020BC320020BC12002057
:1025000000EB81000D300A909DF8B40040F2692183
:1025100010FB01F0FE4901EB8001A4319DF8A00001
:1025200000EBC00001EB00102230102201460990A0
:102530000A98F5F78AFEF748D0F814020521B0FB97
:10254000F1F201FB120000EBC00101EB0011F148B8
:10255000203000EB81029DF8B40040F2692110FBAD
:1025600001F0EB4901EB8001A4319DF8A00000EBE4
:10257000C00001EB001050F81A1F42F8011F40681C
:102580005060E448D0F814020521B0FBF1F201FBE1
:10259000120000EBC00101EB001300E063E1DD4934
:1025A00020319DF8B40000EB400202EB0010DA4A43
:1025B00002EB001230329DF8A00002EB0010007810
:1025C00001F82300D348D0F814020521B0FBF1F242
:1025D00001FB120000EBC00101EB0011CD482030DF
:1025E00000EB81029DF8B40040F2692110FB01F07C
:1025F000C74901EB8001A4319DF8A00000EBC000A9
:1026000001EB0010406BC2F80900C248D0F8140278
:102610000521B0FBF1F201FB120000EBC00101EB60
:102620000011BC48203000EB810100F5FF508269A9
:1026300041F8212F808B8880B648D0F814020521FC
:10264000B0FBF1F081B202200A91F6F741FD0021C2
:102650000620F7F77FFCAF48D0F81402AD49C98BCC
:10266000884206D2AB48D0F81402401CA949C1F8F0
:10267000140200210520F7F76DFC9DF8B40000EB73
:10268000400101EB0010A44901EB001030309DF82F
:10269000A01000EB0110801C0A90007820F00802C6
:1026A0000A98027015E09DF8B40000EB400101EBC0
:1026B0000010994901EB001030309DF8A01000EB9C
:1026C0000110801C0A90007820F0080008300A9958
:1026D000087000229DF8B40040F2692110FB01F05F
:1026E0008B4901EB8001A4319DF8A00000EBC000F4
:1026F00001EB001080F83E209DF8B4100220F7F79F
:1027000029FC9DF8B4109DF8A00000EB0110C21741
:10271000CDE92E0200222E9800EBC00101EB001142
:102720007E4800EB8100C0F81D209DF8B40040F207
:10273000692110FB01F0764901EB8000A4309DF87F
:10274000A01001EBC10100EB011022300A902E987D
:1027500000EBC00101EB0011704800EB81010D316D
:1027600010220991DDE90901F5F76FFD9DF8B4002C
:1027700040F2692110FB01F0654901EB8001A431B1
:102780009DF8A00000EBC00001EB00112E9800EBBB
:10279000C00202EB0012614800EB820051F81A2FD0
:1027A00040F8012F496841609DF8B40000EB4001FA
:1027B00001EB0010584901EB001130319DF8A000E9
:1027C00001EB001001782E9800EBC00202EB001222
:1027D000524800F822102E9800EBC00101EB0011C6
:1027E0004E4800EB81014E48826941F8212F808BD1
:1027F00088809DF8B40040F2692110FB01F0444943
:1028000001EB8001A4319DF8A00000EBC00001EBBA
:102810000010416B2E9800EBC00202EB00123F4803
:1028200000EB8200C0F809109DF8B40000EB4001F5
:1028300001EB0010384901EB001130319DF8A00088
:1028400001EB001041682E9800EBC00202EB001271
:10285000324800EB8200C0F827102E9881B2082081
:102860000A91F7F777FB00229DF8B40040F2692146
:1028700010FB01F0264901EB8001A4319DF8A00076
:1028800000EBC00001EB001080F83E20A7229DF86D
:10289000B40040F2692110FB01F01D4901EB8001F9
:1028A000A4319DF8A00000EBC00001EB00104271C4
:1028B000A2229DF8B40040F2692110FB01F01449F6
:1028C00001EB8001A4319DF8A00000EBC00001EBFA
:1028D0000010827000222E922F92002139912FE059
:1028E000DDE92E10000140EA11720901CDE92E1236
:1028F0009DF8B40000EB4001C1EBC010094901EBA9
:10290000C001BDF8E4000B30085C3038C1170BE0A3
:10291000D4450020BC12002014410020E014002007
:10292000BC320020D87A0020DDE92E34184341EA79
:102930000402CDE92E02BDF8E400401C80B23990BB
:10294000BDF8E4000C28CBDB9DF8B400DDE92E12C5
:1029500040F2692310FB03F0FE4B03EB8003A4332A
:102960009DF8A00000EBC00003EB001040F8221F10
:10297000426000222E922F920021399122E0DDE95F
:102980002E10000140EA11720901CDE92E129DF8C6
:10299000B40000EB4001C1EBC010EF4901EBC001F6
:1029A000BDF8E4001730085C3038C117DDE92E347B
:1029B00040EA03022143CDE92E21BDF8E400401C8A
:1029C00081B23991BDF8E4000C28D8DB9DF8B40041
:1029D000DDE92E1240F2692310FB03F0DD4B03EB1F
:1029E0008000A4309DF8A03003EBC30300EB03107C
:1029F00022308160C26000BF00BF05F0C8B900216D
:102A0000D64A9DF8B40002EB00129DF8A0001154C4
:102A10009DF8B40000EB4001C1EBC010CE4901EBC2
:102A2000C000407870280ED19DF8B40000EB400142
:102A3000C1EBC010C84901EBC0008078FA2802D170
:102A4000B120269042E09DF8B40000EB4001C1EBBC
:102A5000C010C14901EBC000407800F0F000C02870
:102A60000ED19DF8B40000EB4001C1EBC010BA4993
:102A700001EBC0008078FA2802D1B620269025E02C
:102A80009DF8B40000EB4001C1EBC011B24810F852
:102A9000310000F0F000502818D19DF8B40000EB90
:102AA0004001C1EBC010AC4901EBC000407800F020
:102AB000F00030280AD19DF8B40000EB4001C1EBD2
:102AC000C010A54901EBC000817826919DF8B400A3
:102AD00040F2692110FB01F09E4901EB80008178F2
:102AE000289100219D4A9DF8B40002EB00129DF848
:102AF000A00011549DF8B40000EB400101EB001060
:102B0000974901EB001130319DF8A00001EB001056
:102B1000801C0A90007820F0400040300A9908702C
:102B20009048007F012815D19DF8B40000EB4001CA
:102B300001EB00108A4901EB001030309DF8A01025
:102B400000EB0110801C0A90007820F0800080309B
:102B50000A990870BDF89800652874D004DC012833
:102B600009D0032805D175E0B12802D0B62800D1DC
:102B700000E083E182E19DF8B40000EB4001C1EB8D
:102B8000C011754800EBC1000079012806D0022869
:102B900005D0032804D005285AD102E058E057E0B8
:102BA00056E09DF8B40040F2692110FB01F069493C
:102BB00001EB8000A4309DF8A01001EBC10100EBF7
:102BC00001100078F0BB00219DF8B40040F26922AA
:102BD00010FB02F05F4A02EB8000C17001229DF8F9
:102BE000B40040F2692110FB01F05A4901EB800169
:102BF000A4319DF8A00000EBC00001EB00100270B2
:102C0000B6229DF8B40040F2692110FB01F0514951
:102C100001EB8001A4319DF8A00000EBC00001EBA6
:102C200000104271B2229DF8B40040F2692110FBFD
:102C300001F0484901EB8000A4309DF8A01001EBA1
:102C4000C10101E003E02DE000EB0110827000BF44
:102C500000BF13E19DF8B40000EB4001C1EBC010D0
:102C60003D4901EBC000C1793F4880F8101E9DF836
:102C7000B40000EB400101EB0010394901EB0011F9
:102C800030319DF8A00001EB0010801C0A903648FE
:102C900090F8100EC2080A98007862F300000A99B2
:102CA0000870EBE09DF8B40000EB4001C1EBC010F0
:102CB000294901EBC000007900F0F00010B9B820FC
:102CC000269001E0B92026909DF8B40000EB400169
:102CD000C1EBC010204901EBC000007900F00F01EA
:102CE00027910021399120E09DF8B40000EB4001CC
:102CF00001EB00101A4901EB00113031BDF8E4007E
:102D000001EB001041789DF8B40000EB4002C2EBEB
:102D1000C010114A12F830005038814200D112E040
:102D2000BDF8E400401C81B239919DF8B40000EB7D
:102D3000400101EB00100A4901EB0010C179BDF818
:102D4000E4008142D0DC00BFBDF8E4109DF89C0097
:102D500008440BE0D4450020D87A0020483F0020EA
:102D600014410020BC120020BC220020C1B22891D6
:102D70009DF8B40040F2692110FB01F0FE4901EB1F
:102D80008000A4309DF8A01001EBC10100EB011000
:102D9000007801282FD100219DF8B40040F269226B
:102DA00010FB02F0F44A02EB8000C17002229DF891
:102DB000B40040F2692110FB01F0EF4901EB800102
:102DC000A4319DF8A00000EBC00001EB00100270E0
:102DD000B9229DF8B40040F2692110FB01F0E649E8
:102DE00001EB8000A4309DF8A01001EBC10100EBC5
:102DF0000110427141E09DF8B40040F2692110FBDE
:102E000001F0DD4901EB8000A4309DF8A01001EB3A
:102E1000C10100EB0110007801282ED100219DF89E
:102E2000B40040F2692210FB02F0D34A02EB8000AA
:102E3000C17002229DF8B40040F2692110FB01F03C
:102E4000CD4901EB8001A4319DF8A00000EBC0004A
:102E500001EB00100270B9229DF8B40040F2692124
:102E600010FB01F0C44901EB8001A4319DF8A000E2
:102E700000EBC00001EB0010427100BF00BFBCE5D9
:102E80009DF8B40000EB400101EB0010BB4901EBE1
:102E90000010007B20B101287DD002287CD1E5E222
:102EA000B7499DF8B40031F81000801F81B20A9133
:102EB0009DF8B40000EB4001C1EBC010B14901EB3B
:102EC000C000401C09900A99F6F704FD0022CDE9E4
:102ED00030029DF8B40000EB4001C1EBC010A949DD
:102EE00001EBC002A6489DF8B41030F81100401F55
:102EF00011180A9104210A9819F048FBC217CDE96C
:102F00002E022FA815C82E995140604001437DD153
:102F10009D4A9DF8B40002EB001001709DF8B400CA
:102F200000EB4001C1EBC010964901EBC0000179F4
:102F30002691BDF89800312802D0452867D1EAE0F3
:102F40008F489DF8B41030F811001838412190FBDB
:102F5000F1F0C217C1B2CDE92E028C4880F8B81149
:102F600000203990CDE09DF8B40000EB4001C1EBAA
:102F7000C010844901EBC001BDF8E40000EB8010F3
:102F80001430095C824ABDF8E40011549DF8B40085
:102F900000EB400101E0C1E067E2C1EBC0107949FC
:102FA00001EBC001BDF8E40000EB80101A300144D1
:102FB0000A9108210A9819F0A7FA8DED0F0A744AB0
:102FC0000C32BDF8E4000F9902EB001041609DF84F
:102FD000B40000EB4001C1EBC0106A4901EBC00135
:102FE000BDF8E40000EB8010323001440A91082162
:102FF0000A9819F089FA8DED0F0A654A0C32BDF86E
:10300000E4000F9902EB0010016001E085E083E02D
:103010009DF8B40000EB4001C1EBC010594901EB31
:10302000C001BDF8E40000EB80103A3001440A9181
:1030300008210A9819F068FA8DED0F0A544A0C32EB
:10304000BDF8E4000F9902EB001081609DF8B40018
:1030500000EB4001C1EBC0104A4901EBC001BDF8D3
:10306000E40000EB8010423001440A9108210A98E4
:1030700019F04AFA8DED0F0A454A0C32BDF8E4000A
:103080000F9902EB0010C1609DF8B40000EB400105
:1030900001EB0010394901EB00113031BDF8E400BB
:1030A00001EB0010801C0A90007820F08000803036
:1030B0000A9908709DF8B40000EB4001C1EBC01004
:1030C000304901EBC0022E489DF8B41030F81100D1
:1030D000401E125C9DF8B40040F2692110FB01F023
:1030E000254901EB8000A4309DF8A01001EBC1013F
:1030F00000EB011080F83C20BDF8E400401C80B2D9
:103100003990BDF8E4000021DDE92E34C01AA14158
:10311000FFF629AF00E000BF00BFBCE29DF8B4009D
:1031200000EB4001C1EBC010164901EBC000407D2F
:103130009DF8B41001EB4102C2EBC111114A02EB40
:10314000C101897D40EA0120C217CDE92E029DF818
:10315000B40000EB4001C1EBC0100A4901EBC00113
:103160000A9115210A98F6F799FB0022CDE9300261
:103170002FA819C82E990DE0D44500201441002035
:10318000646C0020D87A0020483F0020BC32002028
:10319000753400205940604001437CD19DF8B40053
:1031A00000EB4001C1EBC011FD4810F83100401E9A
:1031B000C1B228910021FB4A9DF8B40002EB001235
:1031C0009DF8A0001154F84A9DF8A00011549FEDFD
:1031D000F70A10EE101A0C329DF8A00002EB001056
:1031E00041609DF8B40000EB4001C1EBC010EC4918
:1031F00001EBC00081799DF8B40000EB4002C2EB06
:10320000C010E74A02EBC000407941EA002000EE1E
:10321000100AB8EEC00A9FEDE61AC0EE010A9DF84A
:10322000B40000EB4001C1EBC010114601EBC0003F
:1032300001799DF8B40000EB4002C2EBC010D84AFF
:1032400002EBC000C07841EA002000EE100AB8EEA0
:10325000C00A30EE800A10EE101AD34A0C329DF8E4
:10326000A00002EB001001609DF8B40000EB4001EB
:10327000C1EBC010CA4901EBC000817A9DF8B400CF
:1032800000EB4002C2EBC010C54A02EBC000407A1E
:1032900041EA002000E0E8E000EE100AB8EEC00AC3
:1032A0009FEDC31AC0EE010A9DF8B40000EB400187
:1032B000C1EBC010114601EBC000017A9DF8B400CB
:1032C00000EB4002C2EBC010B54A02EBC000C0796F
:1032D00041EA002000EE100AB8EEC00A30EE800A83
:1032E00010EE101AB04A0C329DF8A00002EB00104C
:1032F00081609DF8B40000EB4001C1EBC010A8490B
:1033000001EBC000C07A00F0800038BB9DF8B4002B
:1033100000EB4001C1EBC010A14901EBC000017BF3
:103320009DF8B40000EB4002C2EBC0109C4A02EBD7
:10333000C000C07A41EA002000EE100AF8EEC00A90
:10334000B3EE001A80EE810A10EE100A964A0C3293
:103350009DF8A01002EB0111C86047E09DF8B40091
:1033600000EB4001C1EBC0108D4901EBC000017BB7
:103370009DF8B40000EB4002C2EBC010884A02EB9B
:10338000C000C07A41EA0020404280B200EE100A3C
:10339000B8EEC00A8DED030A0398F5F7BFF99FED6B
:1033A000850B53EC102BCDE904019DED040B51EC82
:1033B000100BF5F797F89FED810B53EC102BCDE92F
:1033C00006019DED060B51EC100BF5F716F8CDE953
:1033D00008019DED080B51EC100BF5F7B2F9724A9C
:1033E0000C329DF8A01002EB0111C8609DF8B400EA
:1033F00000EB400101EB0010724901EB001030308E
:103400009DF8A01000EB0110801C0A90007820F0BD
:10341000800180310A9801709DF8B40000EB4001F2
:10342000C1EBC0105E4901EBC000C27D9DF8B40045
:1034300040F2692110FB01F0634901EB8001A431E6
:103440009DF8A00000EBC00001EB001080F83C20CC
:103450009DF8B40000EB400101EB0010594901EB6D
:103460000010C179594880F8B81114E19DF8B410E2
:1034700001EB4100C0EBC110494901EBC000C0792C
:103480009DF8B41001EB4102C2EBC111444A02EBBA
:10349000C101097A40EA0120C217CDE92E029DF848
:1034A000B41001EB4100C0EBC1103D4901EBC0017C
:1034B0000A9107210A98F6F7F1F90022CDE93002C6
:1034C000DDE93042DDE92E1061405040014366D114
:1034D0009DF8B41001EB4100C0EBC110304911F868
:1034E0003000401EC1B2289100212E4A9DF8B40040
:1034F00002EB001001702C4A9DF8A00011549DF8B9
:10350000B41001EB4100C0EBC110254901EBC00034
:10351000817908460191F5F77BF8CDE902019DED2F
:10352000021B9FED2B0B1DF0CBF98DED060B9DF8CB
:10353000B41001EB4100C0EBC110194901EBC00010
:1035400001799DF8B40000EB4002C2EBC010144AB0
:1035500002EBC000C07841EA002000EE100AB8EE8D
:10356000C00A8DED030A0398F5F7D8F8CDE90401F8
:103570009DED060B53EC102B9DED040B51EC100B45
:10358000F4F7B0FFCDE908019DED080B51EC100BED
:10359000F5F7D7F8044A0C329DF8A0101CE079E04A
:1035A000D87A0020483F0020753400200000000039
:1035B00000FF7F47000000000000304000000000D6
:1035C0000000000014410020D4450020BC3200203F
:1035D000000000000000244002EB011148601FEDD4
:1035E0000D0A10EE100A9DF8A01002EB0111086000
:1035F0001FED120A10EE100A9DF8A01002EB011147
:1036000088601FED160A10EE100A9DF8A01002EB5C
:103610000111C8609DF8B41001EB410000EB0110EE
:1036200002F6934101EB001030309DF8A01000EB42
:103630000110801C0A90007820F0800080300A99E8
:1036400008709DF8B41001EB4100C0EBC110F749C0
:1036500001EBC000427A9DF8B40040F2692110FBF2
:1036600001F0F34901EB8001A4319DF8A00000EBCB
:10367000C00001EB001080F83C209DF8B41001EB75
:10368000410000EB0110EB4901EB0010C179EA4861
:1036900080F8B81100BF00BF04F079BB9DF8B410EA
:1036A00001EB4100C0EBC110E04901EBC000C17863
:1036B0009DF8B40000EB4002C2EBC010DB4A02EB05
:1036C000C000807841EA002129919DF8B41001EBF7
:1036D0004100C0EBC110114601EBC001BDF8A400D0
:1036E000401C095C9DF8B40000EB4002C2EBC01026
:1036F000CE4A02EBC002BDF8A400105C41EA0020F3
:10370000C217CDE92E029DF8B41001EB4100C0EBC9
:10371000C110C64901EBC0000A90BDF8A410F6F72D
:10372000BDF80022CDE93002DDE93042DDE92E109E
:103730006140504001437DD19DF8B41001EB410040
:10374000C0EBC110B94901EBC000417828910021BC
:1037500039911CE09DF8B41001EB410000EB011021
:10376000B44901EB00113031BDF8E40001EB001069
:1037700041789DF8A000814204D1BDF8E400C1B2B7
:10378000289112E0BDF8E400401C81B239919DF807
:10379000B41001EB410000EB0110A64901EB001051
:1037A000C179BDF8E4008142D4DC00BF9DF8B410BB
:1037B00001EB410000EB01109E4901EB001030309D
:1037C0009DF8A01000EB0110801C0A90007820F0FA
:1037D000800180310A9801709DF8B41001EB41001E
:1037E000C0EBC110914901EBC00001792691002185
:1037F000924A9DF8B40002EB00129DF8A00011540B
:103800009DF8B41001EB410000EB0110894901EB78
:10381000001130319DF8A00001EB0010801C0A90CF
:10382000007820F0400040300A990870BDF89800F8
:10383000F22800E0F0E37DD006DC05287BD00628E6
:1038400009D0F12878D1E8E3F32876D0F42875D0B0
:10385000F628F7D1FDE30621119100213691F9E315
:10386000BDF84400401C81B211919DF8B41001EBE9
:103870004100C0EBC1106D4901EBC001BDF844002F
:10388000095C2691BDF84400401C81B21191BDF83D
:103890009800F12804D0F2287ED0F3287DD1FCE3F3
:1038A0009DF8B41001EB4100C0EBC1105F4901EB82
:1038B000C001BDF84400095C2991BDF84400401CDA
:1038C00081B211919DF8B40000EB400101EB0010B2
:1038D000584901EB001130319DF8A020BDF8D80007
:1038E000104401EB0010407A00F0010038B39DF85D
:1038F000B40040F2692110FB01F04D4901EB800159
:10390000A4319DF8A020BDF8D800104400EBC00001
:1039100001EB001090F88E0000F0010078B99DF8DE
:10392000B40040F2692110FB01F0414901EB800134
:10393000A43105E0FDE3FDE3FDE3FDE3FDE349E044
:103940009DF8A020BDF8D800104400EBC00001EBAA
:10395000001090F88000E8B3002139912FE09DF825
:10396000B40040F2692110FB01F0314901EB800104
:10397000A4319DF8A020BDF8D800104400EBC00091
:1039800001EB001000F18101BDF8E4000A5C9DF834
:10399000B40000EB400101E0A1E39FE301EB001064
:1039A000244901EB00100E30BDF8E410405C824267
:1039B00000D008E0BDF8E400401C81B23991BDF8A8
:1039C000E4000428CBDB00BFBDF8E400042860D18C
:1039D000042100E05DE0399137E09DF8B40040F249
:1039E000692110FB01F0124901EB8001A4319DF81F
:1039F000A020BDF8D800104400EBC00001EB00107F
:103A000000F18101BDF8E4000A5C9DF8B40000EB10
:103A1000400101EB0010074901EB00100E30BDF82A
:103A2000E410405C82420BD013E00000D87A002002
:103A3000D445002014410020BC320020483F002023
:103A4000BDF8E400401C81B23991BDF8E4000A28B9
:103A5000C3DB00BFBDF8E4000A281AD09DF8B4000B
:103A600040F2692110FB01F0FC4901EB8000A43019
:103A70009DF8A020BDF8D810114401EBC10100EB66
:103A800001108E300A90007820F00100401C0A9945
:103A90000870BDF8A4000F287ED19DF8B40000EB9B
:103AA000400101EB0010EE4901EB001130319DF8AF
:103AB000A020BDF8D800104401EB0010801C0A9033
:103AC000007820F00401091D0A9801700021399145
:103AD0002AE09DF8B40000EB4001C1EBC010E149C1
:103AE00001EBC001BDF84420BDF8E40010440A5CBD
:103AF0009DF8B40040F2692110FB01F0D74901EBB9
:103B00008001A4319DF8A030BDF8D800184400EB26
:103B1000C00001EB00113F31BDF8E4000A54BDF8CC
:103B2000E400401C81B23991BDF8E4000A28D0DBE2
:103B3000BDF844000A3081B21191002139912AE088
:103B40009DF8B40000EB4001C1EBC010C54901EB8A
:103B5000C001BDF84420BDF8E40010440A5C9DF8A3
:103B6000B40040F2692110FB01F0BC4901EB800177
:103B7000A4319DF8A030BDF8D800184400EBC00077
:103B800001EB00115831BDF8E4000A54BDF8E4001F
:103B9000401C81B2399100E040E2BDF8E400022807
:103BA000CEDBBDF84400801C81B211919DF8B400B9
:103BB00000EB4001C1EBC010AA4901EBC001BDF808
:103BC0004400085C01049DF8B40000EB4002C2EB25
:103BD000C010A44A02EBC002BDF84400401C105CB7
:103BE00041EA00219DF8B40000EB4002C2EBC01096
:103BF0009C4A02EBC002BDF84400801C105C0143EB
:103C00009DF8B40040F2692210FB02F0934A02EBE7
:103C10008002A4329DF8A030BDF8D800184400EB13
:103C2000C00002EB0010C166BDF84400C01C81B2A8
:103C300011918D4890F8A008F0BB002139911DE04A
:103C40009DF8B40040F2692110FB01F0834901EBBB
:103C50008001A4319DF8A020BDF8D800104400EBED
:103C6000C00001EB00103F30BDF8E410405C00B133
:103C700008E0BDF8E400401C81B23991BDF8E400D1
:103C80000A28DDDB00BFBDF8E4000A2818D1402275
:103C90009DF8B40040F2692110FB01F06F4901EB7F
:103CA0008001A4319DF8A030BDF8D800184400EB85
:103CB000C00001EB001000E055E080F876204CE1F8
:103CC0009DF8B40040F2692110FB01F0634901EB5B
:103CD0008001A4319DF8A020BDF8D800104400EB6D
:103CE000C00001EB001090F87600E0BB00202A90A5
:103CF0000DE10020379029E09DF8B40040F26921E1
:103D000010FB01F0554901EB8001A4319DF8A02082
:103D1000BDF8D800104400EBC00001EB00113F31AA
:103D2000BDF8DC00001D095C9DF8A80000EB400216
:103D30004E4800EB4202BDF8DC00105C814200D02E
:103D400008E0BDF8DC00401C81B23791BDF8DC0012
:103D50000628D1DB00BFBDF8DC0006287DD1032298
:103D60009DF8B40000E0F8E040F2692110FB01F09A
:103D70003A4901EB8001A4319DF8A030BDF8D8008C
:103D8000184400EBC00001EB001080F876209DF88D
:103D9000B40000EB400101EB0010314901EB0012CF
:103DA00030329DF8A000BDF8D810084402EB001096
:103DB000801C0A90007820F004020A98027000200B
:103DC00039901CE020229DF8B40040F2692110FBDC
:103DD00001F0224901EB8001A4319DF8A030BDF82B
:103DE000D800184400EBC00001EB00114931BDF8C8
:103DF000E4000A54BDF8E400401C81B23991BDF8DA
:103E0000E4000F28DEDB002039901CE020229DF822
:103E1000B40040F2692110FB01F0104901EB800170
:103E2000A4319DF8A030BDF8D800184400EBC000C4
:103E300001EB00115B31BDF8E4000A54BDF8E40069
:103E4000401C81B23991BDF8E4000A28DEDB002273
:103E50009DF8B40040F269210AE053E0D445002007
:103E600014410020D87A0020BC32002044350020C4
:103E700010FB01F0FE4901EB8001A4319DF8A03058
:103E8000BDF8D800184400EBC00001EB001080F82A
:103E90007020002139911CE000229DF8B40040F20E
:103EA000692110FB01F0F24901EB8001A4319DF87A
:103EB000A030BDF8D800184400EBC00001EB0011A1
:103EC0007131BDF8E4000A54BDF8E400401C81B231
:103ED0003991BDF8E4000528DEDB9DF8B40040F21E
:103EE000692110FB01F0E24901EB8001A4319DF84A
:103EF000A020BDF8D800104400EBC00001EB00107A
:103F0000C06E0CE09DF8A800401CC1B22A91D948AF
:103F1000B0F886029DF8A81088423FF7EAAE00BFCD
:103F2000D448B0F886029DF8A810884215D14022E6
:103F30009DF8B40040F2692110FB01F0CC4901EB7F
:103F40008001A4319DF8A030BDF8D800184400EBE2
:103F5000C00001EB001080F876209DF8B40040F21C
:103F6000692110FB01F0C24901EB8001A4319DF8E9
:103F7000A020BDF8D800104400EBC00001EB0010F9
:103F800090F87600032804D0112818D0402842D198
:103F90002BE0F2229DF8B40040F2692110FB01F001
:103FA000B34901EB8001A4319DF8A030BDF8D800E1
:103FB000184400EBC00001EB001042712BE0F3222B
:103FC0009DF8B40040F2692110FB01F0A84901EB13
:103FD0008001A4319DF8A030BDF8D800184400EB52
:103FE000C00001EB0010427115E0F2229DF8B40010
:103FF00040F2692110FB01F09D4901EB8001A431E1
:104000009DF8A030BDF8D800184400EBC00001EBCB
:104010000010427100BF61E0FEE3D7E09DF8B400FC
:1040200000EB400101EB0010934901EB001130312E
:104030009DF8A020BDF8D800104401EB0010801CB2
:104040000A90007820F004020A9802709DF8B400EB
:1040500001E0EFE3AAE040F2692110FB01F084499E
:1040600001EB8001A4319DF8A020BDF8D8001044D8
:1040700000EBC00001EB001090F88E0000F0010092
:1040800060B300229DF8B40040F2692110FB01F0FA
:10409000774901EB8001A43100E06BE09DF8A0308E
:1040A000BDF8D800184400EBC00001EB0010A0F8E8
:1040B0008C2005229DF8B40040F2692110FB01F02C
:1040C0006B4901EB8001A4319DF8A030BDF8D80008
:1040D000184400EBC00001EB0010427160E09DF855
:1040E000B40040F2692110FB01F0614901EB80014D
:1040F000A4319DF8A020BDF8D800104400EBC0000A
:1041000001EB001090F8760040281CD100229DF8A9
:10411000B40040F2692110FB01F0554901EB800128
:10412000A4319DF8A030BDF8D800184400EBC000C1
:1041300004E0F1E3F1E3F1E3F1E3F1E301EB00107B
:1041400080F8762000BF00BFF1229DF8B40040F255
:10415000692110FB01F0464901EB8001A4319DF873
:10416000A030BDF8D800184400EBC00001EB0010EF
:10417000427115E0F1229DF8B40040F2692110FB74
:1041800001F03B4901EB8001A4319DF8A030BDF85E
:10419000D800184400EBC00001EB0010427100BFD2
:1041A00000BFBDF8D800401C81B236919DF8B40024
:1041B00000EB4001C1EBC011304800EBC100417978
:1041C000BDF8D80081423FF74BABA7E39DF8B400A0
:1041D00040F2692110FB01F0254901EB8000A43079
:1041E0009DF8A01001EBC10100EB0110007820BB8D
:1041F00001229DF8B40040F2692110FB01F01C4936
:1042000001EB8001A4319DF8A00000EBC00001EBA0
:1042100000100270F4229DF8B40040F2692110FBF6
:1042200001F0134901EB8000A4309DF8A01001EBD0
:10423000C10100EB01104271C7E09DF8B40000EB32
:10424000400101EB00100C4901EB001030309DF8EB
:10425000A01000EB0110407A00F00100A0B39DF81F
:10426000B40040F2692110FB01F0014908E00000B0
:10427000D4450020BC32002014410020D87A002010
:1042800001EB8000A4309DF8A01001EBC10100EB10
:10429000011090F88E0000F00100A8B99DF8B4005C
:1042A00040F2692110FB01F0F74901EB8000A430D6
:1042B0009DF8A01001EBC10100EB011090F8800007
:1042C00010B1002039902AE07FE09DF8B40040F260
:1042D000692110FB01F0EC4901EB8001A4319DF84C
:1042E000A00000EBC00001EB001000F18101BDF85F
:1042F000E4000A5C9DF8B40000EB400101EB001003
:10430000E24901EB00100E30BDF8E410405C82423F
:1043100000D008E0BDF8E400401C81B23991BDF83E
:10432000E4000428D1DB00BFBDF8E40004284CD130
:10433000399029E09DF8B40040F2692110FB01F0AA
:10434000D14901EB8001A4319DF8A00000EBC00031
:1043500001EB001000F18101BDF8E4000A5C9DF85A
:10436000B40000EB400101EB0010C84901EB001064
:104370000E30BDF8E410405C824200D008E0BDF889
:10438000E400401C81B23991BDF8E4000A28D1DB79
:1043900000BFBDF8E4000A2817D09DF8B40040F231
:1043A000692110FB01F0B84901EB8000A4309DF8B1
:1043B000A01001EBC10100EB01108E300A900078D3
:1043C00020F00100401C0A990870BDF8A4001128D3
:1043D00071D19DF8B40000EB400101EB0010AB4936
:1043E00001EB001030309DF8A01000EB0110801C94
:1043F0000A90007820F00401091D0A98017000213C
:10440000399125E09DF8B40000EB4001C1EBC010EC
:104410009F4901EBC001BDF8E400401D0A5C9DF816
:10442000B40040F2692110FB01F0974901EB8001D3
:10443000A4319DF8A00000EBC00001EB00113F315A
:10444000BDF8E4000A54BDF8E400401C81B2399183
:10445000BDF8E4000A28D5DB0020399025E09DF85E
:10446000B40000EB4001C1EBC010894901EBC00171
:10447000BDF8E4000F300A5C9DF8B40040F26921F9
:1044800010FB01F0804901EB8001A4319DF8A000F0
:1044900000EBC00001EB00115831BDF8E4000A54F4
:1044A000BDF8E400401C81B23991BDF8E400022857
:1044B000D5DBBFE2FFE7BDF8A40014287DD19DF84D
:1044C000B40000EB400101EB0010704901EB00105B
:1044D00030309DF8A01000EB0110801C0A9000788D
:1044E00020F00401091D0A9801700021399125E08E
:1044F0009DF8B40000EB4001C1EBC010644901EB32
:10450000C001BDF8E400401D0A5C9DF8B40040F213
:10451000692110FB01F05C4901EB8001A4319DF899
:10452000A00000EBC00001EB00113F31BDF8E4003A
:104530000A54BDF8E400401C81B23991BDF8E40092
:104540000A28D5DB0020399025E09DF8B40000EB67
:104550004001C1EBC0104E4901EBC001BDF8E400C1
:104560000F300A5C9DF8B40040F2692110FB01F0A5
:10457000454901EB8001A4319DF8A00000EBC0008B
:1045800001EB00115831BDF8E4000A54BDF8E40015
:10459000401C81B23991BDF8E4000228D5DB9DF8BA
:1045A000B40000EB4001C1EBC010394901EBC00081
:1045B000407C01049DF8B40000E0ECE100EB400217
:1045C000C2EBC010324A02EBC000807C41EA0021FD
:1045D0009DF8B40000EB4002C2EBC0102C4A02EB85
:1045E000C000C07C01439DF8B40040F2692210FB7A
:1045F00002F0254A02EB8000A4309DF8A02002EBD7
:10460000C20200EB0210C166224890F8A008C8BBA5
:10461000002039901AE09DF8B40040F2692110FBA7
:1046200001F0194901EB8001A4319DF8A00000EBD5
:10463000C00001EB00103F30BDF8E410405C00B159
:1046400008E0BDF8E400401C81B23991BDF8E400F7
:104650000A28E0DB00BFBDF8E4000A281CD1402294
:104660009DF8B40040F2692110FB01F0064901EB0E
:104670008000A4309DF8A01001EBC10100EB0110F7
:1046800080F876202FE10000D4450020144100205E
:10469000D87A0020BC3200209DF8B40040F2692195
:1046A00010FB01F0FE4901EB8000A4309DF8A01042
:1046B00001EBC10100EB011090F87600F0BB002087
:1046C0002A90EDE00020379026E09DF8B40040F2FB
:1046D000692110FB01F0F24901EB8001A4319DF842
:1046E000A00000EBC00001EB00113F31BDF8DC0081
:1046F000001D095C9DF8A80000EB4002E94800EBB2
:104700004202BDF8DC00105C814200D008E0BDF838
:10471000DC00401C81B23791BDF8DC000628D4DBF8
:1047200000BFBDF8DC00062877D103229DF8B40055
:1047300040F2692110FB01F0D94900E0D3E001EB20
:104740008001A4319DF8A00000EBC00001EB001037
:1047500080F876209DF8B40000EB400101EB0010DA
:10476000D14901EB001030309DF8A01000EB011092
:10477000801C0A90007820F004020A980270002041
:10478000399019E020229DF8B40040F2692110FB15
:1047900001F0C34901EB8001A4319DF8A00000EBBA
:1047A000C00001EB00114931BDF8E4000A54BDF826
:1047B000E400401C81B23991BDF8E4000F28E1DB30
:1047C0000020399019E020229DF8B40040F26921C0
:1047D00010FB01F0B24901EB8001A4319DF8A0006B
:1047E00000EBC00001EB00115B31BDF8E4000A549E
:1047F000BDF8E400401C81B23991BDF8E4000A28FC
:10480000E1DB00229DF8B40040F2692110FB01F0C9
:10481000A34901EB800101E0AFE23CE0A4319DF847
:10482000A00000EBC00001EB001080F87020002118
:1048300039911AE057E100229DF8B40040F2692155
:1048400010FB01F0964901EB8001A4319DF8A00016
:1048500000EBC00001EB00117131BDF8E4000A5417
:10486000BDF8E400401C81B23991BDF8E400052890
:10487000E1DB9DF8B40040F2692110FB01F08849AA
:1048800001EB8000A4309DF8A01001EBC10100EB0A
:104890000110C06E0CE09DF8A800401CC1B22A9126
:1048A0008248B0F886029DF8A81088423FF70AAF08
:1048B00000BF7E48B0F886029DF8A810884212D149
:1048C00040229DF8B40040F2692110FB01F07449C8
:1048D00001EB8000A4309DF8A01001EBC10100EBBA
:1048E000011080F876209DF8B40040F2692110FB99
:1048F00001F06B4901EB8000A4309DF8A01001EBA2
:10490000C10100EB011090F87600032809D01128AE
:104910001AD040283ED12AE08DE0BDE12CE2CFE064
:1049200006E1F2229DF8B40040F2692110FB01F08B
:104930005B4901EB8000A4309DF8A01001EBC101A0
:1049400000EB0110427125E0F3229DF8B40040F223
:10495000692110FB01F0524901EB8000A4309DF861
:10496000A01001EBC10100EB0110427112E0F22234
:104970009DF8B40040F2692110FB01F0484901EBB9
:104980008001A4319DF8A00000EBC00001EB0010F5
:10499000427100BF4EE09DF8B40000EB400101EB16
:1049A0000010414901EB001030309DF8A01000EBE1
:1049B0000110801C0A90007820F004020A9802700E
:1049C0009DF8B40040F2692110FB01F0344901EB7D
:1049D0008000A4309DF8A01001EBC10100EB011094
:1049E00090F88E0000F0010020B300229DF8B40082
:1049F00040F2692110FB01F0294901EB8001A4314B
:104A00009DF8A00000EBC00001EB0010A0F88C2086
:104A100005229DF8B40040F2692110FB01F0204905
:104A200001EB8000A4309DF8A01001EBC10100EB68
:104A300001104271A0E19DF8B40040F2692110FB21
:104A400001F0174901EB8000A4309DF8A01001EBA4
:104A5000C10100EB011090F87600402813D100222C
:104A60009DF8B40040F2692110FB01F00C4901EB04
:104A70008000A4309DF8A01001EBC10100EB0110F3
:104A800080F8762000BF00BFF1229DF8B40040F20C
:104A9000692110FB01F0024901EB8000A43007E01E
:104AA000D44500204435002014410020BC320020B1
:104AB0009DF8A01001EBC10100EB011042715BE118
:104AC000F1229DF8B40040F2692110FB01F0FE498B
:104AD00001EB8001A4319DF8A00000EBC00001EBC8
:104AE0000010427148E103229DF8B40040F26921B0
:104AF00010FB01F0F44901EB8001A4319DF8A00006
:104B000000EBC00001EB00100270F1229DF8B40030
:104B100040F2692110FB01F0EB4901EB8000A43069
:104B20009DF8A01001EBC10100EB0110427123E1DF
:104B300002229DF8B40040F2692110FB01F0E24925
:104B400001EB8001A4319DF8A00000EBC00001EB57
:104B500000100270F6229DF8B40040F2692110FBAB
:104B600001F0D94901EB8001A4319DF8A00000EBD0
:104B7000C00001EB0010427101229DF8B40040F228
:104B8000692110FB01F0D04901EB8001A4319DF8AF
:104B9000A00000EBC00001EB001080F88020002195
:104BA000399126E09DF8B40000EB4001C1EBC01044
:104BB000C64901EBC001BDF8E400401D0A5C9DF848
:104BC000B40040F2692110FB01F0BF4901EB800104
:104BD000A4319DF8A00000EBC00001EB001000F133
:104BE0008101BDF8E4000A54BDF8E400401C81B224
:104BF0003991BDF8E4000A28D4DBBDF8A4001428DC
:104C000049D19DF8B40000EB4001C1EBC010AF49A1
:104C100001EBC000C27B9DF8B40040F2692110FB9B
:104C200001F0A94901EB8001A4319DF8A00000EB3F
:104C3000C00001EB001080F877200021399126E0B8
:104C40009DF8B40000EB4001C1EBC0109F4901EB9F
:104C5000C001BDF8E40010300A5C9DF8B40040F2D9
:104C6000692110FB01F0984901EB8001A4319DF806
:104C7000A00000EBC00001EB001000F17901BDF8CD
:104C8000E4000A54BDF8E400401C81B23991BDF83B
:104C9000E4000428D4DB6FE09DF8B40000EB400191
:104CA000C1EBC010894901EBC00081799DF8B400C7
:104CB00000EB4002C2EBC010844A02EBC000407916
:104CC00041EA00229DF8B40040F2692110FB01F096
:104CD0007D4901EB8001A4319DF8A00000EBC000EC
:104CE00001EB0010A0F88C209DF8B40040F269217F
:104CF00010FB01F0744901EB8001A4319DF8A00084
:104D000000EBC00001EB0010B0F88C109DF8B4006F
:104D100000EB400202EB00106D4A02EB0010408BEA
:104D2000814228DBF1229DF8B40040F2692110FB9A
:104D300001F0654901EB8001A4319DF8A00000EB72
:104D4000C00001EB001042719DF8B40040F26921EF
:104D500010FB01F05C4901EB8000A4309DF8A0102D
:104D600001EBC10100EB01108E300A90007820F0B9
:104D700001020A98027000BF00BF03F008B89DF856
:104D8000B40000EB4001C1EBC010504901EBC00082
:104D900001792891002136911CE09DF8B40000EBC8
:104DA000400101EB00104A4901EB00113031BDF820
:104DB000D80001EB001041789DF8A000814204D199
:104DC000BDF8D800C1B2289112E0BDF8D800401C4F
:104DD00081B236919DF8B40000EB400101EB001068
:104DE0003B4901EB0010C179BDF8D8008142D4DC09
:104DF00000BF9DF8B40000EB400101EB0010344906
:104E000001EB001030309DF8A01000EB0110801C69
:104E10000A90007820F0400140310A9801709DF816
:104E2000B40000EB4001C1EBC010284901EBC00009
:104E3000C1782691BDF89800172834D2DFE800F039
:104E4000330C0F331215181B1E3333333333332116
:104E5000242733332A2D30000720299023E0072010
:104E6000299020E0062029901DE0062029901AE0D4
:104E70000620299017E01220299014E0072029909D
:104E800011E0092029900EE0062029900BE0062071
:104E9000299008E00B20299005E00B20299002E0E2
:104EA0002A20299000BF00BFBDF8A400001FC1B296
:104EB0000A919DF8B40000EB4001C1EBC01003491A
:104EC00001EBC000C01C05E0D4450020D87A0020CA
:104ED0001441002009900A99F4F7FCFA37909DF8E4
:104EE000B40000EB4001C1EBC010FE4901EBC00172
:104EF000BDF8A400401E095CBDF8DC0081427DD1F4
:104F00009DF8B40000EB4001C1EBC010F54901EB86
:104F1000C0004078002871DD9DF8B40000EB40012E
:104F2000C1EBC010EF4901EBC001BDF8A4000A5C61
:104F30009DF8B40040F2692110FB01F0EA4901EB51
:104F40008001A4319DF8A00000EBC00001EB00102F
:104F500080F83C200021E54A9DF8B40002EB0012E5
:104F60009DF8A0001154E248007F012815D19DF85A
:104F7000B40000EB400101EB0010DE4901EB001032
:104F800030309DF8A01000EB0110801C0A900078D2
:104F900020F0800080300A990870BDF8980007283A
:104FA0007ED007DC07287CD2DFE800F07BFDFC7BAD
:104FB000FBFAF90010380728F5D2DFE810F0EF0906
:104FC000D2097200720007000800600500BFBDF83A
:104FD0009800142866D19DF8B40000EB4001C1EBA5
:104FE000C010C04901EBC000407901069DF8B40033
:104FF00000EB4002C2EBC010BA4A00E0FEE302EB55
:10500000C000807941EA00419DF8B40000EB400205
:10501000C2EBC010B34A02EBC000C07941EA0021E4
:105020009DF8B40000EB4002C2EBC010AD4A02EBA9
:10503000C000007A01439DF8B40040F2692210FBE1
:1050400002F0A94A02EB8002A4329DF8A00000EB16
:10505000C00002EB0010C0F81A109DF8B40040F236
:10506000692110FB01F0A04901EB8001A4319DF8FA
:10507000A00000EBC00001EB0010D0F81A100846A9
:105080000A9100210AF008FACDE92E019DF8B4003A
:1050900000EB400101EB0010964901EB001002E02B
:1050A000FEE3FEE380E0007F00F003019DF8B40022
:1050B00000EB400202EB00108E4A02EB0010007F72
:1050C000C0F3011001449DF8B40000EB400202EB74
:1050D0000010884A02EB0010007FC0F38100091A1B
:1050E00008460591F3F783FACDE906019DED061B0D
:1050F0009FED810B1BF0E4FB8DED080B9DED080B84
:1051000051EC100BF3F7E5FACDE930019DF8B4004E
:1051100040F2692110FB01F0734901EB8001A431D9
:105120009DF8A00000EBC00001EB0010416B0846A9
:10513000079100210AF0B0F9DDE92E32A0FB03450A
:1051400001FB035100FB021502220023DDE93001BF
:10515000F3F738F8231845EB0100CDE90830DDE915
:105160003023DDE90801F3F72DF8CDE92E01DDE963
:105170002E010AF051FF01469DF8B40040F2692269
:1051800010FB02F0584A02EB8000A4309DF8A020EA
:1051900002EBC20200EB0210C0F81E1048E0FDE373
:1051A00098E3CCE3FBE3DDE3BDF8980015283FD19D
:1051B0009DF8B40000EB4001C1EBC010494901EB80
:1051C000C000407901069DF8B40000EB4002C2EB3C
:1051D000C010444A02EBC000807941EA00419DF8CA
:1051E000B40000EB4002C2EBC0103E4A02EBC0002C
:1051F000C07941EA00219DF8B40000EB4002C2EB07
:10520000C010384A02EBC000007A01439DF8B40098
:1052100040F2692210FB02F0334A02EB8000A43016
:105220009DF8A02002EBC20200EB0210C0F81E1095
:105230009DF8B40000EB4001C1EBC010294901EB1F
:10524000C000417A2E4880F80F1E9DF8B40000EB94
:10525000400101EB0010274901EB001130319DF8AE
:10526000A00001EB0010801C0A90254890F80F0E5A
:10527000C2090A98007862F300000A990870204871
:1052800090F80F0E00F00300012806D01C4890F89B
:105290000F0E00F0030003283CD19DF8B40000EB92
:1052A000400101EB0010134901EB001030309DF874
:1052B000A01000EB0110801C0A90007820F0020181
:1052C000891C0A9801709DF8B40000EB400101EBC5
:1052D0000010084901EB001130319DF8A00001EBEE
:1052E00000100FE0D87A0020D4450020483F00206D
:1052F000BC120020144100200000000000002440E7
:10530000BC220020801C0A90007820F020020A981D
:10531000027014E09DF8B40000EB400101EB0010B6
:10532000FE4901EB001030309DF8A01000EB011099
:10533000801C0A90007820F002020A9802709DF802
:10534000B40000EB400101EB0010F44901EB001147
:1053500030319DF8A00001EB00108078C0F34002CE
:105360009DF8B40040F2692110FB01F0EC4901EB1B
:105370008000A4309DF8A01001EBC10100EB0110EA
:10538000007EC0F34000824266D09DF8B40040F237
:10539000692110FB01F0E24901EB8000A4309DF887
:1053A000A01001EBC10100EB011018300A909DF82C
:1053B000B40000EB400101EB0010D84901EB0010F4
:1053C00030309DF8A01000EB0110807842080A9858
:1053D000007862F341000A9908709DF8B40000EB70
:1053E000400101EB0010CD4901EB001030309DF879
:1053F000A01000EB01108078C0F3400038BB9DF88E
:10540000B40000EB400101EB0010C44901EB0010B7
:1054100030309DF8A01000EB0110801C0A9000783D
:1054200020F020020A98027001229DF8B40040F298
:10543000692110FB01F0BA4901EB8000A4309DF80E
:10544000A01001EBC10100EB011080F83E209DF897
:10545000B4100220F4F77EFD9DF8B40000EB40018B
:1054600001EB0010AD4901EB001130319DF8A000B7
:1054700001EB0010807800F001029DF8B40040F2CA
:10548000692110FB01F0A64901EB8000A4309DF8D2
:10549000A01001EBC10100EB0110007E00F0010043
:1054A00082425FD09DF8B40040F2692110FB01F008
:1054B0009B4901EB8000A4309DF8A01001EBC101D5
:1054C00000EB011018300A909DF8B40000EB400189
:1054D00001EB0010914901EB001130319DF8A00063
:1054E00001EB001081780A98027861F300020270E3
:1054F0009DF8B40000EB400101EB0010874901EB7F
:10550000001030309DF8A01000EB0110807800F002
:10551000010040BB9DF8B40000EB400101EB00101E
:105520007E4901EB001030309DF8A01000EB011017
:10553000801C0A90007820F020020A980270002255
:105540009DF8B40040F2692110FB01F0744901EBB1
:105550008000A4309DF8A01001EBC10100EB011008
:1055600080F83D2012E19DF8B40040F2692110FB63
:1055700001F06B4901EB8000A4309DF8A01001EB15
:10558000C10100EB011090F83E0098B901229DF88E
:10559000B40040F2692110FB01F0614901EB800089
:1055A000A4309DF8A01001EBC10100EB011080F8C0
:1055B0003D2027E000229DF8B40040F2692110FB55
:1055C00001F0574901EB8001A4319DF8A00000EBE8
:1055D000C00001EB001080F83D209DF8B40000EB06
:1055E000400101EB00104D4901EB001030309DF8F7
:1055F000A01000EB0110801C0A90007820F001023E
:105600000A980270474890F8A008E0BB4648407FDF
:10561000012838D14448D0F814024349C98B884244
:1056200031D29DF8B40040F2692110FB01F03C49F1
:1056300001EB8000A4309DF8A01001EBC10100EB4C
:10564000011090F83D0001281DD19DF8B40040F2F2
:10565000692110FB01F0324901EB8000A4309DF874
:10566000A01001EBC10100EB011090F87D0050B9D2
:105670009DF8B40000EB400101EB0010274901EB5D
:105680000011303100E081E09DF8A00001EB001036
:1056900001789DF8B40040F2692210FB02F0204A24
:1056A00002EB8000417005229DF8B40040F26921B0
:1056B00010FB01F01A4901EB8001A4319DF8A00014
:1056C00000EBC00001EB0010427100229DF8B40015
:1056D00000EB400101EB0010104901EB00113031EB
:1056E0009DF8A00001EB001042609DF8B41002206C
:1056F000F4F730FC0021399123E000229DF8B4003A
:1057000040F2692110FB01F0054901EB8001A43151
:105710009DF8A00000EBC00008E00000144100204C
:10572000D4450020BC320020BC12002001EB001147
:105730003F31BDF8E4000A54BDF8E400401C81B2DA
:105740003991BDF8E4001428D7DB0020399019E026
:1057500000229DF8B40040F2692110FB01F0FE49DF
:1057600001EB8001A4319DF8A00000EBC00001EB2B
:1057700000115B31BDF8E4000A54BDF8E400401CA0
:1057800081B23991BDF8E4000A28E1DB9DF8B4004C
:1057900040F2692110FB01F0EF4901EB8000A430D9
:1057A0009DF8A01001EBC10100EB01100078012869
:1057B00012DC02229DF8B40040F2692110FB01F0D6
:1057C000E54901EB8000A4309DF8A01001EBC10178
:1057D00000EB011002707CE09DF8B40040F26921FA
:1057E00010FB01F0DC4901EB8000A4309DF8A01013
:1057F00001EBC10100EB0110007800E0F9E30228A1
:105800002FDC00219DF8B40040F2692210FB02F069
:10581000D14A02EB8000C17003229DF8B40040F22F
:10582000692110FB01F0CC4901EB8001A4319DF806
:10583000A00000EBC00001EB0010027007229DF8F1
:10584000B40040F2692110FB01F0C34901EB800074
:10585000A4309DF8A01001EBC10100EB01104271D2
:1058600037E09DF8B40040F2692110FB01F0BA491D
:1058700001EB8001A4319DF8A00000EBC00001EB1A
:10588000001001789DF8B40040F2692210FB02F08C
:10589000B14A02EB8000007981421AD1AF4801E0A1
:1058A000C5E1FDE390F80F0EC0F3401088B1162259
:1058B0009DF8B40040F2692110FB01F0A64901EB0C
:1058C0008000A4309DF8A01001EBC10100EB011095
:1058D0004271E5E314229DF8B40040F2692110FB07
:1058E00001F09D4901EB8001A4319DF8A00000EB7F
:1058F000C00001EB0010427101219DF8B40040F29C
:10590000692210FB02F0944A02EB8000C1709DF8FE
:10591000B40000EB400101EB0010A2F5986101EB2F
:10592000001130319DF8A00001EB0010801C0A909E
:10593000007820F0200020300A990870B0E314228B
:105940009DF8B40040F2692110FB01F0824901EB9F
:105950008001A4319DF8A00000EBC00001EB001015
:1059600042719DE39DF8B40040F2692110FB01F003
:10597000794901EB8000A430BDF8D81001EBC101DA
:1059800000EB01108079012827D100229DF8B40096
:1059900040F2692110FB01F06F4901E0FDE33AE0BC
:1059A00001EB8001A431BDF8D80000EBC00001EB91
:1059B0000010827114229DF8B40040F2692110FB9E
:1059C00001F0654901EB8000A4309DF8A01001EBC7
:1059D000C10100EB011042711CE000219DF8B400F0
:1059E00040F2692210FB02F05B4A02EB8000C170BA
:1059F00005229DF8B40040F2692110FB01F05649E0
:105A000001EB8000A4309DF8A01001EBC10100EB78
:105A10000110427144E301219DF8B40040F2692273
:105A200010FB02F04C4A02EB8000C17014229DF87A
:105A3000B40040F2692110FB01F0474901EB8001FD
:105A4000A4319DF8A00000EBC00001EB00104271F2
:105A50009DF8B40000EB400101EB0010404901EB60
:105A6000001130319DF8A00001EB0010801C0A905D
:105A7000007820F00400001D0A99087010E300204F
:105A80002E902F90002139911EE0DDE92E100002AA
:105A900040EA11620902CDE92E129DF8B40000EB34
:105AA0004001C1EBC0102F4901EBC001BDF8E4007B
:105AB000401D085CDDE92E341843CDE92E04BDF805
:105AC000E400401C80B23990BDF8E4000328DCDB20
:105AD000DDE92E010AF0A0FA01469DF8B40040F27B
:105AE000692210FB02F01C4A02EB8002A4329DF8EE
:105AF000A00000EBC00002EB0010C0F81E10002256
:105B00002E922F92002139911EE0DDE92E10000225
:105B100040EA11620902CDE92E129DF8B40000EBB3
:105B20004001C1EBC0100F4901EBC001BDF8E4001A
:105B30000830085CDDE92E341843CDE92E04BDF8A9
:105B4000E400401C80B23990BDF8E4000328DCDB9F
:105B5000DDE92E0108E00000D4450020BC22002031
:105B600014410020D87A00200AF056FA01469DF828
:105B7000B40040F2692210FB02F0FE4A02EB800200
:105B8000A4329DF8A00000EBC00002EB0010C0F8AA
:105B90001A1000222E922F92002139911EE0DDE989
:105BA0002E10000240EA11620902CDE92E129DF882
:105BB000B40000EB4001C1EBC010EF4901EBC001A4
:105BC000BDF8E4001330085CDDE92E341843CDE95C
:105BD0002E04BDF8E400401C80B23990BDF8E4000A
:105BE0000328DCDB9DF8B4002E9940F2692210FBFB
:105BF00002F0E04A02EB8002A4329DF8A00000EB24
:105C0000C00002EB0010416307229DF8B40040F28F
:105C1000692110FB01F0D74901EB8000A4309DF809
:105C2000A01001EBC10100EB01104271C9E300209B
:105C30002E902F90002139911FE0DDE92E100002F7
:105C400040EA11620902CDE92E129DF8B40000EB82
:105C50004001C1EBC010C84901EBC001BDF8E40030
:105C6000401D085CDDE92E3440EA0302CDE92E2414
:105C7000BDF8E400401C81B23991BDF8E40004286D
:105C8000DBDBDDE92E010AF0C7F99DF8B42040F214
:105C9000692312FB03F2B74B03EB8203A4339DF895
:105CA000A02002EBC20203EB021222329060D1600C
:105CB00000222E922F92002139911FE0DDE92E1053
:105CC000000240EA11620902CDE92E129DF8B400EB
:105CD00000EB4001C1EBC010A74901EBC001BDF8CA
:105CE000E4000930085CDDE92E3440EA0302CDE926
:105CF0002E24BDF8E400401C81B23991BDF8E400C7
:105D00000428DBDBDDE92E010AF086F99DF8B420DA
:105D100040F2692312FB03F2964B03EB8203A43398
:105D20009DF8A02002EBC20203EB021242F8220F00
:105D300051609DF8B40040F2692110FB01F08D49DB
:105D400001EB8000A4309DF8A01001EBC10100EB35
:105D5000011000789DF8B41040F2692211FB02F1A5
:105D6000844A02EB8101097988426ED1834890F818
:105D70000F0EC0F3401090B117229DF8B40040F20E
:105D8000692110FB01F07B4901EB8000A4309DF8F4
:105D9000A01001EBC10100EB0110427111E01422CF
:105DA0009DF8B40040F2692110FB01F0714901EB4C
:105DB0008001A4319DF8A00000EBC00001EB0010B1
:105DC00042716F4890F8A008F0BB00229DF8B40023
:105DD00040F2692110FB01F0664901EB8000A4301C
:105DE0009DF8A01001EBC10100EB011080F83E20EE
:105DF0006448D0F814020521B0FBF1F201FB120057
:105E000000EBC00101EB00115E48203000EB810087
:105E10000021C0F81D105B48D0F814020521B0FB2A
:105E2000F1F201FB120000EBC00101EB001155483B
:105E3000203000EB81000D300A909DF8B40040F254
:105E4000692110FB01F001E0D4E0B7E1494901EB21
:105E50008000A4309DF8A01001EBC10100EB0110FF
:105E600022301022014609900A98F2F7EEF94548CF
:105E7000D0F814020521B0FBF1F201FB120000EB97
:105E8000C00101EB00113F48203000EB81029DF87A
:105E9000B40040F2692110FB01F0364901EB8001AA
:105EA000A4319DF8A00000EBC00001EB001050F8F9
:105EB0001A1F42F8011F406850603248D0F814029F
:105EC0000521B0FBF1F201FB120000EBC00101EB78
:105ED00000132C4920319DF8B40000EB400202EB86
:105EE0000010294A02EB001230329DF8A00002EBAC
:105EF0000010007801F823002248D0F81402052190
:105F0000B0FBF1F201FB120000EBC00101EB00114C
:105F10001C48203000EB81029DF8B40040F269215A
:105F200010FB01F0134901EB8001A4319DF8A000A2
:105F300000EBC00001EB0010406BC2F809001148F3
:105F4000D0F814020521B0FBF1F201FB120000EBC6
:105F5000C00101EB00110B48203000EB8101084823
:105F6000826941F8212F808B88800648D0F814027E
:105F700005210BE0D4450020D87A0020BC22002067
:105F8000BC320020BC12002014410020B0FBF1F014
:105F900081B202200A91F3F79BF800210620F3F763
:105FA000D9FFF948D0F81402F749C98B884206D2C4
:105FB000F548D0F81402401CF349C1F8140200213E
:105FC0000520F3F7C7FF9DF8B40000EB400101EB9B
:105FD0000010EE4901EB001030309DF8A01000EBEE
:105FE0000110801C0A90007820F008020A980270C4
:105FF00029E0E7E19DF8B40000EB400101EB00105F
:10600000E24901EB001030309DF8A01000EB0110C8
:10601000801C0A90007820F0080008300A99087067
:1060200000229DF8B40040F2692110FB01F0D8492C
:1060300001EB8000A4309DF8A01001EBC10100EB42
:10604000011080F83E209DF8B4100220F3F782FF83
:106050009DF8B4109DF8A00000EB0110C217CDE927
:106060002E0200222E9800EBC00101EB0011C9485E
:1060700000EB8100C0F81D209DF8B40040F26921BA
:1060800010FB01F0C24901EB8000A4309DF8A01084
:1060900001EBC10100EB011022300A902E9800E0C4
:1060A0008FE100EBC00101EB0011BA4800EB810069
:1060B0000D30102209900A99F2F7C7F89DF8B41034
:1060C00040F2692011FB00F0B14901EB8001A431DD
:1060D0009DF8A00000EBC00001EB00112E9800EB32
:1060E000C00202EB0012AB4800EB820051F81A2FFD
:1060F00040F8012F496841609DF8B41001EB410060
:1061000000EB0110A14901EB001130319DF8A00016
:1061100001EB001001782E9800EBC00202EB001298
:106120009C4800F822102E9800EBC00101EB0011F2
:10613000984800EB81019848826941F8212F808BB3
:1061400088809DF8B41040F2692011FB00F090495E
:1061500001EB8001A4319DF8A00000EBC00001EB31
:106160000010416B2E9800EBC00202EB0012894830
:1061700000EB8200C0F809109DF8B41001EB41005B
:1061800000EB0110814901EB001130319DF8A000B6
:1061900001EB001041682E9800E091E000EBC00296
:1061A00002EB00127B4800EB8200C0F827102E980B
:1061B00081B208200A91F3F7CDFE80E09DF8B4107B
:1061C00040F2692011FB00F0714901EB8001A4311C
:1061D0009DF8A00000EBC00001EB001001789DF8D5
:1061E000B40040F2692210FB02F0694A02EB800021
:1061F0000079814263DA9DF8B41001EB410000EBB5
:106200000110624901EB001030309DF8A01000EB46
:106210000110801C0A90007820F00401091D0A98E2
:1062200001709DF8B41001EB410000EB01105749DB
:1062300001EB001130319DF8A00001EB0010801C33
:106240000A90007820F0800080300A9908700120C0
:106250009DF8B41040F2692211FB02F14C4A02EBA6
:106260008101C8709DF8B41040F2692011FB00F064
:10627000114601EB800002799DF8B40040F26921DB
:1062800010FB01F0424901EB8001A4319DF8A00010
:1062900000EBC00001EB0010027014229DF8B40066
:1062A00040F2692110FB01F0394901EB8000A43074
:1062B0009DF8A01001EBC10100EB0110427180E0DC
:1062C0000121354880F8C4179DF8B41040F26920C8
:1062D00011FB00F02E4901EB8001A4319DF8A000D4
:1062E00000EBC00001EB001001789DF8B40040F213
:1062F000692210FB02F0264A02EB800000798142FD
:106300002EDA00219DF8B40040F2692210FB02F061
:106310001F4A02EB8000C17001229DF8B40040F2D8
:10632000692110FB01F01A4901EB8001A4319DF8AD
:10633000A00000EBC00001EB0010027014229DF8D9
:10634000B40040F2692110FB01F0114901EB80001B
:10635000A4309DF8A01001EBC10100EB01104271C7
:106360002FE014229DF8B40040F2692110FB01F0E7
:10637000074901EB8000A4309DF8A01001EBC1019A
:1063800000EB011042711CE0BC12002014410020FF
:10639000D4450020E0140020BC32002014229DF8D7
:1063A000B40040F2692110FB01F0FE4901EB8000CE
:1063B000A4309DF8A01001EBC10100EB0110427167
:1063C00000BF00BFFEE39DF8B41040F2692011FB4E
:1063D00000F0F44901EB8000817828919DF8B41019
:1063E00001EB4100C0EBC110EF4911F830102991C9
:1063F0009DF8B41040F2692011FB00F0E94901EB6F
:106400008001A4319DF8A00000EBC00001EB00105A
:10641000417926919DF8B41001EB4100C0EBC11009
:10642000E14901EBC0010A91BDF8A4100A98F4F704
:1064300017FB37909DF8B41001EB4100C0EBC11081
:10644000D94901EBC001BDF8A400095CBDF8DC002E
:1064500081427DD19DF8B41001EB4100C0EBC11029
:10646000D14901EBC0004078002871DD0021CF4AFE
:106470009DF8B40002EB00129DF8A0001154BDF885
:106480009800892865D00CDC14287CD004DC08280E
:106490007AD0102879D1FDE3152877D08028F9D15A
:1064A000F9E38B2873D08C2872D08E2871D08F2876
:1064B000F0D1BDF8A4000D286CD19DF8B41001EB0B
:1064C0004100C0EBC110B84901EBC0004178B848A9
:1064D00080F8111E9DF8B41001EB4100C0EBC11013
:1064E000B14901EBC000C17AB14880F8121E9DF895
:1064F000B41040F2692011FB00F0AA4901EB8000C2
:10650000A4309DF8A01001EBC10100EB0110007850
:1065100003287DDCA64890F8120E002879DD9DF84E
:10652000B41040F2692011FB00F09E4901EB80019C
:10653000A4319DF8A00000EBC00001EB00110A910E
:106540000878401CC1B20A9801709DF8B41001E0AF
:10655000FEE3FEE340F2692011FB00F0914901EBFC
:106560008000A4309DF8A01001EBC10100EB0110E8
:10657000007804284DDB9DF8B41001EB410000EBDE
:1065800001108C4907E0FDE3FDE3FDE3FDE3FDE3DE
:10659000FDE3FDE3FDE301EB001030309DF8A010BA
:1065A00000EB0110801C0A90814890F8120EC0F395
:1065B0000010C0F101020A98007862F300000A9905
:1065C00008707B4890F8110EC0F3C000F0BB9DF836
:1065D000B41001EB410000EB0110764901EB001013
:1065E00030309DF8A01000EB01108078C0F340100F
:1065F00060B39DF8B41001EB410000EB01106D4950
:1066000001EB001030309DF8A01000EB011001E00C
:1066100057E0F1E0801C0A90007820F00200801C16
:106620000A9908709DF8B41040F2692011FB00F03F
:106630005C4901EB8000A4309DF8A01001EBC10182
:1066400000EB011018300A90007800E009E020F01B
:106650000200801C0A9908709DF8B4100220F3F71C
:1066600079FC00219DF8B40040F2692210FB02F091
:106670004C4A02EB8000C17004229DF8B40040F245
:10668000692110FB01F0474901EB8001A4319DF81D
:10669000A00000EBC00001EB001002708C229DF8FE
:1066A000B40040F2692110FB01F03E4901EB80008B
:1066B000A4309DF8A01001EBC10100EB0110427164
:1066C000B2E39DF8B41040F2692011FB00F03549A7
:1066D00001EB8001A4319DF8A00000EBC00001EBAC
:1066E000001001789DF8B40040F2692210FB02F01E
:1066F0002C4A02EB8000007981427DD19DF8B410D4
:1067000001EB410000EB01102A4901EB0010303091
:106710009DF8A01000EB0110801C0A90244890F80E
:10672000120EC0F30010C0F101000A990A7860F35C
:1067300000020A709DF8B41001EB410000EB01105B
:106740001C4901EB001030309DF8A01000EB011047
:10675000801C0A90164890F8110EC2080A9800781A
:1067600062F341000A9908709DF8B41001EB4100F2
:1067700000EB01100F4901EB001130319DF8A00032
:1067800001EB00108078C0F340029DF8B40040F2A5
:10679000692110FB01F0034901EB8000A4309DF852
:1067A000A01009E0D4450020D87A0020483F0020FE
:1067B000BC2200201441002001EBC10100EB0110BC
:1067C000007EC0F34000824264D09DF8B41040F2D5
:1067D000692011FB00F0FC4901EB8000A4309DF81A
:1067E000A01001EBC10100EB011018300A909DF8D8
:1067F000B41001EB410000E0D3E200EB0112F348DA
:1068000000EB021030309DF8A01000EB01108078F2
:1068100042080A98007862F341000A9908709DF8CE
:10682000B41001EB410000EB0110E84901EB00104E
:1068300030309DF8A01000EB01108078C0F34000CC
:1068400018BB01229DF8B40040F2692110FB01F051
:10685000DD4901EB8001A4319DF8A00000EBC000F0
:1068600001EB001042739DF8B40040F2692110FB67
:1068700001F0D54901EB8000A4309DF8A01001EB98
:10688000C10100EB011080F83E209DF8B4100220F9
:10689000F3F760FB9DF8B41001EB410000EB011031
:1068A000CA4901EB001130319DF8A00001EB001046
:1068B000807800F001029DF8B40040F2692110FBDD
:1068C00001F0C14901EB8000A4309DF8A01001EB5C
:1068D000C10100EB0110007E00F00100824276D081
:1068E0009DF8B41040F2692011FB00F0B64901EBAD
:1068F0008000A4309DF8A01001EBC10100EB011055
:1069000018300A909DF8B41001EB410000EB011023
:10691000AE4901EB001130319DF8A00001EB0010F1
:1069200082780A98017862F3000101709DF8B41032
:1069300001EB410000EB0110A44901EB00103030E5
:106940009DF8A01000EB0110807800F00100E8BB7A
:106950009DF8B41001EB410000EB01109B4901EBE5
:10696000001030309DF8A01000EB01108078C0F3CB
:10697000401068B39DF8B41040F2692011FB00F09C
:10698000914901EB8000A4309DF8A01001EBC101FA
:1069900000EB011090F83E00D0B99DF8B41040F221
:1069A000692011FB00F0884901EB8000A4309DF8BC
:1069B000A01001EBC10100EB0110407B40B99DF834
:1069C000B41001EB410000EB011002E045E06FE183
:1069D0002FE07E4901EB001030309DF8A01000EB55
:1069E00001108078C0F3400018BB01229DF8B4006C
:1069F00040F2692110FB01F0734901EB8001A431E1
:106A00009DF8A00000EBC00001EB001042739DF860
:106A1000B40040F2692110FB01F06B4901EB8000EA
:106A2000A4309DF8A01001EBC10100EB011080F82B
:106A30003E2000229DF8B40040F2692110FB01F0D5
:106A4000614901EB8000A4309DF8A01001EBC10169
:106A500000EB011080F83D2025E19DF8B41040F2D4
:106A6000692011FB00F0584901EB8000A4309DF82B
:106A7000A01001EBC10100EB011090F83E0098B9A5
:106A800001229DF8B40040F2692110FB01F04E494B
:106A900001EB8000A4309DF8A01001EBC10100EBD8
:106AA000011080F83D2027E000229DF8B40040F25C
:106AB000692110FB01F0444901EB8001A4319DF8EC
:106AC000A00000EBC00001EB001080F83D209DF815
:106AD000B41001EB410000EB01103C4901EB001147
:106AE00030319DF8A00001EB0010801C0A90007866
:106AF00020F001020A980270354890F8A00880B191
:106B00009DF8B41001EB410000EB01102F4901EB9F
:106B1000001030309DF8A01000EB0110807A0228A0
:106B200051D12C48407F01284DD12A48D0F8140279
:106B30002849C98B884246D29DF8B41040F269209A
:106B400011FB00F0204901EB8000A4309DF8A0105B
:106B500001EBC10100EB011090F83D00012832D19A
:106B60009DF8B41040F2692011FB00F0164901EBCA
:106B70008000A4309DF8A01001EBC10100EB0110D2
:106B800090F87D00F8B99DF8B41001EB410000EBDE
:106B900001100E4901EB001130319DF8A00001EB0E
:106BA000001001789DF8B40040F2692210FB02F059
:106BB000054A02EB8000417008229DF8B40040F2C3
:106BC000692109E0FEE36EE0D44500201441002075
:106BD000BC320020BC12002010FB01F0FE4901EB8A
:106BE0008001A4319DF8A00000EBC00001EB001073
:106BF000427100229DF8B40000EB400101EB00104F
:106C0000F64901EB001130319DF8A00001EB0010B6
:106C100042609DF8B4100220F3F79CF900213991ED
:106C200019E000229DF8B40040F2692110FB01F048
:106C3000E94901EB8001A4319DF8A00000EBC00000
:106C400001EB00113F31BDF8E4000A54BDF8E40047
:106C5000401C81B23991BDF8E4001428E1DB002129
:106C600039911CE000229DF8B40040F2692110FB2C
:106C700001F0D94901EB8001A4319DF8A00000EB9F
:106C8000C00001EB00115B31BDF8E4000A54BDF80F
:106C9000E40001E0FFE1C7E3401C81B23991BDF897
:106CA000E4000A28DEDB9DF8B4100220F3F752F965
:106CB0009DF8B41040F2692011FB00F0C64901EBC9
:106CC0008000A4309DF8A01001EBC10100EB011081
:106CD0008078802835D19DF8B41001EB410000EB9D
:106CE0000110BE4901EB001030309DF8A01000EB00
:106CF00001108078C0F3400018BB9DF8B41001EB80
:106D0000410000EB0110B54901EB001030309DF857
:106D1000A01000EB01108078C0F3401088B9152254
:106D20009DF8B40040F2692110FB01F0AA4901EB83
:106D30008000A4309DF8A01001EBC10100EB011010
:106D400042719DF8B41001EB410000EB011001E02D
:106D5000EDE3B7E1A14901EB001030309DF8A01040
:106D600000EB01108078C0F34000D8B18F229DF86D
:106D7000B40040F2692110FB01F0974901EB80005B
:106D8000A43007E0FDE364E14FE2FBE3F4E14DE210
:106D90007EE35DE19DF8A01001EBC10100EB011065
:106DA000427141E09DF8B41040F2692011FB00F0FF
:106DB000894901EB8000A4309DF8A01001EBC101CE
:106DC00000EB0110807B01282ED100229DF8B40039
:106DD00040F2692110FB01F07F4901EB8001A431F1
:106DE0009DF8A00000EBC00001EB001082738C2224
:106DF0009DF8B40040F2692110FB01F0764901EBE7
:106E00008001A4319DF8A00000EBC00001EB001050
:106E1000427100219DF8B40040F2692210FB02F09B
:106E20006D4A02EB8000C1709DF8B41001EB410087
:106E300000EB0110694901EB0010007BF0BB9DF8ED
:106E4000B41001EB4100C0EBC110654901EBC0007B
:106E5000807800049DF8B41001EB4102C2EBC1112F
:106E60005F4A02EBC101C97840EA01209DF8B410E5
:106E700001EB4102C2EBC111594A02EBC101097990
:106E80000843C117CDE9080109F0C6F801469DF88D
:106E9000B40040F2692210FB02F04F4A02EB80027C
:106EA000A4329DF8A00000EBC00002EB0010C0F877
:106EB0001E109DF8B41001EB410000E035E0C0EB7E
:106EC000C110474901EBC000407901049DF8B400AE
:106ED00000EB4002C2EBC010414A02EBC0008079D7
:106EE00041EA00209DF8B41001EB4102C2EBC11150
:106EF0003B4A02EBC101C9790843C117CDE908013A
:106F000009F08AF89DF8B41040F2692211FB02F1F1
:106F1000314A02EB8101A4319DF8A02002EBC202AC
:106F200001EB0211C1F81A0092E09DF8B41001EBD8
:106F30004100C0EBC1102A4901EBC0008078010676
:106F40009DF8B40000EB4002C2EBC010244A02EBF3
:106F5000C000C07841EA00419DF8B40000EB400257
:106F6000C2EBC0101E4A02EBC000007941EA0021CA
:106F70009DF8B40000EB4002C2EBC010184A02EBCF
:106F8000C00040790843C117CDE9080109F044F871
:106F900001469DF8B40040F2692210FB02F00E4A4F
:106FA00002EB8002A4329DF8A00000EBC00002EBCF
:106FB0000010C0F81E109DF8B41001EB4100C0EBAA
:106FC000C110074901EBC000807901069DF8B400AB
:106FD00000EB400206E00000D445002014410020F0
:106FE000D87A0020C2EBC010FE4A02EBC000C07984
:106FF00041EA00419DF8B40000EB4002C2EBC01032
:10700000F84A02EBC000007A41EA00209DF8B41073
:1070100001EB4102C2EBC111F24A02EBC101497A14
:107020000843C117CDE9080108F0F6FF9DF8B41038
:1070300040F2692211FB02F1EB4A02EB8101A4311B
:107040009DF8A02002EBC20201EB0211C1F81A0068
:10705000EBE0BDF8A40003281CD18F229DF8B400FA
:1070600040F2692110FB01F0DF4901EB8001A431FE
:107070009DF8A00000EBC00001EB0010427101215F
:107080009DF8B40040F2692210FB02F0D64A02EBF0
:107090008000C170C9E0BDF8A400032811D18F227F
:1070A0009DF8B40040F2692110FB01F0CE4901EBDC
:1070B0008000A4309DF8A01001EBC10100EB01108D
:1070C0004271B2E0BDF8A400032854D19DF8B41079
:1070D00040F2692011FB00F0C34901EB8000A430AD
:1070E000BDF8D81001EBC10100EB01108079012837
:1070F00024D100229DF8B40040F2692110FB01F078
:10710000B94901EB8001A431BDF8D80000EBC00003
:1071100001EB001082718F229DF8B40040F26921CA
:1071200010FB01F0B04901EB8000A4309DF8A010E5
:1071300001EBC10100EB011042711CE008229DF837
:10714000B40040F2692110FB01F0A74901EB800176
:10715000A4319DF8A00000EBC00001EB00104271CB
:1071600000219DF8B40040F2692210FB02F09E4A13
:1071700002EB8000C17058E0BDF8A400032854D190
:107180009DF8B41040F2692011FB00F0964901EB24
:107190008000A430BDF8D81001EBC10100EB011054
:1071A0008079012824D100229DF8B40040F26921A1
:1071B00010FB01F08C4901EB8001A431BDF8D8002F
:1071C00000EBC00001EB001082718F229DF8B4002B
:1071D00040F2692110FB01F0834901EB8001A431E9
:1071E0009DF8A00000EBC00001EB001042711CE014
:1071F00008229DF8B40040F2692110FB01F07A49A1
:1072000001EB8001A4319DF8A00000EBC00001EB70
:107210000010427100219DF8B40040F2692210FB79
:1072200002F0714A02EB8000C170FDE3BDF8A400DA
:1072300008287DD19DF8B41001EB4100C0EBC110CE
:10724000684901EBC000807801069DF8B40000EBAE
:107250004002C2EBC010634A02EBC000C07841EAB2
:1072600000419DF8B40000EB4002C2EBC0105D4A43
:1072700002EBC000007941EA00219DF8B40000EB68
:107280004002C2EBC010574A02EBC00040790843ED
:10729000C117CDE9080108F0BFFE9DF8B41040F217
:1072A000692211FB02F1504A02EB8102A4329DF8DF
:1072B000A01001EBC10102EB011148639DF8B4106D
:1072C00040F2692011FB00F0474901EB8000A43037
:1072D0009DF8A01001EBC10100EB011000789DF8B2
:1072E000B41040F2692211FB02F13F4A02EB810126
:1072F0000979884231DA00219DF8B40040F2692210
:1073000010FB02F0384A02EB8000C17005229DF8A4
:10731000B40040F2692110FB01F0334901EB800118
:10732000A4319DF8A00000EBC00001EB001000E0CC
:1073300079E002708E229DF8B40040F2692110FBC2
:1073400001F0294901EB8000A4309DF8A01001EB69
:10735000C10100EB0110427165E09DF8B41040F2EC
:10736000692011FB00F0204901EB8000A430BDF83A
:10737000D81001EBC10100EB01108079012835D153
:1073800000229DF8B40040F2692110FB01F016497B
:1073900001EB8001A431BDF8D80000EBC00001EB87
:1073A000001082718F229DF8B40040F2692110FB19
:1073B00001F00D4901EB8001A4319DF8A00000EB24
:1073C000C00000E0FDE301EB0010427101219DF8D7
:1073D000B40040F2692210FB02F0034A02EB800085
:1073E000C17020E0D87A0020D44500208E229DF87C
:1073F000B40040F2692110FB01F0FE4901EB80016D
:10740000A4319DF8A00000EBC00001EB0010427118
:1074100000219DF8B40040F2692210FB02F0F54A09
:1074200002EB8000C170FFE2BDF8A40003282ED15A
:1074300000219DF8B40040F2692210FB02F0ED4AF1
:1074400002EB8000C17001229DF8B40040F2692176
:1074500010FB01F0E74901EB8001A431BDF8D80031
:1074600000EBC00001EB001082718C229DF8B4008B
:1074700040F2692110FB01F0DE4901EB8001A431EB
:107480009DF8A00000EBC00001EB00104271CBE2C0
:10749000BDF8A4000F2876D19DF8B41001EB41008F
:1074A00000EB0110D44901EB0010007BF0BB002081
:1074B0002E902F90002139911FE0DDE92E1000025F
:1074C00040EA11620902CDE92E129DF8B41001EBD9
:1074D0004100C0EBC110C94901EBC001BDF8E40097
:1074E000C0F10600085CDDE92E341843CDE92E0416
:1074F000BDF8E400401C80B23990BDF8E4000528D6
:10750000DBDB9DF8B400DDE92E1240F2692310FBAD
:1075100003F0B84B03EB8003A4339DF8A00000EB0D
:10752000C00003EB001040F8221F01E046E0FDE33D
:10753000426000222E922F920021399120E0DDE955
:107540002E10000240EA11620902CDE92E129DF8C8
:10755000B40000EB4001C1EBC010A84901EBC00131
:10756000BDF8E400C0F10B00085CDDE92E3440EA10
:107570000302CDE92E24BDF8E400401C81B239910C
:1075800002E0E7E340E33EE3BDF8E4000528D6DB94
:107590009DF8B400DDE92E2140F2692310FB03F0D1
:1075A000944B03EB8000A4309DF8A03003EBC303A1
:1075B00000EB031022308260C1607EE000202E903C
:1075C0002F90002139911FE0DDE92E10000240EAE2
:1075D00011620902CDE92E129DF8B41001EB4100B1
:1075E000C0EBC110854901EBC001BDF8E400C0F15A
:1075F0000700085CDDE92E341843CDE92E04BDF800
:10760000E400401C80B23990BDF8E4000628DBDBC2
:107610009DF8B400DDE92E1240F2692310FB03F05F
:10762000744B03EB8003A4339DF8A00000EBC00073
:1076300003EB001040F8221F426000222E922F928E
:107640000021399120E0DDE92E10000240EA1162AC
:107650000902CDE92E129DF8B41001EB4100C0EBF8
:10766000C110664901EBC000BDF8E410C1F10D0185
:10767000405CDDE92E3440EA0302CDE92E24BDF85A
:10768000E400401C81B23991BDF8E4000628DADB41
:107690009DF8B400DDE92E1240F2692310FB03F0DF
:1076A000544B03EB8000A4309DF8A03003EBC303E0
:1076B00000EB031022308160C2609DF8B41040F2EC
:1076C000692011FB00F04B4901EB8001A4319DF8CA
:1076D000A00000EBC00001EB001001789DF8B400A1
:1076E00040F2692210FB02F0424A02EB800000796E
:1076F00081427DD1424890F8A008E8BB4148D0F8CB
:1077000014020521B0FBF1F201FB120101EBC100F3
:1077100000EB01113B48203000EB81000021C0F854
:107720001D103848D0F814020521B0FBF1F201FB1E
:10773000120101EBC10000EB01113248203000EBD7
:1077400081000D300A909DF8B41040F2692011FBC1
:1077500000F0284901EB8001A4319DF8A00000EB66
:10776000C00001EB001022301022014609900A9857
:10777000F0F76BFD234800E0E7E0D0F814020521A4
:10778000B0FBF1F201FB120101EBC10000EB0111B2
:107790001C48203000EB81029DF8B40040F26921C2
:1077A00010FB01F0134901EB8001A4319DF8A0000A
:1077B00000EBC00001EB001050F81A1F42F8011F47
:1077C000406850600F48D0F814020521B0FBF1F278
:1077D00001FB120101EBC10000EB0113094920314B
:1077E0009DF8B40000EB400202EB0010024A0BE0EF
:1077F000A3E10000D445002014410020D87A0020E5
:10780000BC320020BC12002002EB001230329DF886
:10781000A00002EB0010007801F82300A1F1200085
:10782000D0F814020521B0FBF1F201FB120101EBCB
:10783000C10000EB0111FE4800EB810100F5FF5093
:10784000826941F8212F808B8880F9482038D0F850
:1078500014020521B0FBF1F201FB120101EBC100A2
:1078600000EB0111F24800EB81029DF8B40040F2F8
:10787000692110FB01F0EF4901EB8001A4319DF873
:10788000A00000EBC00001EB0010406BC2F8090043
:10789000E7482038D0F814020521B0FBF1F201FBD3
:1078A000120101EBC10000EB0111E14800EB810284
:1078B0009DF8B40000EB400101EB0010DE4901EB44
:1078C000001130319DF8A00001EB00104068C2F8B3
:1078D0002700D7482038D0F814020521B0FBF1F07A
:1078E00081B202200A91F1F7F3FB00210620F2F7A2
:1078F00031FBCF482038D0F81402CD492039C98B4C
:10790000884208D2CA482038D0F81402401CC8491E
:107910002039C1F8140200210520F2F71BFB9DF865
:10792000B41001EB410000EB0110C34901EB001062
:1079300030309DF8A01000EB0110801C0A900078F8
:1079400020F008020A98027015E09DF8B41001EBCF
:10795000410000EB0110B84901EB001030309DF8F8
:10796000A01000EB0110801C0A90007820F00800A5
:1079700008300A9908709DF8B41001EB410000EB43
:107980000110AD4901EB001030309DF8A01000EB64
:107990000110801C0A90007820F020020A980270E2
:1079A0009DF8B4100220F2F7D5FA9DF8B4009DF8C6
:1079B000A01001EB0010C217CDE92E0200222E9874
:1079C00000EBC00101EB00119C4800EB8100C0F806
:1079D0001D209DF8B41040F2692011FB00F095497C
:1079E00001EB8000A4309DF8A01001EBC10100EB79
:1079F000011022300A902E9800EBC00101EB00111B
:107A00008E4800EB81010D3110220991DDE9090159
:107A1000F0F71BFC9DF8B41040F2692011FB00F058
:107A2000844901EB800100E0AFE1A4319DF8A000A2
:107A300000EBC00001EB00112E9800EBC00202EB3E
:107A400000127E4800EB820051F81A2F40F8012FF7
:107A5000496841609DF8B41001EB410000EB011052
:107A6000754901EB001130319DF8A00001EB0010C9
:107A700001782E9800EBC00202EB00126F4800F86C
:107A800022102E9800EBC00101EB00116B4800EBB7
:107A900081016B48826941F8212F808B88809DF895
:107AA000B41040F2692011FB00F0624901EB800143
:107AB000A4319DF8A00000EBC00001EB0010416B69
:107AC0002E9800EBC00202EB00125C4800EB820033
:107AD000C0F809109DF8B41001EB410000EB011053
:107AE000554901EB001130319DF8A00001EB001069
:107AF00041682E9800EBC00202EB00124F4800EBE9
:107B00008200C0F827102E9881B208200A91F2F75F
:107B100021FA00229DF8B40040F2692110FB01F027
:107B2000444901EB8000A4309DF8A01001EBC10195
:107B300000EB011080F83E2053E09DF8B41001EBFB
:107B4000410000EB01103C4901EB001030309DF882
:107B5000A01000EB0110801C0A90007820F00400B7
:107B6000001D0A9908709DF8B41001EB410000EB6C
:107B70000110314901EB001030309DF8A01000EBEE
:107B80000110801C0A90007820F0800180310A9852
:107B9000017001219DF8B40040F2692210FB02F04F
:107BA000244A02EB8000C1709DF8B41040F26920B5
:107BB00011FB00F0114601EB800002799DF8B40042
:107BC00000E0E4E040F2692110FB01F0194901EB0B
:107BD0008000A4309DF8A01001EBC10100EB011062
:107BE00002708F229DF8B40040F2692110FB01F071
:107BF000104901EB8000A4309DF8A01001EBC101F9
:107C000000EB01104271C0E0BDF8A40003285BD175
:107C100001210B4880F8C4179DF8B41040F2692088
:107C200011FB00F0034901EB8001A4310AE00000E0
:107C3000DC120020D445002014410020E014002074
:107C4000BC3200209DF8A00000EBC00001EB00104A
:107C500001789DF8B40040F2692210FB02F0FE4A60
:107C600002EB8000007981422FDA00219DF8B400F8
:107C700040F2692210FB02F0F74A02EB8000C1706B
:107C800001229DF8B40040F2692110FB01F0F24995
:107C900001EB8001A4319DF8A00000EBC00001EBD6
:107CA000001002708F229DF8B40040F2692110FB91
:107CB00001F0E94901EB8000A4309DF8A01001EB30
:107CC000C10100EB0110427143E09DF8B41040F295
:107CD000692011FB00F0E04901EB8000A4309DF821
:107CE000A01001EBC10100EB01108078802830D199
:107CF00000219DF8B40040F2692210FB02F0D64A40
:107D000002EB8000C17080229DF8B40040F269212E
:107D100010FB01F0D04901EB8001A4319DF8A000D7
:107D200000EBC00001EB0010427100E02EE00022E9
:107D30009DF8B40040F2692110FB01F0C64901EB47
:107D40008000A4309DF8A01001EBC10100EB0110F0
:107D500082701AE0BDF8A400032815D10021BF48A5
:107D600080F8C4178F229DF8B40040F2692110FBFF
:107D700001F0B94901EB8000A4309DF8A01001EB9F
:107D8000C10100EB0110427100BF00BF00BF00BF86
:107D9000B248C07DB0B1B2499DF8B40031F81010BE
:107DA0000A919DF8B41001EB4100C0EBC110AD4940
:107DB00001EBC001012309919DF8B420DDE909011F
:107DC000F2F766FE0021399111E000219DF8B40020
:107DD00000EB4002C2EBC010A24A02EBC002BDF8A9
:107DE000E4001154BDF8E400401C81B23991BDF8A3
:107DF000E400142843DAE8E79B499DF8B40011F841
:107E00001000C009D8BB9DF8B40011F81000C0F3F1
:107E1000C300062832D2DFE800F0036291FEFD3392
:107E20009DF8B41001EB4100C0EBC1108D4901EB8E
:107E3000C0010A918DA10A981AF054F81290129874
:107E4000E0B100219DF8B40000EB4000864A3C32CE
:107E500002EB8000416001219DF8B40000EB40007E
:107E600002EB8000817080499DF8B40001EB400175
:107E70000A91087820F078002830087060E160E10D
:107E80009DF8B41001EB4100C0EBC110754901EB46
:107E9000C0010A9175A10A981AF024F8129012985C
:107EA000E0B100219DF8B40000EB40006E4A3C3286
:107EB00002EB8000416001219DF8B40000EB40001E
:107EC00002EB8000817068499DF8B40001EB40012D
:107ED0000A91087820F078002030087030E19DF891
:107EE000B41001EB4100C0EBC1105E4901EBC001D1
:107EF0000A915EA10A9819F0F5FF12901298E0B16C
:107F000000219DF8B40000EB4000574A3C3202EBE0
:107F10008000416001219DF8B40000EB400002EBBD
:107F20008000817050499DF8B40001EB40010A9136
:107F3000087820F078001830087001E100219DF8E1
:107F4000B40000EB4000484A3C3202EB8000416044
:107F500001219DF8B40000EB400002EB800081702D
:107F60009DF8B41001EB4100C0EBC1103D4901EB9D
:107F7000C0011298801D095C30399DF8B40000EBF7
:107F80004002C2EBC010374A02EBC0031298401DFA
:107F9000185C303841EA0010C117CDE9080107F03C
:107FA0007BFA334988719DF8B41001EB4100C0EBB6
:107FB000C1102C4901EBC0010A912EA10A9819F0B9
:107FC00091FF1290129838B39DF8B41001EB410064
:107FD000C0EBC111234800EBC1011298401C085CA2
:107FE000302826DB9DF8B41001EB4100C0EBC11036
:107FF0001C4901EBC0011298401C095C30399DF806
:10800000B40000EB4002C2EBC010164A02EBC00203
:10801000129802E06AE03CE02FE0105C303841EA60
:108020000010C117CDE9080107F036FA1049C871F0
:1080300023E09DF8B41001EB4100C0EBC1100949E9
:1080400001EBC0011298085C3038C117CDE9080176
:1080500007F022FA06490FE0D4450020BC32002088
:10806000646C0020D87A0020DC3E00204F4B0000DA
:108070005C3B00202C000000C8713A499DF8B40018
:1080800001EB40010A91087820F078001830087060
:1080900056E09DF8B41001EB4100C0EBC11032492D
:1080A00001EBC0010A91AFF23C010A9819F01AFFE6
:1080B00012901298C8B100202C49086029499DF8F7
:1080C000B40001EB40010A91087820F08001803172
:1080D0000A9801704FF47A719DF8B40000EB4000EB
:1080E000204A3C3202EB8000816029E09DF8B41008
:1080F00001EB4100C0EBC1101B4901EBC0010A912B
:10810000AFF298010A9819F0EDFE12901298B0B1F2
:10811000174890F8C60720F08001154880F8C61768
:1081200010499DF8B40001EB40010A91087820F055
:1081300078000830087000200E498870486000BF41
:1081400000BF0D4800780D49097808440C490978AA
:1081500008440C4909780844002872F4ADAE3AB0DE
:1081600070BD0000DC3E0020D87A00208802424228
:10817000BC320020A46C002012000020130000205C
:10818000140000201500002007B5D2B000211A917C
:10819000199118911791169115911491002212922C
:1081A0001392109211920F910E910D910C910B91CF
:1081B0000A91F9A006C8CDE90812F9A006C8CDE9D0
:1081C0000612002105910020F7490870529800EB33
:1081D000400101EB0010F54901EB00108179169187
:1081E000F349529801EB00115398085C05287DDD96
:1081F0000621EF4A529802EB0012539811540022C4
:1082000040F2692152984843EA4901EB8001A431C8
:10821000539800EBC00001EB00100270529800EB85
:10822000400101EB0010E14901EB0011303153989E
:1082300001EB0010807820F08002529800EB4001A2
:1082400001EB0010D94901EB00113031539801EBDB
:108250000010827040F2692152984843D54901EBE1
:108260008001A431539800EBC00001EB001090F89E
:108270008E0020F0080240F2692152984843CD490F
:1082800001EB8001A431539800EBC00001EB00101A
:1082900080F88E2040F2692152984843C54901EB8D
:1082A0008001A431539800EBC00001EB001090F85E
:1082B0008E0020F0010240F2692152984843BD49E6
:1082C00001EB8001A431539800EBC00001EB0010DA
:1082D00080F88E20529800EB400101EB0010B3496A
:1082E00001EB00108079092817D200E087E0DFE871
:1082F00000F085051525354555657500E52240F2E8
:10830000692152984843AB4901EB8000A43053994E
:1083100001EBC10100EB011042716FE0A12240F2BC
:10832000692152984843A34901EB8000A430539936
:1083300001EBC10100EB011042715FE0A12240F2AC
:108340006921529848439B4901EB8000A43053991E
:1083500001EBC10100EB011042714FE0B12240F28C
:10836000692152984843934901EB8000A430539906
:1083700001EBC10100EB011042713FE0312240F2FC
:108380006921529848438B4901EB8000A4305399EE
:1083900001EBC10100EB011042712FE0F42240F229
:1083A000692152984843834901EB8000A4305399D6
:1083B00001EBC10100EB011042711FE0062240F207
:1083C0006921529848437B4901EB8000A4305399BE
:1083D00001EBC10100EB011042710FE0152240F2E8
:1083E000692152984843734901EB8000A4305399A6
:1083F00001EBC10100EB0110427100BF00BF6C49ED
:108400006C39529811F810000121B1EBD01F46F0E1
:108410006486529800EB400101EB0010634901EBC8
:108420000010407B02287DD10DE013F019FE624957
:1084300048620846406AC0F300410E915E48406AB7
:10844000C0F342010D910D980028EED000201A9043
:1084500011E05749529801EB0011BDF86800014442
:1084600004910878401CC1B204980170BDF86800FE
:10847000401C81B21A91BDF868001028E9DB552133
:108480005298C0EB001000EB80004C4A02F830100C
:10849000FD215298C0EB001000EB800002EBC00001
:1084A0004170AA215298C0EB001000EB800002EB53
:1084B000C000817000215298C0EB001000EB8000DA
:1084C00002EBC000C1705298C0EB001000EB8000BE
:1084D00002EBC000017161215298C0EB001000EB6B
:1084E000800002EBC000417100215298C0EB0010E7
:1084F00000EB800002EBC0008171FA215298C0EBC2
:10850000001000EB800002EBC000C1712A48183057
:1085100041795298C0EB001000EB800002EBC000E4
:10852000017200E0FEE32448183001795298C0EB54
:10853000001000EB800002EBC00041721E481830B2
:10854000C1785298C0EB001000EB800002EBC00035
:1085500081721948183081785298C0EB001000EBF6
:10856000800002EBC000C172134818304178529865
:10857000C0EB001000EB800002EBC00001730E485E
:10858000017E5298C0EB001000EB800002EBC000AF
:10859000417300211A912DE00169323031303000F1
:1085A00001693230453030001600002014410020AF
:1085B000483F0020D4450020BC32002078710020C4
:1085C000FE48406ABDF86810C1F10301C900C84007
:1085D000C1B25298C0EB001000EB8000F84A02EBE9
:1085E000C002BDF8680010301154BDF86800401C8E
:1085F00081B21A91BDF868000428E1DB5298C0EB03
:10860000001000EB8000EE4A02EBC00054990175A7
:1086100015210F91002140F2692252985043E94AF6
:1086200002EB80004171549808B95120549054983D
:10863000002806F01487549815287BD00FDCA0F191
:108640000B000A2877D2DFE810F0F6044305790022
:10865000440576007600620139017600D805A1282C
:108660006AD006DC502868D0512807D0522862D141
:10867000FEE3A2287ED0A428F9D147E1CF4890F8A4
:10868000A008012825D100201A9015E0BDF8680047
:108690000E30CD49095C5298C0EB001000EB800011
:1086A000C74A02EBC002BDF8680015301154BDF88E
:1086B0006800401C81B21A91C448C0880838BDF8CF
:1086C00068108842E2DCC148C088C01D80B20F90AB
:1086D0002FE05298C0EB001000EB8000B84A02EB8C
:1086E000C0005499017500211A9115E0002152989B
:1086F000C0EB001000EB8000B14A02EBC002BDF8F5
:108700003C001154BDF83C00401C81B20F91BDF8F3
:108710006800401C81B21A91529800EB400101EBB5
:108720000010AB4901EB0010C179BDF8680081422F
:10873000DCDCFDE3FDE3FDE3E6E00EE1A548408877
:1087400001125298C0EB001000EB80009C4A02EB33
:10875000C002BDF83C001154BDF83C00401C81B281
:108760000F919C484088C1B25298C0EB001000EBBA
:10877000800000E0C9E0924A02EBC002BDF83C0074
:108780001154BDF83C00401C81B20F9140F26921A8
:10879000529848438B4901EB8001083140F269222D
:1087A00052985043874A02EB800090F8A00000EBFB
:1087B000400202EB001001EB4000408C0112529885
:1087C000C0EB001000EB80007D4A02EBC002BDF858
:1087D0003C001154BDF83C00401C81B20F9140F2A6
:1087E000692152984843774901EB8001083140F2F2
:1087F000692252985043734A02EB800090F8A0001F
:1088000000EB400202EB001001EB4000408CC1B2D3
:108810005298C0EB001000EB8000694A02EBC002E6
:10882000BDF83C001154BDF83C00401C81B20F91D2
:1088300040F2692152984843624901EB80010831B6
:1088400040F26922529850435E4A02EB800090F851
:10885000A00000EB400202EB001001EB4000408C56
:1088600000F5806081B201200491F0F795FB0021B2
:108870001A9117E057490E31BDF86800095C52980B
:10888000C0EB001000EB80004D4A02EBC002BDF8C7
:108890003C30BDF8680018441154BDF86800401C15
:1088A00081B21A91BDF86800B0F5007FE2DBBDF837
:1088B0003C0000F5007081B20F913AE700201A9059
:1088C00015E0BDF868000E303F49095C5298C0EBD6
:1088D000001000EB80003A4A02EBC002BDF86800CD
:1088E00015301154BDF86800401C81B21A91374808
:1088F000C0880838BDF868108842E2DC3348C08878
:10890000C01D80B20F9013E300BF00BF00BF002066
:108910001A9015E0BDF868000E302B49095C52989A
:10892000C0EB001000EB8000254A02EBC002BDF84E
:10893000680015301154BDF86800401C81B21A91CE
:108940002248C0880838BDF868108842E2DC1F4819
:10895000C088C01D80B20F90EAE2002140F2692277
:1089600052985043174A02EB8000817157E340F25E
:10897000692152984843134901EB8000817952984C
:10898000C0EB001000EB80000D4A02EBC002BDF806
:108990003C001154BDF83C00401C81B20F9140F2E4
:1089A000692152984843074901EB8000807900EB28
:1089B000400101EB001006490EE00000BC3200202F
:1089C00078710020D4450020A0920020BC12002025
:1089D00014410020C430002001EB0010016808465B
:1089E0000491002107F018FBCDE9120100211A9132
:1089F0001EE0BDF86800C0F10200C200DDE912010E
:108A0000CDE91B10EFF70FFCC2B25298C0EB00107B
:108A100000EB8000FE4901EBC000BDF83C30BDF822
:108A2000681019444254BDF86800401C80B21A9086
:108A3000BDF868000328DCDBBDF83C00C01C81B237
:108A40000F9140F2692152984843F24901EB8000AE
:108A5000807900EB400101EB0010EF4901EB0010C1
:108A6000017908460491002107F0D6FAC1B2529864
:108A7000C0EB001000EB8000E54A02EBC002BDF83D
:108A80003C001154BDF83C00401C81B20F9140F2F3
:108A9000692152984843DF4901EB8000807900EB5F
:108AA000400101EB0010DC4901EB00104179084660
:108AB0000491002107F0B0FAC1B25298C0EB001047
:108AC00000EB8000D24A02EBC002BDF83C0011541A
:108AD000BDF83C00401C81B20F9140F269215298D0
:108AE0004843CC4901EB8000807900EB400101EB69
:108AF0000010C94901EB001081790846049100215A
:108B000007F08AFAC1B25298C0EB001000EB800067
:108B1000BF4A02EBC002BDF83C001154BDF83C0056
:108B2000401C81B20F9140F2692152984843B949E3
:108B300001EB8000807900EB400101EB0010B649A9
:108B400001EB0010C17908460491002107F064FA96
:108B5000C1B25298C0EB001000EB8000AC4A02EBAF
:108B6000C002BDF83C001154BDF83C00401C81B26D
:108B70000F9140F2692152984843A64901EB8000C9
:108B8000807900EB400101EB0010A34901EB0010DC
:108B9000816808460491002107F03EFAC1B252985C
:108BA000C0EB001000EB8000994A02EBC002BDF858
:108BB0003C001154BDF83C00401C81B20F9140F2C2
:108BC000692152984843934901EB8000807900EB7A
:108BD000400101EB0010904901EB0010017B0846B9
:108BE0000491002107F018FAC1B25298C0EB0010AE
:108BF00000EB8000864A02EBC002BDF83C00115435
:108C0000BDF83C00401C81B20F9140F2692152989E
:108C10004843804901EB8000807900EB400101EB83
:108C200000107D4901EB0010807906287BD10020DF
:108C30001A908AE040F2692152984843754901EB45
:108C40008000807900EB400101EB0010724901EBDC
:108C500000113031BDF8680001EB001001780846C2
:108C60000491002107F0D8F9C1B25298C0EB00106E
:108C700000EB8000664A02EBC002BDF8680000EB22
:108C80004003BDF83C001844115440F26921529849
:108C90004843604901EB8000807900EB400101EB23
:108CA00000105D4901EB00113031BDF8680001EBA7
:108CB0000010417808460491002107F0ADF9C1B2D7
:108CC0005298C0EB001000EB8000514A02EBC0024A
:108CD000BDF8680000EB4003BDF83C001844401CA0
:108CE000115440F26921529848434A4901EB8000EF
:108CF000807900EB400101EB0010474901EB0011C6
:108D00003031BDF8680001EB0010017A084604918B
:108D1000002107F081F9C1B25298C0EB001000EBBE
:108D2000800001E0CCE336E0394A02EBC002BDF836
:108D3000680000EB4003BDF83C001844801C11544F
:108D4000BDF86800401C81B21A91529800EB4001B6
:108D500001EB0010304901EB0010C179BDF868004B
:108D600081423FF767AF40F2692152984843294951
:108D700001EB8000807900EB400101EB00102649F7
:108D800001EB0010C07900EB4001BDF83C00084445
:108D900081B20F9131E100201A9060E040F2692128
:108DA000529848431B4901EB8000807900EB400159
:108DB00001EB0010184901EB00113031BDF86800DB
:108DC00001EB0010017808460491002107F024F916
:108DD000C2B25298C0EB001000EB80000C4901EBCE
:108DE000C003BDF86810BDF83C0000EB41001A5408
:108DF00040F2692152984843064901EB800080798E
:108E000000EB400101EB0010034901EB001105E00C
:108E100078710020D4450020144100203031BDF885
:108E2000680001EB0010417808460491002107F02A
:108E3000F3F8C2B25298C0EB001000EB8000FE497C
:108E400001EBC003BDF86810BDF83C0000EB410029
:108E5000401C1A54BDF86800401C81B21A91529807
:108E600000EB400101EB0010F44901EB001000E0C1
:108E700030E1C179BDF8680081428FDC40F26921A0
:108E800052984843EE4901EB8000807900EB4001A5
:108E900001EB0010E94901EB0010C179BDF83C007D
:108EA00000EB410081B20F9140F269215298484392
:108EB000E34901EB8000807900EB400101EB0010F9
:108EC000DE4901EB0010007F00F003015298C0EB77
:108ED000001000EB8000D84A02EBC002BDF83C0055
:108EE0001154BDF83C00401C81B20F9140F2692141
:108EF00052984843D24901EB8000807900EB400151
:108F000001EB0010CD4901EB0010007FC0F301110F
:108F100040F2692252985043C94A02EB800080799E
:108F200000EB400202EB0010C44A02EB001002E02A
:108F300080E163E163E1007FC0F3810041EA001159
:108F40005298C0EB001000EB8000BB4A02EBC0025D
:108F5000BDF83C001154BDF83C00401C81B20F919B
:108F600000211A9127E040F2692152984843B44900
:108F700001EB8000807900EB400101EB0010AF496C
:108F800001EB00113031BDF8680001EB0010817A6F
:108F90005298C0EB001000EB8000A74A02EBC00221
:108FA000BDF83C30BDF8680018441154BDF86800A5
:108FB000401C81B21A91529800EB400101EB001065
:108FC0009E4901EB0010C179BDF868008142CADCFE
:108FD00040F2692152984843994901EB8000807919
:108FE00000EB400101EB0010944901EB0010C17946
:108FF000BDF83C00084481B20F9140F269215298BB
:1090000048438F4901EB80008079401CC1B240F297
:109010006922529850438A4A02EB8000817140F2E3
:10902000692152984843864901EB800080790428E1
:10903000FFF69DACFEE0834841795298C0EB0010EA
:1090400000EB80007C4A02EBC00041757D4801794D
:109050005298C0EB001000EB800002EBC00081755D
:109060007848C1785298C0EB001000EB800002EB0A
:10907000C000C175734881785298C0EB001000EBB6
:10908000800002EBC00001766E4841785298C0EB38
:10909000001000EB800002EBC000417669481838F0
:1090A000017E5298C0EB001000EB800002EBC00084
:1090B0008176BDF83C00801D81B20F91002140F205
:1090C0006922529850435E4A02EB80004171B1E040
:1090D000B0E0AFE000201A9089E040F26921529898
:1090E0004843574901EB80000830BDF8681001EB98
:1090F000410202EB011110F81100E8B3002240F226
:109100006921529848434E4901EB80010831BDF86E
:10911000680000EB400303EB001001F8102040F260
:10912000692152984843464901EB80010831BDF856
:10913000680000EB400202EB001001EB40004078B9
:1091400001125298C0EB001000EB80003A4A02EB8B
:10915000C002BDF83C001154BDF83C00401C81B277
:109160000F9140F2692152984843354901EB800143
:109170000831BDF8680000E012E000EB400202EBAD
:10918000001001EB400041785298C0EB001000EB5A
:109190008000294A02EBC002BDF83C0011541CE0DB
:1091A000FF215298C0EB001000EB8000224A02EB36
:1091B000C002BDF83C001154BDF83C00401C81B217
:1091C0000F91FF215298C0EB001000EB80001A4A6B
:1091D00002EBC002BDF83C001154BDF83C00401C3D
:1091E00081B20F91BDF86800401C81B21A91BDF8A0
:1091F00068000428FFF671AF1CE01BE01AE00021B4
:109200000F911A9111E00021529800EB4002C2EB3D
:10921000C0100D4A02EBC002BDF868000D301154B9
:10922000BDF86800401C81B21A91BDF8680005289D
:10923000E9DB00BF00BF09E0787100201441002085
:10924000D4450020D4320020D87A0020BDF83C005C
:10925000C01F010A5298C0EB001000EB8000FA4AD0
:1092600002EBC0008173BDF83C00C01FC1B2529830
:10927000C0EB001000EB800002EBC000C1730021C6
:109280001A9123E05298C0EB001000EB8000EE49E9
:1092900001EBC001BDF868001430095C0491DDE900
:1092A0000D210498F0F77BFD01465298C0EB0010A9
:1092B00000EB8000E44A02EBC002BDF86800143005
:1092C0001154BDF86800401C81B21A91BDF83C00F1
:1092D000C01FBDF868108842D4DCDC48C07D98B15E
:1092E000BDF83C00C01F81B204915298C0EB001041
:1092F00000EB8000D44901EBC000C01D00230390A7
:10930000529A0499F1F7C4FBBDF83C00C01F81B22A
:1093100004915298C0EB001000EB8000CA4901EBA9
:10932000C000C01D03900499F0F7B8FA05900598A5
:10933000020A5298C0EB001000EB8000C24901EB1A
:10934000C000BDF83C104254BDF83C00401C80B247
:109350000F900598C2B25298C0EB001000EB80004D
:10936000B94901EBC000BDF83C104254BDF83C00C7
:10937000401C80B20F90BDF83C00401F020A52987A
:10938000C0EB001000EB8000AF4901EBC000C270E1
:10939000BDF83C00401FC2B25298C0EB001000EB79
:1093A000800001EBC0000271BDF83C00401F80B29C
:1093B00004905298C0EB001000EB800001EBC0005D
:1093C000401D0390049912F0ABFF01465298C0EB88
:1093D000001000EB80009C4A02EBC002BDF83C008C
:1093E0001154BDF83C00401C81B20F91529830B12D
:1093F000012815D0022825D0032849D135E0BDF831
:109400003C0060B180219248F1F70CFBBDF83C00B4
:109410009049086001218F48001FF0F7BFFA37E03C
:10942000BDF83C0068B108218948F1F7FBFABDF8A6
:109430003C008849A4394867012186483438F0F750
:10944000ADFA25E0BDF83C0070B14FF48071824860
:10945000F1F7E8FABDF83C007E49183108600121B7
:109460007C481430F0F79AFA12E0BDF83C0070B175
:109470004FF480617648F1F7D5FABDF83C007549A4
:10948000A439C865012173484C38F0F787FA00BF4A
:1094900000BF6E48C07D002805F0E1875298C0EB00
:1094A000001000EB8000684901EBC001002304912B
:1094B000BDF83C10529A0498F1F7EAFA05F0CFBFD4
:1094C0006648007F012805F0F9859DF858000028BE
:1094D000F9D09DF85800092885F07B85DFE810F069
:1094E000F92A09004C09510EC6123C167317482080
:1094F000FB26529800EB400101EB0010584901EBAC
:1095000000113031539801EB001041780846049166
:10951000002106F081FDC1B2159140F269215298F7
:109520004843504901EB8001A431539800EBC0003F
:1095300001EB0010017840F2692252985043494AE9
:1095400002EB80000079814208D1012140F26922BA
:1095500052985043434A02EB8000C17042495298EE
:1095600001EB00115398085C401CC1B23E4A52986E
:1095700002EB00125398115440F26921529848436B
:10958000384901EB8000A430539901EBC10100EB95
:10959000011090F88E00C0F3C00090B1529800EB1B
:1095A000400101EB00102E4901EB001041790B4600
:1095B0004FF4805204914FF4E131529806F01AFCB6
:1095C00019E0529800EB400101EB0010244901EB37
:1095D000001041790491529800EB400101EB00101A
:1095E0001F4901EB0010016803914FF48052049B66
:1095F000529806F0FFFB5498C52876D012DCB528A7
:1096000074D008DC112872D0122871D0132870D0C1
:10961000B22869D1A2E3B6286CD0B9286BD0C32890
:10962000F7D1DEE2D92868D006DCCA287DD0CE2862
:109630007CD0D528EDD119E0E12878D0E52877D085
:10964000E728E6D1E7E3000078710020BC32002073
:10965000000C0240A460024000000240BC12002046
:1096600014410020D4450020483F0020F5215298A5
:10967000C0EB001000EB8000F64A02F830109DF8B5
:1096800054105298C0EB001000EB800002EBC000B9
:109690004170A2215298C0EB001000EB800002EB59
:1096A000C0008170D5215298C0EB001000EB800003
:1096B00002EBC000C1705298C0EB001000EB8000BC
:1096C000114601EBC00104910321049806F080FBD0
:1096D00001465298C0EB001000EB8000DD4A02EB1F
:1096E000C000017105210F91F8E2FDE349E0FCE3C0
:1096F000FCE3FCE3F3E25AE1FFE7F5215298C0EB0B
:10970000001000EB8000D34A02F830109DF854108E
:109710005298C0EB001000EB800002EBC0004170DB
:10972000A2215298C0EB001003E099E2F4E3F4E3C5
:10973000F4E300EB800002EBC0008170D921529865
:10974000C0EB001000EB800002EBC000C17052982B
:10975000C0EB001000EB8000114601EBC00104914A
:109760000321049806F034FB01465298C0EB001028
:1097700000EB8000B74A02EBC000017105210F9198
:10978000B2E7F5215298C0EB001000EB8000B14A1F
:1097900002F830109DF854105298C0EB001000EB06
:1097A000800002EBC0004170529800EB400101EBD9
:1097B0000010A94901EB0010007BA0BB40F2692119
:1097C00052984843A54901EB8000A430539901EB1E
:1097D000C10100EB01108068B0F5100F05D34FF404
:1097E00010000021CDE9100110E040F269215298EB
:1097F00048439A4901EB8000A430539901EBC10121
:1098000000EB011080680022CDE91002A5215298DA
:10981000C0EB001000EB80008E4A02EBC0008170AC
:1098200000211A911FE046E0BDF86800C0F1020077
:10983000C200DDE91010CDE91D0108461D99EEF7C3
:10984000F2FCC1B25298C0EB001000EB8000814ADC
:1098500002EBC002BDF86800C01C1154BDF86800DE
:10986000401C81B21A91BDF868000328DCDBB521E9
:109870005298C0EB001000EB8000764A02EBC0006B
:1098800081715298C0EB001000EB8000114601EB93
:10989000C00104910621049806F09AFA01465298F4
:1098A000C0EB001000EB80006A4A02EBC000C171FF
:1098B00008210F917AE040F26921529848436749A4
:1098C00001EB8000A430539901EBC10100EB0110C2
:1098D0008068B0F1104F05D34FF010400021CDE962
:1098E000100110E040F26921529848435B4901EBB6
:1098F0008000A430539901EBC10100EB0110806896
:109900000022CDE91002A6215298C0EB001000EB16
:109910008000504A02EBC000817000211A911EE0C5
:10992000BDF86800C0F10300C200DDE91010CDE908
:109930001F0108461F99EEF776FCC2B25298C0EBA1
:10994000001000EB8000434901EBC003BDF8680044
:10995000C01C1A54BDF86800401C80B21A90BDF8B3
:1099600068000428DCDBB5215298C0EB001000EB46
:109970008000384A02EBC000C1715298C0EB001061
:1099800000EB8000114601EBC0010491072104980F
:1099900006F01EFA01465298C0EB001000EB800062
:1099A0002C4A02EBC000017209210F919CE6F521BF
:1099B0005298C0EB001000EB8000264A02F83010ED
:1099C0009DF854105298C0EB001000EB800002EBA1
:1099D000C0004170529800EB400101EB00101E499D
:1099E00001EB0010007BA0BB40F269215298484374
:1099F0001A4901EB8000A430539901EBC10100EB3F
:109A000001108068B0F5100F05D14FF4100100204F
:109A1000CDE9101010E040F26921529848430F49F7
:109A200001EB8000A430539901EBC10100EB011060
:109A300080680022CDE91002A5215298C0EB0010E9
:109A400000EB8000034A02EBC000817000211A91F4
:109A500025E04CE07871002014410020D44500201E
:109A6000BDF86800C0F10200C200DDE91010CDE9C8
:109A7000210108462199EEF7D6FBC2B25298C0EBFD
:109A8000001000EB8000F84901EBC003BDF868004E
:109A9000C01C1A54BDF86800401C80B21A90BDF872
:109AA00068000328DCDBB9215298C0EB001000EB02
:109AB0008000ED4A02EBC00081715298C0EB0010AB
:109AC00000EB8000114601EBC001049106210498CF
:109AD00006F07EF901465298C0EB001000EB8000C2
:109AE000E14A02EBC000C17108210F9178E040F219
:109AF000692152984843DD4901EB8000A430539915
:109B000001EBC10100EB01108068B0F1104F05D1ED
:109B10004FF010400021CDE9100110E040F2692122
:109B200052984843D14901EB8000A430539901EB8E
:109B3000C10100EB011080680022CDE91002A621CE
:109B40005298C0EB001000EB8000C74A02EBC00047
:109B5000817000211A911CE0BDF86800C0F103007B
:109B6000C200DDE91001CDE92310EEF75CFBC2B2C3
:109B70005298C0EB001000EB8000BB4901EBC00322
:109B8000BDF86800C01C1A54BDF86800401C80B2C3
:109B90001A90BDF868000428DEDBB9215298C0EBAA
:109BA000001000EB8000B04A02EBC000C171529877
:109BB000C0EB001000EB8000114601EBC0010491E6
:109BC0000721049806F004F901465298C0EB0010F2
:109BD00000EB8000A44A02EBC000017209210F9142
:109BE00082E5F5215298C0EB001000EB80009E4A00
:109BF00002F830109DF854105298C0EB001000EBA2
